:020000040800F2
:1000000000060020E1010008E3010008E301000808
:10001000E3010008E3010008E3010008E301000830
:10002000E3010008E3010008E30100089D2F000838
:10003000E3010008E3010008E3010008E301000810
:10004000E3010008E3010008E3010008E301000800
:10005000E3010008E3010008453200086D320008A2
:1000600095320008BD320008E5320008E3010008BF
:10007000E3010008E3010008E3010008E3010008D0
:10008000E3010008E3010008E3010008E3010008C0
:10009000E3010008E3010008E30100080D33000854
:1000A000E3010008E3010008E3010008E3010008A0
:1000B000E1330008E3010008E3010008E301000860
:1000C000E3010008E3010008E3010008E301000880
:1000D000E3010008E3010008E3010008E301000870
:1000E00071330008E3010008E3010008E3010008A0
:1000F000E3010008E3010008E3010008E301000850
:10010000E3010008E3010008E3010008E30100083F
:10011000E3010008E3010008E3010008E30100082F
:10012000E3010008E3010008E3010008E30100081F
:10013000E3010008E3010008E3010008E30100080F
:10014000E3010008E3010008E3010008512700086B
:10015000E3010008E3010008E3010008E3010008EF
:10016000E3010008E3010008E3010008E3010008DF
:10017000E3010008E3010008E3010008E3010008CF
:10018000E3010008E3010008E3010008E3010008BF
:10019000E3010008E3010008E3010008E3010008AF
:1001A000E3010008E3010008E3010008E30100089F
:1001B000E3010008E3010008E3010008E30100088F
:1001C000E3010008E3010008E3010008E30100087F
:1001D000E3010008E3010008E3010008E30100086F
:1001E00002E000F000F8FEE772B6374880F30888B6
:1001F000364880F3098836483649086040F20000E6
:10020000CCF200004EF63471CEF200010860BFF36C
:100210004F8FBFF36F8F40F20000C0F2F0004EF638
:100220008851CEF200010860BFF34F8FBFF36F8F8C
:100230004FF00000E1EE100A4EF63C71CEF20001E4
:100240000860062080F31488BFF36F8F01F048FF29
:1002500002F042FE4FF055301F491B4A91423CBF0D
:1002600041F8040BFAE71D49184A91423CBF41F896
:10027000040BFAE71A491B4A1B4B9A423EBF51F83E
:10028000040B42F8040BF8E700201849184A914281
:100290003CBF41F8040BFAE701F026FF02F070FEC4
:1002A000144C154DAC4203DA54F8041B8847F9E7A7
:1002B00000F042F8114C124DAC4203DA54F8041B22
:1002C0008847F9E701F00EBF000600200022002059
:1002D0000000000808ED00E00000002000060020FB
:1002E000B0370008002200204022002040220020D9
:1002F000602E0020E0010008E0010008E001000895
:10030000E00100082DE9F04F2DED108AC1F80CD066
:10031000C3689D46BDEC108ABDE8F08F002383F3CF
:1003200011882846A047002001F08AFAFEE701F074
:1003300019FA00DFFEE7000038B500F0BFFB01F05E
:100340009FFE054601F0C2FE0446C8B90E4B9D4211
:1003500018D001339D4218BF044641F2883504BFCE
:1003600001240025002001F095FE0CB100F074F886
:1003700000F018FD284600F0C3F800F06DF8F9E72A
:100380000025EFE70546EDE7010007B008B500F0EE
:1003900067FBA0F120035842584108BD07B541F260
:1003A0001203022101A8ADF8043000F077FB03B07E
:1003B0005DF804FB38B5302383F3118817480368D0
:1003C0000BB101F009FB164A144800234FF47A716F
:1003D00001F0F8FA002383F31188124C236813B15B
:1003E0002368013B2360636813B16368013B63606A
:1003F0000D4D2B7833B963687BB9022000F034FCD3
:10040000322363602B78032B07D163682BB902205A
:1004100000F02AFC4FF47A73636038BD402200205C
:10042000B50300086023002058220020084B1870F4
:1004300003280CD8DFE800F008050208022000F0CD
:1004400003BC022000F0F0BB024B00225A60704750
:100450005822002060230020244B254A10B51C465A
:100460001968013140D004339342F9D16268214BBD
:100470009A4239D9204B9B6803F1006303F580331E
:100480009A4231D2002000F033FB0220FFF7CEFF6A
:100490001A4B1A6C00221A64196E1A66196E596C7E
:1004A0005A64596E5A665A6E5A6942F080025A610D
:1004B0005A6922F080025A615A691A6942F0005260
:1004C0001A611A6922F000521A611B6972B64FF064
:1004D000E0233021C3F8084DD4E9003281F31188BC
:1004E0009D4683F30888104710BD00BF0000010837
:1004F00020000108FFFF0008002200200038024011
:100500002DE9F04F93B0AA4B00902022FF210AA8BA
:100510009D6800F0F1FBA74A1378A3B9A648012112
:1005200003601170302383F3118803680BB101F06D
:1005300053FAA24AA04800234FF47A7101F042FA1C
:10054000002383F31188009B13B19D4B009A1A601E
:100550009C4A009C1378032B1EBF00231370984AFB
:100560004FF0000A18BF5360D3465646D1460120CB
:1005700000F06AFB24B1924B1B68002B00F0118243
:10058000002000F06DFA0390039B002BF2DB0120AA
:1005900000F04AFB039B213B162BE8D801A252F83E
:1005A00023F000BF0106000829060008BD06000868
:1005B0006F0500086F0500086F0500084707000871
:1005C000170900083108000893080008BB08000854
:1005D000E10800086F050008F30800086F0500082F
:1005E00065090008A10600086F050008A9090008B0
:1005F0000D060008A10600086F0500089308000812
:100600000220FFF7C3FE002840F0F581009B022185
:10061000BAF1000F08BF1C4605A841F21233ADF82D
:10062000143000F03BFAA2E74FF47A7000F018FAA9
:10063000071EEBDB0220FFF7A9FE0028E6D0013FF2
:10064000052F00F2DA81DFE807F0030A0D101336F8
:1006500005230593042105A800F020FA17E054486B
:100660000421F9E758480421F6E758480421F3E744
:100670004FF01C08404600F03DFA08F104080590D0
:10068000042105A800F00AFAB8F12C0FF2D10120DC
:1006900000FA07F747EA0B0B5FFA8BFB4FF00009F4
:1006A00000F076FB26B10BF00B030B2B08BF0024E8
:1006B000FFF774FE5BE746480421CDE7002EA5D086
:1006C0000BF00B030B2BA1D10220FFF75FFE0746B7
:1006D00000289BD0012000F00BFA0220FFF7A6FEB5
:1006E00000261FFA86F8404600F012FA044690B140
:1006F0000021404600F01CFA01360028F1D1BA462C
:10070000044641F21213022105A8ADF814303E460A
:1007100000F0C4F92BE70120FFF788FE2546244BA3
:100720009B68AB4207D9284600F0E4F9013040F05D
:1007300067810435F3E7234B00251D70204BBA4633
:100740005D603E46ACE7002E3FF460AF0BF00B035C
:100750000B2B7FF45BAF0220FFF768FE322000F026
:100760007FF9B0F10008FFF651AF18F003077FF4EE
:100770004DAF0F4A926808EB050393423FF646AF30
:10078000B8F5807F3FF742AF124B0193B84523DDA8
:100790004FF47A7000F064F90390039A002AFFF690
:1007A00035AF019B039A03F8012B0137EDE700BF3A
:1007B000002200205C23002040220020B503000816
:1007C000602300205822002004220020082200205C
:1007D0000C2200205C220020C820FFF7D7FD07462E
:1007E00000283FF413AF1F2D11D8C5F12002424558
:1007F0000AAB25F0030028BF424683490192184402
:1008000000F054FA019A8048FF2100F075FA4FEA8F
:10081000A8037D490193C8F38702284600F074FAC3
:10082000064600283FF46DAF019B05EB830537E7D3
:100830000220FFF7ABFD00283FF4E8AE00F0A4F97A
:1008400000283FF4E3AE0027B846704B9B68BB42DC
:1008500018D91F2F11D80A9B01330ED027F003039C
:1008600012AA134453F8203C05934046042205A9DC
:1008700000F0C2FA04378046E7E7384600F03AF95C
:100880000590F2E7CDF81480042105A800F006F9E0
:1008900006E70023642104A8049300F0F5F800287B
:1008A0007FF4B4AE0220FFF771FD00283FF4AEAE36
:1008B000049800F051F90590E6E70023642104A8AC
:1008C000049300F0E1F800287FF4A0AE0220FFF7C7
:1008D0005DFD00283FF49AAE049800F04DF9EAE778
:1008E0000220FFF753FD00283FF490AE00F05CF9C2
:1008F000E1E70220FFF74AFD00283FF487AE05A993
:10090000142000F057F904210746049004A800F0D1
:10091000C5F83946B9E7322000F0A2F8071EFFF605
:1009200075AEBB077FF472AE384A926807EB0903D5
:1009300093423FF66BAE0220FFF728FD00283FF4FC
:1009400065AE27F003074F44B9453FF4A9AE4846CA
:1009500000F0D0F80421059005A800F09FF809F1F7
:100960000409F1E74FF47A70FFF710FD00283FF417
:100970004DAE00F009F9002844D00A9B01330BD09A
:1009800008220AA9002000F0BFF900283AD020224E
:10099000FF210AA800F0B0F9FFF700FD1C4800F0A5
:1009A00055FF13B0BDE8F08F002E3FF42FAE0BF0D3
:1009B0000B030B2B7FF42AAE0023642105A80593BB
:1009C00000F062F8074600287FF420AE0220FFF70F
:1009D000DDFC804600283FF419AEFFF7DFFC41F252
:1009E000883000F033FF059800F004FA464600F026
:1009F000CFF93C46BBE5064652E64FF0000905E656
:100A0000BA467EE637467CE65C22002000220020C3
:100A1000A086010070B50F4B1B780133DBB2012BB0
:100A20000C4611D80C4D29684FF47A730E6AA2FB5C
:100A30000332014622462846B047844204D1074B80
:100A400000221A70012070BD4FF4FA7000F0FEFE13
:100A50000020F8E710220020082600209423002020
:100A600007B50023024601210DF107008DF807307C
:100A7000FFF7D0FF20B19DF8070003B05DF804FB3D
:100A80004FF0FF30F9E700000A4608B50421FFF7F0
:100A9000C1FF80F00100C0B2404208BD30B4054C37
:100AA0002368DD69044B0A46AC460146204630BC4B
:100AB000604700BF08260020A086010070B501F045
:100AC000E5F9094E094D30800024286833888342B7
:100AD00008D901F0D5F92B6804440133B4F5803FFF
:100AE0002B60F2D370BD00BF962300206823002046
:100AF00001F07ABA00F1006000F5803000687047BC
:100B000000F10060920000F5803001F005BA0000AD
:100B1000054B1A68054B1B889B1A834202D9104467
:100B200001F0AEB900207047682300209623002012
:100B300038B5084D044629B128682044BDE838403E
:100B400001F0BEB92868204401F0A2F90028F3D0D2
:100B500038BD00BF6823002010F003030AD1B0F5B0
:100B6000047F05D200F10050A0F51040D0F8003805
:100B7000184670470023FBE700F10050A0F5104035
:100B8000D0F8100A70470000064991F8243033B1BC
:100B90000023086A81F824300822FFF7B1BF012042
:100BA000704700BF6C230020014B1868704700BFDE
:100BB000002004E070B5194B1D68194B0138C5F3CE
:100BC0000B0408442D0C04221E88A6420BD15C683D
:100BD0000A46013C824213460FD214F9016F4EB10E
:100BE00002F8016BF6E7013A03F10803ECD1814208
:100BF0000B4602D22C2203F8012B0A4A0524168840
:100C0000AE4204D1984284BF967803F8016B013C50
:100C100002F10402F3D1581A70BD00BF002004E0B5
:100C2000C4340008B0340008022804D1054B4FF04A
:100C300080429A6170470128FCD1024B4FF000526C
:100C4000F7E700BF00000240022804D1054B4FF433
:100C500080429A6170470128FCD1024B4FF4005248
:100C6000F7E700BF00000240022805D1064A536999
:100C700083F48043536170470128FCD1024A5369D1
:100C800083F40053F6E700BF0000024070B504464D
:100C90004FF47A764CB1412C254628BF412506FBFE
:100CA00005F000F0D3FD641BF4E770BD10B5002320
:100CB000934203D0CC5CC4540133F9E710BD00006B
:100CC00010B5013810F9013F3BB191F900409C4249
:100CD00003D11AB10131013AF4E71AB191F90020B8
:100CE000981A10BD1046FCE703460246D01A12F9C6
:100CF000011B0029FAD1704702440346934202D0F7
:100D000003F8011BFAE770472DE9F8431F4D14461D
:100D100095F824200746884652BBDFF870909CB3B4
:100D200095F824302BB92022FF2148462F62FFF787
:100D3000E3FF95F82400C0F10802A24228BF224632
:100D4000D6B24146920005EB8000FFF7AFFF95F861
:100D50002430A41B1E44F6B2082E17449044E4B27B
:100D600085F82460DBD1FFF70FFF0028D7D108E01A
:100D70002B6A03EB82038342CFD0FFF705FF0028E5
:100D8000CBD10020BDE8F8830120FBE76C230020D5
:100D9000024B1A78024B1A70704700BF9423002050
:100DA0001022002010B5104C104800F0B5F8214674
:100DB0000E4800F0DDF82468626DD2F8043843F084
:100DC0000203C2F804384FF47A70FFF75FFF084956
:100DD000204600F0D3F9626DD2F8043823F0020304
:100DE000C2F8043810BD00BF903500080826002066
:100DF000983500087047000030B5094D0A4491420B
:100E00000DD011F8013B5840082340F30004013B8A
:100E10002C4013F0FF0384EA5000F6D1EFE730BD19
:100E20002083B8ED026843681143016003B118479D
:100E30007047000013B5446BD4F894341A681178E5
:100E4000042915D1217C022912D119791289012393
:100E50008B4013420CD101A904F14C0001F0F8FEC3
:100E6000D4F89444019B21790246206800F0D0F91F
:100E700002B010BD143001F07BBE00004FF0FF3314
:100E8000143001F075BE00004C3001F04DBF000081
:100E90004FF0FF334C3001F047BF0000143001F039
:100EA00049BE00004FF0FF31143001F043BE000096
:100EB0004C3001F019BF00004FF0FF324C3001F010
:100EC00013BF00000020704710B5D0F894341A68A2
:100ED00011780429044617D1017C022914D15979CB
:100EE000528901238B4013420ED1143001F0DCFDF6
:100EF000024648B1D4F894444FF480736179206875
:100F0000BDE8104000F072B910BD0000406BFFF763
:100F1000DBBF0000704700007FB5124B0360002369
:100F20004360C0E90233012502260F4B05740446D5
:100F30000290019300F18402294600964FF48073D9
:100F4000143001F08DFD094B0294CDE9006304F5E6
:100F500023724FF48073294604F14C0001F054FED3
:100F600004B070BDE43400080D0F0008350E000811
:100F70000B68302282F311880A7903EB82029061B8
:100F80004A79093243F822008A7912B103EB8203CD
:100F900098610223C0F894140374002080F3118830
:100FA0007047000038B5037F044613B190F8543001
:100FB000ABB9201D01250221FFF734FF04F1140015
:100FC00025776FF0010100F069FC84F8545004F1BA
:100FD0004C006FF00101BDE8384000F05FBC38BD47
:100FE00010B5012104460430FFF71CFF00232377CE
:100FF00084F8543010BD000038B504460025143084
:1010000001F046FD04F14C00257701F015FE201D8E
:1010100084F854500121FFF705FF2046BDE8384011
:10102000FFF752BF90F8443003F06003202B07D144
:1010300090F84520212A4FF0000303D81F2A06D834
:1010400000207047222AFBD1C0E90E3303E0034A97
:1010500082630722C26303640120704711220020CB
:1010600037B5D0F894341A681178042904461AD197
:10107000017C022917D11979128901238B4013426F
:1010800011D100F14C05284601F096FE58B101A996
:10109000284601F0DDFDD4F89444019B21790246F5
:1010A000206800F0B5F803B030BD0000F0B500EBEB
:1010B000810385B09E6904460D46FEB1302383F35B
:1010C000118804EB8507301D0821FFF7ABFEFB6894
:1010D0005B691B6806F14C001BB1019001F0C6FD75
:1010E000019803A901F0B4FD024648B1039B2946CB
:1010F000204600F08DF8002383F3118805B0F0BD81
:10110000FB685A691268002AF5D01B8A013B13401C
:10111000F1D104F14402EAE7093138B550F8214031
:10112000DCB1302383F31188D4F894241368527906
:1011300003EB8203DB689B695D6845B1042160189D
:10114000FFF770FE294604F1140001F0B7FC2046B9
:10115000FFF7BAFE002383F3118838BD7047000003
:1011600001F016B8012303700023C0E90133C36105
:1011700083620362C36243620363704738B5044607
:10118000302383F311880025C0E90355C0E90555D4
:10119000416001F00DF80223237085F31188284681
:1011A00038BD000070B500EB810305465069DA6078
:1011B0000E46144618B110220021FFF79DFDA069CC
:1011C00018B110220021FFF797FD31462846BDE8EF
:1011D000704001F0B7B80000826802F0011282602E
:1011E0000022C0E90422826101F038B9F0B400EBBA
:1011F00081044789E4680125A4698D403D43458108
:1012000023600023A2606360F0BC01F053B90000CA
:10121000F0B400EB81040789E468012564698D401E
:101220003D43058123600023A2606360F0BC01F0B0
:10123000CDB9000070B50223002504460370C0E953
:101240000255C0E90455C564856180F8345001F049
:1012500015F863681B6823B129462046BDE8704035
:10126000184770BD0378052B10B504460AD080F8E6
:1012700050300523037043681B680BB10421984765
:101280000023A36010BD00000178052906D190F865
:101290005020436802701B6803B118477047000074
:1012A00070B590F83430044613B1002380F8343020
:1012B00004F14402204601F0F3F863689B68B3B977
:1012C00094F8443013F0600535D00021204601F039
:1012D00093FB0021204601F085FB63681B6813B176
:1012E000062120469847062384F8343070BD2046F6
:1012F00098470028E4D0B4F84A30E26B9A4288BF9D
:10130000E36394F94430E56B002B4FF0300380F237
:101310000381002D00F0F280092284F8342083F349
:1013200011880021D4E90E232046FFF771FF002326
:1013300083F31188DAE794F8452003F07F0343EA4A
:10134000022340F20232934200F0C58021D8B3F567
:10135000807F48D00DD8012B3FD0022B00F0938026
:10136000002BB2D104F14C02A2630222E263236497
:10137000C1E7B3F5817F00F09B80B3F5407FA4D136
:1013800094F84630012BA0D1B4F84C3043F002035E
:1013900032E0B3F5006F4DD017D8B3F5A06F31D060
:1013A000A3F5C063012B90D8636894F846205E686B
:1013B00094F84710B4F848302046B047002884D04D
:1013C0004368A3630368E3631AE0B3F5106F36D094
:1013D00040F6024293427FF478AF5C4BA363022352
:1013E000E3630023C3E794F84630012B7FF46DAF2D
:1013F000B4F84C3023F00203C4E90E55A4F84C3085
:10140000256478E7B4F84430B3F5A06F0ED194F8B2
:10141000463084F84E30204600F088FF63681B6831
:1014200013B1012120469847032323700023C4E908
:101430000E339CE704F14F03A3630123C3E7237832
:10144000042B10D1302383F311882046FFF7C4FE0C
:1014500085F311880321636884F84F5021701B685D
:101460000BB12046984794F84630002BDED084F824
:101470004F300423237063681B68002BD6D00221F1
:1014800020469847D2E794F848301D0603F00F0134
:1014900020460AD500F0F6FF012804D002287FF488
:1014A00014AF2B4B9AE72B4B98E700F0DDFFF3E7E7
:1014B00094F84630002B7FF408AF94F8483013F0CE
:1014C0000F01B3D01A06204602D501F0A9FAADE704
:1014D00001F09CFAAAE794F84630002B7FF4F5AEB1
:1014E00094F8483013F00F01A0D01B06204602D517
:1014F00001F082FA9AE701F075FA97E7142284F86E
:10150000342083F311882B462A4629462046FFF7CC
:101510006DFE85F31188E9E65DB1152284F834206B
:1015200083F311880021D4E90E232046FFF75EFEE5
:10153000FDE60B2284F8342083F311882B462A46DB
:1015400029462046FFF764FEE3E700BF1435000894
:101550000C3500081035000838B590F834300446D2
:10156000002B3ED0063BDAB20F2A34D80F2B32D8EC
:10157000DFE803F037313108223231313131313196
:1015800031313737C56BB0F84A309D4214D2C36849
:101590001B8AB5FBF3F203FB12556DB9302383F3BD
:1015A00011882B462A462946FFF732FE85F311881B
:1015B0000A2384F834300EE0142384F834303023C6
:1015C00083F3118800231A4619462046FFF70EFEC2
:1015D000002383F3118838BD036C03B198470023BF
:1015E000E7E70021204601F007FA0021204601F03C
:1015F000F9F963681B6813B1062120469847062352
:10160000D7E7000010B590F83430142B044629D0E9
:1016100017D8062B05D001D81BB110BD093B022BF2
:10162000FBD80021204601F0E7F90021204601F017
:10163000D9F963681B6813B1062120469847062331
:1016400019E0152BE9D10B2380F83430302383F3D4
:10165000118800231A461946FFF7DAFD002383F3A9
:101660001188DAE7C3689B695B68002BD5D1036CEE
:1016700003B19847002384F83430CEE70023037584
:10168000826803691B6899689142FBD25A680360BB
:1016900042601060586070470023037582680369D8
:1016A0001B6899689142FBD85A68036042601060D9
:1016B0005860704708B50846302383F311880B7DC6
:1016C000032B05D0042B0DD02BB983F3118808BD53
:1016D0008B6900221A604FF0FF338361FFF7CEFF62
:1016E0000023F2E7D1E9003213605A60F3E700000B
:1016F000FFF7C4BF054BD9680875186802681A60FF
:10170000536001220275D860FEF7FCBD98230020CB
:1017100030B50C4BDD684B1C87B004460FD02B4610
:10172000094A684600F04EF92046FFF7E3FF009BA8
:1017300013B1684600F050F9A86907B030BDFFF753
:10174000D9FFF9E798230020B5160008044B1A6862
:10175000DB6890689B68984294BF00200120704726
:1017600098230020084B10B51C68D86822681A60BE
:10177000536001222275DC60FFF78EFF0146204690
:10178000BDE81040FEF7BEBD9823002038B5074CD9
:1017900007490848012300252370656001F044FBD8
:1017A0000223237085F3118838BD00BF0026002076
:1017B0001C3500089823002000F044B9034A516802
:1017C00053685B1A9842FBD8704700BF001000E0D6
:1017D0008B60022308618B82084670478368A3F1FF
:1017E000840243F8142C026943F8442C426943F8FC
:1017F000402C094A43F8242CC26843F8182C0222D2
:1018000003F80C2C002203F80B2C044A43F8102C8C
:10181000A3F12000704700BF1D030008982300209B
:1018200008B5FFF7DBFFBDE80840FFF761BF000028
:10183000024BDB6898610F20FFF75CBF9823002004
:10184000302383F31188FFF7F3BF000008B501468A
:10185000302383F311880820FFF75AFF002383F316
:10186000118808BD064BDB6839B1426818605A60C0
:10187000136043600420FFF74BBF4FF0FF30704709
:10188000982300200368984206D01A6802605060CE
:1018900099611846FFF72CBF7047000038B5044621
:1018A0000D462068844200D138BD036823605C6027
:1018B0008561FFF71DFFF4E710B503689C68A2423D
:1018C0000CD85C688A600B604C6021605960996834
:1018D0008A1A9A604FF0FF33836010BD1B68121B99
:1018E000ECE700000A2938BF0A2170B504460D460E
:1018F0000A26601901F092FA01F07EFA041BA54253
:1019000003D8751C2E460446F3E70A2E04D9BDE819
:101910007040012001F0C8BA70BD0000F8B5144B4A
:101920000D46D96103F1100141600A2A19698260EC
:1019300038BF0A22016048601861A818144601F0F7
:101940005FFA0A2701F058FA431BA342064606D362
:101950007C1C281901F062FA27463546F2E70A2F67
:1019600004D9BDE8F840012001F09EBAF8BD00BFDF
:1019700098230020F8B506460D4601F03DFA0F4ABF
:10198000134653F8107F9F4206D12A46014630463F
:10199000BDE8F840FFF7C2BFD169BB68441A2C19F3
:1019A00028BF2C46A34202D92946FFF79BFF2246B7
:1019B00031460348BDE8F840FFF77EBF982300207A
:1019C000A823002010B4C0E9032300235DF8044BD2
:1019D0004361FFF7CFBF000010B5194C236998424F
:1019E0000DD0D0E90032816813605A609A680A44C9
:1019F0009A60002303604FF0FF33A36110BD2346BC
:101A0000026843F8102F53600022026022699A4254
:101A100003D1BDE8104001F0FBB9936881680B4425
:101A2000936001F0E9F92269E1699268441AA242DF
:101A3000E4D91144BDE81040091AFFF753BF00BFB5
:101A4000982300202DE9F047DFF8BC8008F110074B
:101A50002C4ED8F8105001F0CFF9D8F81C40AA68E5
:101A6000031B9A423ED81444D5E900324FF00009D6
:101A7000C8F81C4013605A60C5F80090D8F81030C0
:101A8000B34201D101F0C4F989F31188D5E90331DA
:101A900028469847302383F311886B69002BD8D0F0
:101AA00001F0AAF96A69A0EB04094A4582460DD201
:101AB000022001F0F9F90022D8F81030B34208D121
:101AC00051462846BDE8F047FFF728BF121A2244C6
:101AD000F2E712EB090938BF4A4629463846FFF7B4
:101AE000EBFEB5E7D8F81030B34208D01444211A01
:101AF000C8F81C00A960BDE8F047FFF7F3BEBDE8D9
:101B0000F08700BFA8230020982300200020704702
:101B1000FEE70000704700004FF0FF307047000004
:101B200002290CD0032904D00129074818BF00203E
:101B30007047032A05D8054800EBC20070470448E7
:101B400070470020704700BFF435000820220020B5
:101B5000A835000870B59AB00546084601A9144694
:101B600000F0C2F801A8FFF7BFF8431C5B00C5E90D
:101B700000340022237003236370C6B201AB023429
:101B80001046D1B28E4204F1020401D81AB070BDE1
:101B900013F8011B04F8021C04F8010C0132F0E7F1
:101BA00008B5302383F311880348FFF759FA00235F
:101BB00083F3118808BD00BF0826002090F8443048
:101BC00003F01F02012A07D190F845200B2A03D108
:101BD0000023C0E90E3315E003F06003202B08D189
:101BE000B0F848302BB990F84520212A03D81F2A95
:101BF00004D8FFF717BA222AEBD0FAE7034A826328
:101C00000722C26303640120704700BF182200202E
:101C100007B5052917D8DFE801F0191603191920AF
:101C2000302383F31188104A01900121FFF7BAFA9B
:101C300001980E4A0221FFF7B5FA0D48FFF7DCF9CB
:101C4000002383F3118803B05DF804FB302383F392
:101C500011880748FFF7A6F9F2E7302383F31188CC
:101C60000348FFF7BDF9EBE7483500086C3500087D
:101C70000826002038B50C4D0C4C0D492A4604F1BD
:101C80000800FFF767FF05F1CA0204F110000949D7
:101C9000FFF760FF05F5CA7204F118000649BDE8B8
:101CA0003840FFF757BF00BFD02A00202022002075
:101CB00028350008323500083D35000870B5044667
:101CC00008460D46FFF710F8C6B2204601340378E7
:101CD0000BB9184670BD32462946FEF7F1FF0028C1
:101CE000F3D10120F6E700002DE9F04705460C4648
:101CF000FEF7FAFF2B49C6B22846FFF7DFFF08B10F
:101D00000E36F6B228492846FFF7D8FF08B110363C
:101D1000F6B2632E0BD8DFF88C80DFF88C90234F5F
:101D2000DFF894A02E7846B92670BDE8F0872946E2
:101D30002046BDE8F04701F09DBB252E2ED107229D
:101D400041462846FEF7BCFF70B9194B224603F105
:101D5000140153F8040B42F8040B8B42F9D11B78A1
:101D6000137007351534DDE7082249462846FEF78B
:101D7000A7FF98B90F4BA21C197809090232C95D57
:101D800002F8041C13F8011B01F00F015345C95D53
:101D900002F8031CF0D118340835C3E704F8016BCE
:101DA0000135BFE7143600083D350008323600081B
:101DB0001C360008107AFF1F1C7AFF1FBFF34F8FDD
:101DC000024AD368DB03FCD4704700BF003C0240EA
:101DD00008B5094B1B7873B9FFF7F0FF074B1A6979
:101DE000002ABFBF064A5A6002F188325A601A6858
:101DF00022F480621A6008BD2E2D0020003C0240B3
:101E00002301674508B50B4B1B7893B9FFF7D6FF45
:101E1000094B1A6942F000421A611A6842F4805272
:101E20001A601A6822F480521A601A6842F48062BA
:101E30001A6008BD2E2D0020003C02400B28F0B592
:101E400016D80C4C0C4923787BB90C4D0E460C234C
:101E50004FF0006255F8047B46F8042B013B13F069
:101E6000FF033A44F6D10123237051F82000F0BD5E
:101E70000020FCE7602D0020302D002044360008B3
:101E8000014B53F820007047443600080C2070477F
:101E90000B2810B5044601D9002010BDFFF7CEFF76
:101EA000064B53F824301844C21A0BB90120F4E74A
:101EB00012680132F0D1043BF6E700BF4436000857
:101EC0000B2810B5044621D8FFF778FFFFF780FFF5
:101ED0000F4AF323D360C300DBB243F4007343F033
:101EE00002031361136943F480331361FFF766FF44
:101EF000FFF7A4FF074B53F8241000F0D9F8FFF7C1
:101F000081FF2046BDE81040FFF7C2BF002010BD92
:101F1000003C024044360008F8B512F001031446B4
:101F200042D18218B2F1016F57D82D4B1B6813F0C4
:101F3000010352D02B4DFFF74BFFF323EB60FFF76C
:101F40003DFF40F20127032C15D824F00104661848
:101F5000244C401A40F20117B142236900EB0105FD
:101F600024D123F001032361FFF74CFF0120F8BDCA
:101F7000043C0430E7E78307E7D12B6923F440737F
:101F80002B612B693B432B6151F8046B0660BFF357
:101F90004F8FFFF713FF03689E42E9D02B6923F0B0
:101FA00001032B61FFF72EFF0020E0E723F44073CD
:101FB000236123693B4323610B882B80BFF34F8F41
:101FC000FFF7FCFE2D8831F8023BADB2AB42C3D027
:101FD000236923F001032361E4E71846C7E700BF44
:101FE00000380240003C0240084908B50B7828B18F
:101FF0001BB9FFF7EDFE01230B7008BD002BFCD0D1
:10200000BDE808400870FFF7FDBE00BF2E2D002080
:1020100010B50244064BD2B2904200D110BD441C10
:1020200000B253F8200041F8040BE0B2F4E700BF1F
:10203000502800400F4B30B51C6F240407D41C6F90
:1020400044F400741C671C6F44F400441C670A4C81
:10205000236843F4807323600244084BD2B2904259
:1020600000D130BD441C00B251F8045B43F820504D
:10207000E0B2F4E700380240007000405028004011
:1020800007B5012201A90020FFF7C2FF019803B0A4
:102090005DF804FB13B50446FFF7F2FFA04205D03C
:1020A000012201A900200194FFF7C4FF02B010BD76
:1020B00070470000034B1A681AB9034AD2F8742813
:1020C0001A607047642D00200030024008B5FFF709
:1020D000F1FF024B1868C0F3407008BD642D00206A
:1020E00070470000FEE700000A4B0B480B4A904285
:1020F0000BD30B4BDA1C121AC11E22F003028B42C7
:1021000038BF00220021FEF7F7BD53F8041B40F84A
:10211000041BECE7F0370008602E0020602E002042
:10212000602E002070B5D0E915439E6800224FF064
:10213000FF3504EB42135101D3F800090028BEBF5C
:10214000D3F8000940F08040C3F80009D3F8000B31
:102150000028BEBFD3F8000B40F08040C3F8000B4E
:10216000013263189642C3F80859C3F8085BE0D2FD
:102170004FF00113C4F81C3870BD0000890141F014
:102180002001016103699B06FCD41220FFF716BBF6
:1021900010B5054C2046FEF7E5FF4FF0A043636500
:1021A000024BA36510BD00BF682D002098360008C3
:1021B00070B50378012B054650D12A4B446D9842E7
:1021C0001BD1294B5A6B42F080025A635A6D42F080
:1021D00080025A655A6D5A6942F080025A615A6902
:1021E00022F080025A610E2143205B6900F022FC3C
:1021F0001E4BE3601E4BC4F800380023C4F8003EB9
:10220000C02323606E6D4FF40413A3633369002B66
:10221000FCDA012333610C20FFF7D0FA3369DB07C6
:10222000FCD41220FFF7CAFA3369002BFCDA00262F
:10223000A6602846FFF776FF6B68C4F81068DB6875
:10224000C4F81468C4F81C684BB90A4BA3614FF07A
:10225000FF336361A36843F00103A36070BD064BC5
:10226000F4E700BF682D0020003802404014004011
:1022700003002002003C30C0083C30C0F8B5446D7B
:10228000054600212046FFF779FFA96D00234FF096
:1022900001128F68C4F834384FF00066C4F81C2867
:1022A0004FF0FF3004EB431201339F42C2F8006944
:1022B000C2F8006BC2F80809C2F8080BF2D20B682A
:1022C0006A6DEB65636210231361166916F01006E0
:1022D000FBD11220FFF772FAD4F8003823F4FE6322
:1022E000C4F80038A36943F4402343F01003A3610A
:1022F0000923C4F81038C4F814380A4BEB604FF0C7
:10230000C043C4F8103B084BC4F8003BC4F8106944
:10231000C4F80039EB6D03F1100243F48013EA6551
:10232000A362F8BD7436000840800010426D90F83A
:102330004E10D2F8003823F4FE6343EA0113C2F8CA
:10234000003870472DE9F84300EB8103456DDA68EA
:10235000166806F00306731E022B05EB41130C46AC
:1023600080460FFA81F94FEA41104FF00001C3F89F
:10237000101B4FF0010104F1100398BFB60401FADD
:1023800003F391698EBF334E06F1805606F5004681
:1023900000293AD0578A04F15801490137436F5058
:1023A000D5F81C180B43C5F81C382B180021C3F8AE
:1023B000101953690127611EA7409BB3138A928BA2
:1023C0009B08012A88BF5343D8F85C20981842EA3A
:1023D000034301F1400205EB8202C8F85C0021468C
:1023E00053602846FFF7CAFE08EB8900C3681B8AC2
:1023F00043EA8453483464011E432E51D5F81C38F7
:102400001F43C5F81C78BDE8F88305EB4917D7F8DA
:10241000001B21F40041C7F8001BD5F81C1821EA65
:102420000303C0E704F13F0305EB83030A4A5A6044
:1024300028462146FFF7A2FE05EB4910D0F80039E7
:1024400023F40043C0F80039D5F81C3823EA070705
:10245000D7E700BF0080001000040002826D126800
:10246000C265FFF75FBE00005831436D49015B58FC
:1024700013F4004004D013F4001F0CBF022001200D
:10248000704700004831436D49015B5813F4004028
:1024900004D013F4001F0CBF02200120704700007D
:1024A00000EB8101CB68196A0B6813604B685360BD
:1024B0007047000000EB810330B5DD68AA6913683E
:1024C000D36019B9402B84BF402313606B8A146812
:1024D000426D1C44013CB4FBF3F46343033323F02B
:1024E000030302EB411043EAC44343F0C043C0F886
:1024F000103B2B6803F00303012B09B20ED1D2F875
:10250000083802EB411013F4807FD0F8003B14BF71
:1025100043F0805343F00053C0F8003B02EB4112FC
:10252000D2F8003B43F00443C2F8003B30BD00004A
:102530002DE9F041244D6E6D06EB40130446D3F8AF
:10254000087BC3F8087B38070AD5D6F81438190772
:1025500006D505EB84032146DB6828465B6898476F
:10256000FA071FD5D6F81438DB071BD505EB840313
:10257000D968CCB98B69488A5A68B2FBF0F600FB7F
:1025800016228AB91868DA6890420DD2121AC3E985
:102590000024302383F311880B482146FFF78AFF7C
:1025A00084F31188BDE8F081012303FA04F26B89FA
:1025B00023EA02036B81CB68002BF3D0214602484B
:1025C000BDE8F041184700BF682D002000EB8103F3
:1025D00070B5DD68436D6C692668E6604A0156BBDC
:1025E0001A444FF40020C2F810092A6802F00302CE
:1025F000012A0AB20ED1D3F8080803EB421410F4F2
:10260000807FD4F8000914BF40F0805040F00050A3
:10261000C4F8000903EB4212D2F8000940F004406C
:10262000C2F80009D3F83408012202FA01F101438B
:10263000C3F8341870BD19B9402E84BF4020206003
:1026400020682E8A8419013CB4FBF6F440EAC440A9
:1026500040F000501A44C6E72DE9F8433B4D6E6D3B
:1026600006EB40130446D3F80889C3F8088918F02C
:10267000010F4FEA40171AD0D6F81038DB0716D5ED
:1026800005EB8003D9684B691868DA68904230D24C
:10269000121A4FF000091A60C3F80490302383F334
:1026A000118821462846FFF791FF89F3118818F019
:1026B000800F1CD0D6F834380126A640334216D0FD
:1026C00005EB84036D6DD3F80CC0DCF814200134E5
:1026D000E4B2D2F800E005EB04342F4451687145B0
:1026E00015D3D5F8343823EA0606C5F83468BDE8B2
:1026F000F883012303FA04F22B8923EA02032B81D6
:102700008B68002BD3D0214628469847CFE7BCF8EA
:102710001000AEEB0103834228BF0346D7F8180927
:1027200080B2B3EB800FE2D89068A0F1040959F8A9
:10273000048FC4F80080A0EB09089844B8F1040F96
:10274000F5D818440B4490605360C7E7682D00200B
:102750002DE9F74FA24C656D6E69AB691E4016F40A
:1027600080586E6107D02046FEF764FD03B0BDE8D7
:10277000F04F00F047BC002E12DAD5F8003E984822
:102780009B071EBFD5F8003E23F00303C5F8003EAB
:10279000D5F8043823F00103C5F80438FEF774FDBA
:1027A000370505D58E48FFF7BDFC8D48FEF75AFD6D
:1027B000B0040CD5D5F8083813F0060FEB6823F4F5
:1027C00070530CBF43F4105343F4A053EB60310734
:1027D0001BD56368DB681BB9AB6923F00803AB61E9
:1027E0002378052B0CD1D5F8003E7D489A071EBFF3
:1027F000D5F8003E23F00303C5F8003EFEF744FD84
:102800006368DB680BB176489847F30274D4B7026B
:1028100027D5D4F85490DFF8C8B100274FF0010A4B
:1028200009EB4712D2F8003B03F44023B3F5802FA5
:1028300011D1D2F8003B002B0DDA62890AFA07F3B6
:1028400022EA0303638104EB8703DB68DB6813B1CF
:10285000394658469847A36D01379B68FFB29F429F
:10286000DED9F00617D5676D3A6AC2F30A1002F096
:102870000F0302F4F012B2F5802F00F08580B2F55C
:10288000402F08D104EB83030022DB681B6A07F5A5
:10289000805790426AD13003D5F8184813D5E10328
:1028A00002D50020FFF744FEA20302D50120FFF766
:1028B0003FFE630302D50220FFF73AFE270302D54D
:1028C0000320FFF735FE75037FF550AFE00702D513
:1028D0000020FFF7C1FEA10702D50120FFF7BCFED3
:1028E000620702D50220FFF7B7FE23077FF53EAF50
:1028F0000320FFF7B1FE39E7636DDFF8E4A0019331
:1029000000274FF00109A36D9B685FFA87FB9B4589
:102910003FF67DAF019B03EB4B13D3F8001901F495
:102920004021B1F5802F1FD1D3F8001900291BDAFF
:10293000D3F8001941F09041C3F80019D3F80019F9
:102940000029FBDB5946606DFFF718FC218909FA65
:102950000BF321EA0303238104EB8B03DB689B6801
:1029600013B15946504698470137CCE7910708BF45
:10297000D7F80080072A98BF03F8018B02F1010203
:1029800098BF4FEA182884E7023304EB830207F567
:1029900080575268D2F818C0DCF80820DCE9001C27
:1029A000A1EB0C0C002188420AD104EB830463687C
:1029B0009B699A6802449A605A6802445A606AE7BE
:1029C00011F0030F08BFD7F800808C4588BF02F8CC
:1029D000018B01F1010188BF4FEA1828E3E700BF2E
:1029E000682D0020436D03EB4111D1F8003B43F407
:1029F0000013C1F8003B7047436D03EB4111D1F860
:102A0000003943F40013C1F800397047436D03EBFC
:102A10004111D1F8003B23F40013C1F8003B70478B
:102A2000436D03EB4111D1F8003923F40013C1F8D1
:102A30000039704700F1604303F561430901C9B2F1
:102A400083F80013012200F01F039A4043099B0002
:102A500003F1604303F56143C3F880211A607047B6
:102A600030B5039C0172043304FB0325C0E906530F
:102A7000049B03630021059BC160C0E90000C0E91D
:102A80000422C0E90842C0E90A11436330BD0000D6
:102A9000416A0022C0E90411C0E90A22C2606FF055
:102AA0000101FEF7FBBE0000D0E90432934201D1E0
:102AB000C2680AB9181D7047002070470369196081
:102AC000C2680132C260C2691344826903619342E1
:102AD00024BF436A03610021FEF7D4BE38B5044623
:102AE0000D46E3683BB16269131D1268A36213448B
:102AF000E362002007E0237A33B929462046FEF737
:102B0000B1FE0028EDDA38BD6FF00100FBE70000F0
:102B1000C368C269013BC36043691344826943616E
:102B2000934224BF436A436100238362036B03B172
:102B30001847704770B53023044683F31188866ABE
:102B40003EB9FFF7CBFF054618B186F3118828463A
:102B500070BDA36AE26A13F8015BA362934202D3D9
:102B60002046FFF7D5FF002383F31188EFE700002D
:102B70002DE9F84F04460E46174698464FF03009A7
:102B800089F311880025AA46D4F828B0BBF1000FBC
:102B900009D141462046FFF7A1FF20B18BF31188F0
:102BA0002846BDE8F88FD4E90A12A7EB050B521AA4
:102BB000934528BF9346BBF1400F1BD9334601F123
:102BC000400251F8040B43F8040B9142F9D1A36A77
:102BD00040334036A3624035D4E90A239A4202D3F7
:102BE0002046FFF795FF8AF31188BD42D8D289F3BA
:102BF0001188C9E730465A46FEF758F8A36A5B4485
:102C00005E44A3625D44E7E710B5029C01720433A1
:102C100003FB0421C0E906130023C0E90A33039B28
:102C20000363049BC460C0E90000C0E90422C0E95A
:102C30000842436310BD0000026AC260426AC0E9F4
:102C400004220022C0E90A226FF00101FEF726BE2D
:102C5000D0E904239A4201D1C26822B9184650F83B
:102C6000043B0B60704700231846FAE7C368C2694B
:102C70000133C3604369134482694361934224BFB3
:102C8000436A43610021FEF7FDBD000038B50446EC
:102C90000D46E3683BB123691A1DA262E269134441
:102CA000E362002007E0237A33B929462046FEF785
:102CB000D9FD0028EDDA38BD6FF00100FBE7000018
:102CC00003691960C268013AC260C269134482692B
:102CD0000361934224BF436A036100238362036B51
:102CE00003B118477047000070B530230D46044605
:102CF000114683F31188866A2EB9FFF7C7FF10B11A
:102D000086F3118870BDA36A1D70A36AE26A01335D
:102D10009342A36204D3E16920460439FFF7D0FF50
:102D2000002080F31188EDE72DE9F84F04460D46A9
:102D3000904699464FF0300A8AF311880026B34630
:102D4000A76A4FB949462046FFF7A0FF20B187F395
:102D500011883046BDE8F88FD4E90A073A1AA8EB83
:102D60000607974228BF1746402F1BD905F140039D
:102D700055F8042B40F8042B9D42F9D1A36A403347
:102D8000A3624036D4E90A239A4204D3E16920467B
:102D90000439FFF795FF8BF311884645D9D28AF3A2
:102DA0001188CDE729463A46FDF780FFA36A3B44E8
:102DB0003D44A3623E44E5E7D0E904239A4217D19B
:102DC000C3689BB1836A8BB1043B9B1A0ED013601E
:102DD000C368013BC360C3691A44836902619A42B4
:102DE00024BF436A036100238362012318467047AE
:102DF0000023FBE700F030B94FF08043586A70477A
:102E00004FF08043002258631A610222DA60704753
:102E10004FF080430022DA60704700004FF080439B
:102E200058637047FEE7000070B51B4B0163002537
:102E3000044686B0586085620E4600F0BFF804F183
:102E40001003C4E904334FF0FF33C4E90635C4E985
:102E50000044A560E562FFF7CFFF2B460246C4E9B8
:102E6000082304F134010D4A256580232046FEF72E
:102E7000AFFC0123E0600A4A037500927268019278
:102E8000B268CDE90223074B6846CDE90435FEF769
:102E9000C7FC06B070BD00BF00260020A4360008A5
:102EA000A9360008252E0008024AD36A1843D062CA
:102EB000704700BF982300204B6843608B68836095
:102EC000CB68C3600B6943614B6903628B694362E2
:102ED0000B6803607047000008B5264B26481A6946
:102EE00040F2FF110A431A611A6922F4FF7222F0BC
:102EF00001021A611A691A6B0A431A631A6D0A43AE
:102F00001A651E4A1B6D1146FFF7D6FF02F11C0120
:102F100000F58060FFF7D0FF02F1380100F5806016
:102F2000FFF7CAFF02F1540100F58060FFF7C4FF0C
:102F300002F1700100F58060FFF7BEFF02F18C0125
:102F400000F58060FFF7B8FF02F1A80100F580608E
:102F5000FFF7B2FF02F1C40100F58060FFF7ACFF9C
:102F600002F1E00100F58060FFF7A6FFBDE8084030
:102F700000F0EEB80038024000000240B036000811
:102F800008B500F059FAFEF701FCFFF793F8BDE829
:102F90000840FEF76FBE000070470000EFF30983A2
:102FA00005494A6B22F001024A63683383F30988BA
:102FB000002383F31188704700EF00E0302080F396
:102FC000118862B60C4B0D4AD96821F4E0610904FE
:102FD000090C0A43DA60D3F8FC20094942F08072F8
:102FE000C3F8FC200A6842F001020A602022DA7766
:102FF00083F82200704700BF00ED00E00003FA05EF
:10300000001000E010B5302383F311880E4B5B688D
:1030100013F4006314D0F1EE103AEFF30984683C26
:103020004FF08073E361094BDB6B236684F30988FF
:10303000FEF78CFB10B1064BA36110BD054BFBE7FF
:1030400083F31188F9E700BF00ED00E000EF00E036
:103050002F030008320300080F4B1A6C42F00102E4
:103060001A641A6E42F001021A660C4A1B6E9368CB
:1030700043F0010393604FF0804353229A624FF074
:10308000FF32DA6200229A615A63DA605A600122E2
:103090005A611A60704700BF00380240002004E007
:1030A0004FF0804208B51169D3680B40D9B2C943CB
:1030B0009B07116107D5302383F31188FEF77CFB52
:1030C000002383F3118808BD1F4B1A696FEAC252AF
:1030D0006FEAD2521A611A69C2F308021A614FF0FC
:1030E000FF301A695A69586100215A6959615A6951
:1030F0001A6A62F080521A621A6A02F080521A62E8
:103100001A6A5A6A58625A6A59625A6A1A6C42F0C2
:1031100080521A641A6E42F080521A661A6E0B4A76
:10312000106840F480701060186F00F44070B0F5C3
:10313000007F1EBF4FF4803018671967536823F46F
:103140000073536000F054B9003802400070004032
:10315000334B4FF080521A64324A4FF440411160B1
:103160001A6842F001021A601A689107FCD59A6841
:1031700022F003029A602A4B9A6812F00C02FBD1EB
:10318000196801F0F90119609A601A6842F48032F6
:103190001A601A689203FCD55A6F42F001025A670E
:1031A0001F4B5A6F9007FCD51F4A5A601A6842F0AD
:1031B00080721A601B4A53685904FCD5184B1A6870
:1031C0009201FCD5194A9A60194B1A68194B9A4218
:1031D000194B21D1194A1168194A91421CD140F268
:1031E00005121A60144A136803F00F03052BFAD175
:1031F0000B4B9A6842F002029A609A6802F00C0245
:10320000082AFAD15A6C42F480425A645A6E42F447
:1032100080425A665B6E704740F20572E1E700BF7C
:10322000003802400070004008544007009488387D
:10323000002004E011640020003C024000ED00E0AA
:1032400041C20F41074A08B5536903F001035361B6
:1032500023B1054A13680BB150689847BDE8084090
:10326000FFF7D0BE003C0140E02D0020074A08B522
:10327000536903F00203536123B1054A93680BB10C
:10328000D0689847BDE80840FFF7BCBE003C01404D
:10329000E02D0020074A08B5536903F00403536189
:1032A00023B1054A13690BB150699847BDE808403E
:1032B000FFF7A8BE003C0140E02D0020074A08B5FA
:1032C000536903F00803536123B1054A93690BB1B5
:1032D000D0699847BDE80840FFF794BE003C014024
:1032E000E02D0020074A08B5536903F0100353612D
:1032F00023B1054A136A0BB1506A9847BDE80840EC
:10330000FFF780BE003C0140E02D0020164B10B5B9
:103310005C6904F478725A61A30604D5134A936A6F
:103320000BB1D06A9847600604D5104A136B0BB1F5
:10333000506B9847210604D50C4A936B0BB1D06BA8
:103340009847E20504D5094A136C0BB1506C9847B5
:10335000A30504D5054A936C0BB1D06C9847BDE822
:103360001040FFF74FBE00BF003C0140E02D0020A1
:10337000194B10B55C6904F47C425A61620504D5AE
:10338000164A136D0BB1506D9847230504D5134AA7
:10339000936D0BB1D06D9847E00404D50F4A136EBE
:1033A0000BB1506E9847A10404D50C4A936E0BB133
:1033B000D06E9847620404D5084A136F0BB1506F62
:1033C0009847230404D5054A936F0BB1D06F9847F3
:1033D000BDE81040FFF716BE003C0140E02D002084
:1033E00008B5FFF75DFEBDE80840FFF70BBE000023
:1033F000062108B50846FFF71DFB06210720FFF749
:1034000019FB06210820FFF715FB06210920FFF70D
:1034100011FB06210A20FFF70DFB06211720FFF7FD
:1034200009FB06212820FFF705FBBDE8084007211E
:103430001C20FFF7FFBA000008B5FFF745FE00F0BB
:103440000BF8FDF78DFEFDF765FDFFF7A5FDBDE867
:103450000840FFF7CFBC00000023054A194601339E
:10346000102BC2E9001102F10802F8D1704700BF29
:10347000E02D0020034611F8012B03F8012B002A50
:10348000F9D1704753544D3332463F3F3F005354B8
:103490004D3332463430780053544D333246343253
:1034A000780053544D3332463434365858000000B7
:1034B000012033000010410001105A000310590090
:1034C00007103100000000008434000813040000DD
:1034D0008E3400081904000098340008210400000C
:1034E000A234000800000000910E00087D0E0008C4
:1034F000B90E0008A50E0008B10E00089D0E0008C8
:10350000890E0008750E0008C50E000800000000B6
:1035100001000000000000006330000018350008C2
:10352000F0230020002600204172647550696C6F02
:10353000740025424F415244252D424C00255345ED
:103540005249414C2500000002000000000000002C
:10355000AD1000081911000840004000A02A00200A
:10356000B02A00200200000000000000030000005C
:10357000000000005D1100080000000010000000C5
:10358000C02A002000000000010000000000000030
:10359000682D002001010200111C0008211B0008F9
:1035A000BD1B0008A11B000843000000B035000847
:1035B00009024300020100C03209040000010202B6
:1035C0000100052400100105240100010424020269
:1035D0000524060001070582030800FF0904010015
:1035E000020A0000000705010240000007058102F1
:1035F0004000000012000000FC350008120110011C
:1036000002000040091241570002010203010000BC
:103610000403090425424F41524425004D6174655D
:103620006B463430352D57696E672D626473686F51
:1036300074003031323334353637383941424344FF
:10364000454600000040000000400000004000002F
:103650000040000000000100000002000000020025
:103660000000020000000200000002000000020052
:103670000000020000000000A11200085915000817
:103680000516000840004000C82D0020C82D00206D
:1036900001000000D82D0020800000004001000043
:1036A000030000006D61696E0069646C65000000D4
:1036B0000A01A81600000000AAAAAAAA050114007F
:1036C000FF9F00008800000070A70A0000000001B2
:1036D00000000000AAAAAAAA00000001FFFF000043
:1036E000000000000000000000A0A0120000000088
:1036F000AAAAAAAA00505011FFFF000000000088EB
:10370000007708002000000000000000AAAAAAAA72
:1037100010000000FFFF0000000800000000000093
:103720000000000000000000AAAAAAAA00000000F1
:10373000FFFF00000000000000000000000000008B
:1037400000000000AAAAAAAA00000000FFFF0000D3
:103750000000000000000000000000000000000069
:10376000AAAAAAAA00000000FFFF000000000000B3
:103770000000000000000000000000000A0000003F
:103780000000000003000000000000000000000036
:103790000000000000000000000000000000000029
:1037A0000000000000000000000000000000000019
:1037B0007F0000000000000000000F00000000007B
:1037C000FF009600000000080096000000000800BE
:1037D0000400000010360008000000000000000097
:1037E00000000000000000000000000000000000D9
:1037F000FFFFFFFFFFFFFFFFFFFFFFFFFFFFFFFFD9
:10380000FFFFFFFFFFFFFFFFFFFFFFFFFFFFFFFFC8
:10381000FFFFFFFFFFFFFFFFFFFFFFFFFFFFFFFFB8
:020000040801F1
:100000000006002099120108810D0708DD0C070881
:10001000490D0708DD0C0708150D07089B1201089C
:100020009B1201089B1201089B120108F575090833
:100030009B1201089B1201089B1201089B120108E8
:100040009B1201089B1201089B1201089B120108D8
:100050009B1201089B1201088D810908B5810908CE
:10006000DD810908058209082D820908752409081F
:100070009D240908C9240908F5240908212509082F
:100080004925090875250908F92309089B12010863
:100090009B1201089B1201089B1201085582090856
:1000A000A1830908B5830908C9830908CD83090814
:1000B000D1830908E5830908F9830908CD2D0908CA
:1000C000E12D0908052E0908192E09089B120108BF
:1000D0009B120108298309083D83090851830908F7
:1000E000B98209089B1201089B1201081D840908A6
:1000F000218409083584090839840908A1250908DB
:100100009B1201089B1201080D8409089B1201082B
:1001100065830908798309089B1201089B1201086D
:10012000CD250908F5250908212609084D260908C5
:10013000792609089B1201089B1201089B120108ED
:100140009B1201089B1201089B120108217D0908DE
:10015000A1260908CD260908F92609088D83090872
:100160009B1201089B1201089B1201089B120108B7
:100170009B1201089B1201089B1201089B120108A7
:100180009B1201089B1201089B1201089B12010897
:100190009B1201089B1201089B1201089B12010887
:1001A0009B1201089B1201089B1201089B12010877
:1001B0009B1201089B1201089B1201089B12010867
:1001C0009B1201089B1201089B1201089B12010857
:1001D0009B1201089B1201089B1201089B12010847
:1001E000A9270108F93701089194010811FA0208BA
:1001F00041A60408EDC4040825260508E92D0508D4
:1002000021310508999505081DB20508ED3C060841
:10021000255206087D5F06084DFE0608F103070813
:1002200009E707085D070808795508089D7C080854
:1002300039930808C5C20808F1C808080000000082
:1002400081F0004102E000BF83F0004330B54FEA87
:1002500041044FEA430594EA050F08BF90EA020FF4
:100260001FBF54EA000C55EA020C7FEA645C7FEA87
:10027000655C00F0E2804FEA5454D4EB5555B8BFAA
:100280006D420CDD2C4480EA020281EA030382EA1B
:10029000000083EA010180EA020281EA0303362DAD
:1002A00088BF30BD11F0004F4FEA01314FF4801C80
:1002B0004CEA113102D0404261EB410113F0004F92
:1002C0004FEA03334CEA133302D0524263EB430349
:1002D00094EA050F00F0A780A4F10104D5F1200EE7
:1002E0000DDB02FA0EFC22FA05F2801841F1000142
:1002F00003FA0EF2801843FA05F359410EE0A5F116
:1003000020050EF1200E012A03FA0EFC28BF4CF046
:10031000020C43FA05F3C01851EBE37101F00045FC
:1003200007D54FF0000EDCF1000C7EEB00006EEB09
:100330000101B1F5801F1BD3B1F5001F0CD3490893
:100340005FEA30004FEA3C0C04F101044FEA4452EA
:1003500012F5800F80F09A80BCF1004F08BF5FEA71
:10036000500C50F1000041EB045141EA050130BD51
:100370005FEA4C0C404141EB0101013C28BFB1F563
:10038000801FE9D291F0000F04BF01460020B1FAAE
:1003900081F308BF2033A3F10B03B3F120020CDA81
:1003A0000C3208DD02F1140CC2F10C0201FA0CF05F
:1003B00021FA02F10CE002F11402D8BFC2F1200CC4
:1003C00001FA02F120FA0CFCDCBF41EA0C0190407A
:1003D000E41AA2BF01EB0451294330BD6FEA0404C3
:1003E0001F3C1CDA0C340EDC04F11404C4F12002AE
:1003F00020FA04F001FA02F340EA030021FA04F3C0
:1004000045EA030130BDC4F10C04C4F1200220FA16
:1004100002F001FA04F340EA0300294630BD21FA54
:1004200004F0294630BD94F0000F83F4801306BF1A
:1004300081F480110134013D4EE77FEA645C18BF0E
:100440007FEA655C29D094EA050F08BF90EA020FA5
:1004500005D054EA000C04BF1946104630BD91EA9D
:10046000030F1EBF0021002030BD5FEA545C05D1A0
:100470004000494128BF41F0004130BD14F58004DF
:100480003CBF01F5801130BD01F0004545F0FE4153
:1004900041F470014FF0000030BD7FEA645C1ABF88
:1004A000194610467FEA655C1CBF0B46024650EABF
:1004B000013406BF52EA033591EA030F41F40021EB
:1004C00030BD00BF90F0000F04BF0021704730B571
:1004D0004FF4806404F132044FF000054FF0000146
:1004E00050E700BF90F0000F04BF0021704730B507
:1004F0004FF4806404F1320410F0004548BF4042DC
:100500004FF000013EE700BF42004FEAE2014FEA30
:1005100031014FEA02701FBF12F07F4393F07F4F0B
:1005200081F06051704732F07F4208BF704793F00E
:100530007F4F04BF41F40021704730B54FF4607421
:1005400001F0004521F000411CE700BF50EA010224
:1005500008BF704730B54FF000050AE050EA0102CD
:1005600008BF704730B511F0004502D5404261EB3D
:1005700041014FF4806404F132045FEA915C3FF47E
:10058000D8AE4FF003025FEADC0C18BF03325FEA1B
:10059000DC0C18BF033202EBDC02C2F1200300FACC
:1005A00003FC20FA02F001FA03FE40EA0E0021FAF1
:1005B00002F11444BDE600BF70B54FF0FF0C4CF4DF
:1005C000E06C1CEA11541DBF1CEA135594EA0C0F91
:1005D00095EA0C0F00F0DEF82C4481EA030621EACC
:1005E0004C5123EA4C5350EA013518BF52EA033507
:1005F00041F4801143F4801338D0A0FB02CE4FF0B9
:100600000005E1FB02E506F00042E0FB03E54FF0E8
:100610000006E1FB03569CF0000F18BF4EF0010EE0
:10062000A4F1FF04B6F5007F64F5407404D25FEADC
:100630004E0E6D4146EB060642EAC62141EA55518F
:100640004FEAC52040EA5E504FEACE2EB4F1FD0CD1
:1006500088BFBCF5E06F1ED8BEF1004F08BF5FEA4F
:10066000500E50F1000041EB045170BD06F0004601
:1006700046EA010140EA020081EA0301B4EB5C04AE
:10068000C2BFD4EB0C0541EA045170BD41F48011A6
:100690004FF0000E013C00F3AB8014F1360FDEBFCB
:1006A000002001F0004170BDC4F10004203C35DAA7
:1006B0000C341BDC04F11404C4F1200500FA05F32A
:1006C00020FA04F001FA05F240EA020001F00042CB
:1006D00021F0004110EBD37021FA04F642EB060141
:1006E0005EEA430E08BF20EAD37070BDC4F10C046B
:1006F000C4F1200500FA04F320FA05F001FA04F22F
:1007000040EA020001F0004110EBD37041F100011A
:100710005EEA430E08BF20EAD37070BDC4F1200525
:1007200000FA05F24EEA020E20FA04F301FA05F28D
:1007300043EA020321FA04F001F0004121FA04F235
:1007400020EA020000EBD3705EEA430E08BF20EA05
:10075000D37070BD94F0000F0FD101F0004640003F
:1007600041EB010111F4801F08BF013CF7D041EAC1
:10077000060195F0000F18BF704703F000465200C5
:1007800043EB030313F4801F08BF013DF7D043EA96
:100790000603704794EA0C0F0CEA135518BF95EA4C
:1007A0000C0F0CD050EA410618BF52EA4306D1D1D3
:1007B00081EA030101F000414FF0000070BD50EAF2
:1007C000410606BF1046194652EA430619D094EA7C
:1007D0000C0F02D150EA013613D195EA0C0F05D166
:1007E00052EA03361CBF104619460AD181EA0301BA
:1007F00001F0004141F0FE4141F470014FF0000072
:1008000070BD41F0FE4141F4780170BD70B54FF00C
:10081000FF0C4CF4E06C1CEA11541DBF1CEA13558C
:1008200094EA0C0F95EA0C0F00F0A7F8A4EB05046E
:1008300081EA030E52EA03354FEA013100F0888065
:100840004FEA03334FF0805545EA131343EA12632E
:100850004FEA022245EA111545EA10654FEA0026E3
:100860000EF000419D4208BF964244F1FD0404F59C
:10087000407402D25B084FEA3202B61A65EB0305F8
:100880005B084FEA32024FF480104FF4002CB6EBB5
:10089000020E75EB030E22BFB61A754640EA0C0035
:1008A0005B084FEA3202B6EB020E75EB030E22BF75
:1008B000B61A754640EA5C005B084FEA3202B6EBB6
:1008C000020E75EB030E22BFB61A754640EA9C0075
:1008D0005B084FEA3202B6EB020E75EB030E22BF45
:1008E000B61A754640EADC0055EA060E18D04FEA03
:1008F000051545EA16754FEA06164FEAC30343EAA3
:1009000052734FEAC2025FEA1C1CC0D111F4801F6F
:100910000BD141EA00014FF000004FF0004CB6E768
:1009200011F4801F04BF01430020B4F1FD0C88BF07
:10093000BCF5E06F3FF6AFAEB5EB030C04BFB6EB12
:10094000020C5FEA500C50F1000041EB045170BD05
:100950000EF0004E4EEA113114EB5C04C2BFD4EB32
:100960000C0541EA045170BD41F480114FF0000EB6
:10097000013C90E645EA060E8DE60CEA135594EA32
:100980000C0F08BF95EA0C0F3FF43BAF94EA0C0F35
:100990000AD150EA01347FF434AF95EA0C0F7FF4AA
:1009A00025AF104619462CE795EA0C0F06D152EAFE
:1009B00003353FF4FDAE1046194622E750EA4106E2
:1009C00018BF52EA43067FF4C5AE50EA41047FF4F3
:1009D0000DAF52EA43057FF4EBAE12E74FF0FF3C58
:1009E00006E000BF4FF0010C02E000BF4FF0010C29
:1009F0004DF804CD4FEA410C7FEA6C5C4FEA430CA2
:100A000018BF7FEA6C5C1BD001B050EA410C0CBFF0
:100A100052EA430C91EA030F02BF90EA020F002052
:100A2000704710F1000F91EA030F58BF994208BFB9
:100A300090422CBFD8176FEAE37040F00100704776
:100A40004FEA410C7FEA6C5C02D150EA013C07D1CD
:100A50004FEA430C7FEA6C5CD6D152EA033CD3D018
:100A60005DF8040B704700BF8446104662468C4612
:100A70001946634600E000BF01B5FFF7B7FF002845
:100A800048BF10F1000F01BD4DF808EDFFF7F4FF6E
:100A90000CBF012000205DF808FB00BF4DF808EDF9
:100AA000FFF7EAFF34BF012000205DF808FB00BF1C
:100AB0004DF808EDFFF7E0FF94BF012000205DF83E
:100AC00008FB00BF4DF808EDFFF7CEFF94BF0120F3
:100AD00000205DF808FB00BF4DF808EDFFF7C4FFEC
:100AE00034BF012000205DF808FB00BF4FEA410C35
:100AF0007FEA6C5C02D150EA013C0AD14FEA430C18
:100B00007FEA6C5C02D152EA033C02D14FF0000054
:100B100070474FF0010070474FEA410212F5001292
:100B200015D211D56FF47873B3EB625212D94FEA34
:100B3000C12343F0004343EA505311F0004F23FA1E
:100B400002F018BF404270474FF00000704750EA73
:100B5000013005D111F0004008BF6FF00040704730
:100B60004FF00000704700BF4A0011D212F500128A
:100B700011D20DD56FF47873B3EB62520ED44FEAF5
:100B8000C12343F0004343EA505323FA02F0704775
:100B90004FF00000704750EA013002D14FF0FF30B3
:100BA00070474FF0000070474FEA4102B2F1E04356
:100BB00024BFB3F5001CDCF1FE5C0DD901F0004C44
:100BC0004FEAC0024CEA5070B2F1004F40EB830094
:100BD00008BF20F00100704711F0804F21D113F1C0
:100BE0003872BCBF01F00040704741F480114FEAF9
:100BF0005252C2F11802C2F1200C10FA0CF320FA82
:100C000002F018BF40F001004FEAC1234FEAD3239E
:100C100003FA0CFC40EA0C0023FA02F34FEA430308
:100C2000CCE77FEA625307D150EA01331EBF4FF091
:100C3000FE4040F44000704701F0004040F0FE40AC
:100C400040F40000704700BF80F0004002E000BFA9
:100C500081F0004142001FBF5FEA410392EA030FA7
:100C60007FEA226C7FEA236C6AD04FEA1262D2EBF1
:100C70001363C1BFD218414048404140B8BF5B42F6
:100C8000192B88BF704710F0004F40F4000020F08F
:100C90007F4018BF404211F0004F41F4000121F0A5
:100CA0007F4118BF494292EA030F3FD0A2F10102EF
:100CB00041FA03FC10EB0C00C3F1200301FA03F12D
:100CC00000F0004302D5494260EB4000B0F5000F50
:100CD00013D3B0F1807F06D340084FEA310102F10F
:100CE0000102FE2A51D2B1F1004F40EBC25008BFC1
:100CF00020F0010040EA03007047490040EB00008B
:100D0000013A28BFB0F5000FEDD2B0FA80FCACF18B
:100D1000080CB2EB0C0200FA0CF0AABF00EBC250B8
:100D200052421843BCBFD0401843704792F0000FA6
:100D300081F4000106BF80F400000132013BB5E7F9
:100D40004FEA41037FEA226C18BF7FEA236C21D06F
:100D500092EA030F04D092F0000F08BF08467047D4
:100D600090EA010F1CBF0020704712F07F4F04D1A2
:100D7000400028BF40F00040704712F100723CBFB5
:100D800000F50000704700F0004343F0FE4040F4DF
:100D9000000070477FEA226216BF08467FEA23639D
:100DA0000146420206BF5FEA412390EA010F40F488
:100DB000800070474FF0000304E000BF10F00043D4
:100DC00048BF40425FEA000C08BF704743F09643BB
:100DD00001464FF000001CE050EA010208BF7047D6
:100DE0004FF000030AE000BF50EA010208BF70475D
:100DF00011F0004302D5404261EB41015FEA010C72
:100E000002BF84460146002043F0B64308BFA3F169
:100E10008053A3F50003BCFA8CF2083AA3EBC2534B
:100E200010DB01FA02FC634400FA02FCC2F120026A
:100E3000BCF1004F20FA02F243EB020008BF20F0A1
:100E40000100704702F1200201FA02FCC2F1200207
:100E500050EA4C0021FA02F243EB020008BF20EAFC
:100E6000DC7070477BB972B90029BEBF00204FF01B
:100E7000004106E008BF00281CBF6FF000414FF0A2
:100E8000FF3000F007BAADF1080C6DE904CE00297F
:100E900009DB002B1ADB00F095F8DDF804E0DDE952
:100EA000022304B07047404261EB4101002B1BDB81
:100EB00000F088F8DDF804E0DDE9022304B04042E8
:100EC00061EB4101524263EB43037047524263EBD3
:100ED000430300F077F8DDF804E0DDE9022304B015
:100EE000404261EB41017047524263EB430300F023
:100EF00069F8DDF804E0DDE9022304B0524263EB57
:100F00004303704753B94AB9002908BF00281CBFE2
:100F10004FF0FF314FF0FF3000F0BCB9ADF1080CDD
:100F20006DE904CE00F04EF8DDF804E0DDE90223BF
:100F300004B07047430803F05533C01A830803F028
:100F4000333300F03330184400EB101000F00F3052
:100F500000EB002000EB0040000E704707EE900A07
:100F6000F5EEC07AF1EE10FA01D400F00BB8F1EE14
:100F7000677A08B517EE900A00F004F8404261EB7A
:100F8000410108BDD0B5FFF7BFFA0C4B0022064661
:100F90000F46FFF711FBFFF7E7FD0446FFF792FA54
:100FA000074B0022FFF708FB02460B463046394646
:100FB000FFF74AF9FFF7D8FD2146D0BD0000F03D0C
:100FC0000000F0412DE9F047089D04468E46002BB5
:100FD0004DD18A42944669D9B2FA82F252B101FAED
:100FE00002F3C2F1200120FA01F10CFA02FC41EAFD
:100FF000030E94404FEA1C48210CBEFBF8F61FFA82
:101000008CF708FB16E341EA034306FB07F199421C
:101010000AD91CEB030306F1FF3080F01F819942CF
:1010200040F21C81023E63445B1AA4B2B3FBF8F0A9
:1010300008FB103344EA034400FB07F7A7420AD930
:101040001CEB040400F1FF3380F00A81A74240F258
:1010500007816444023840EA0640E41B00261DB1C3
:10106000D4400023C5E900433146BDE8F0878B42F8
:1010700009D9002D00F0EF800026C5E900013046B7
:101080003146BDE8F087B3FA83F6002E4AD18B4291
:1010900002D3824200F2F980841A61EB030301203B
:1010A0009E46002DE0D0C5E9004EDDE702B9FFDE27
:1010B000B2FA82F2002A40F09280A1EB0C014FEAD2
:1010C0001C471FFA8CFE0126200CB1FBF7F307FB2F
:1010D000131140EA01410EFB03F0884208D91CEBD2
:1010E000010103F1FF3802D2884200F2CB8043466F
:1010F000091AA4B2B1FBF7F007FB101144EA01444E
:101100000EFB00FEA64508D91CEB040400F1FF31DC
:1011100002D2A64500F2BB800846A4EB0E0440EACA
:1011200003409CE7C6F12007B34022FA07FC4CEAD3
:10113000030C20FA07F401FA06F31C43F9404FEAC6
:101140001C4900FA06F3B1FBF9F8200C1FFA8CFEDB
:1011500009FB181140EA014108FB0EF0884202FA2F
:1011600006F20BD91CEB010108F1FF3A80F08880F0
:10117000884240F28580A8F102086144091AA4B2AD
:10118000B1FBF9F009FB101144EA014100FB0EFE2E
:101190008E4508D91CEB010100F1FF346CD28E455D
:1011A0006AD90238614440EA0840A0FB0294A1EBEE
:1011B0000E01A142C846A64656D353D05DB1B3EB4B
:1011C000080261EB0E0101FA07F722FA06F3F1407B
:1011D0001F43C5E9007100263146BDE8F087C2F122
:1011E0002003D8400CFA02FC21FA03F3914001439A
:1011F0004FEA1C471FFA8CFEB3FBF7F007FB1036D3
:101200000B0C43EA064300FB0EF69E4204FA02F47E
:1012100008D91CEB030300F1FF382FD29E422DD9D1
:10122000023863449B1B89B2B3FBF7F607FB163306
:1012300041EA034106FB0EF38B4208D91CEB010186
:1012400006F1FF3816D28B4214D9023E6144C91A06
:1012500046EA004638E72E46284605E70646E3E616
:101260001846F8E64B45A9D2B9EB020864EB0C0E20
:101270000138A3E74646EAE7204694E74046D1E72F
:10128000D0467BE7023B614432E7304609E76444DD
:10129000023842E7704700BF02E000F000F8FEE7C6
:1012A00072B6374880F30888364880F30988364894
:1012B0003649086040F20000CCF200004EF634716E
:1012C000CEF200010860BFF34F8FBFF36F8F40F283
:1012D0000000C0F2F0004EF68851CEF20001086026
:1012E000BFF34F8FBFF36F8F4FF00000E1EE100A96
:1012F0004EF63C71CEF200010860062080F314889F
:10130000BFF36F8F86F0D4F985F03CFA4FF055307B
:101310001F491B4A91423CBF41F8040BFAE71D49A3
:10132000184A91423CBF41F8040BFAE71A491B4A9C
:101330001B4B9A423EBF51F8040B42F8040BF8E7EE
:1013400000201849184A91423CBF41F8040BFAE7C3
:1013500086F0B2F985F06AFA144C154DAC4203DA06
:1013600054F8041B8847F9E701F00EFA114C124DAE
:10137000AC4203DA54F8041B8847F9E786F09AB9BF
:1013800000060020002200200000010808ED00E017
:101390000000002000060020E0900B080022002042
:1013A000A0250020A025002098330120E00101089D
:1013B0003C0201083C0201083C0201082DE9F04F03
:1013C0002DED108AC1F80CD0C3689D46BDEC108A83
:1013D000BDE8F08F002383F311882846A047002042
:1013E00084F056FFFEE784F0B3FD00DFFEE7000067
:1013F00001F0FF01102A2BDB10F0070F08D010F8C6
:10140000013B013A8B422DD010F0070F42B3F6D1C9
:10141000F0B441EA012141EA014122F007047FF0E2
:1014200000070023F0E80256083C85EA010586EA39
:10143000010685FA47F5A3FA87F586FA47F6A5FA75
:1014400087F68EB9EED1F0BC01F0FF0102F0070281
:1014500032B110F8013B013A83EA010313B1F8D12C
:101460000020704701387047002D06BF354603380D
:10147000073815F0010F07D1013015F4807F02BF46
:10148000013015F4C03F0130F0BC0138704700BF97
:1014900010F8012B11F8013B012A28BF9A42F7D01E
:1014A000D01A7047034613F8012B002AFBD1181AF3
:1014B0000138704738B50022002304460D46FFF777
:1014C000EDFA28B920462946BDE8384000F00AB8B0
:1014D000204605F1004100F005F8404261EB410172
:1014E00038BD00BFD0B50C4B002206460F46FFF7B3
:1014F00063F8FFF739FB0446FEF7E4FF074B0022D1
:10150000FFF75AF802460B4630463946FEF79CFE76
:10151000FFF72AFB2146D0BD0000F03D0000F0415E
:1015200000207047704700007047000070470000BF
:10153000002070470020704700207047012070474E
:10154000002070477047000000207047002070475F
:10155000704700007047000000207047002070476F
:1015600070B5154ED6F8F80503681B68984704282F
:101570001ADC01281DDC002814BF012441240F4B74
:101580001D68E86A0368DB69984701280AD0D6F825
:10159000F8250B4B9A4205D0EB6A93F89C300BB1BF
:1015A00044F08004204670BD0A2814BF0124192489
:1015B000E5E71924E3E700BFA8550020A425002093
:1015C000A85B0020044BD3F8F80503F5C0629042F5
:1015D00014BF042002207047A8550020014B93F847
:1015E000A8047047A84500207047000038B5C578AA
:1015F0000B461C2D044628BF1C251C220021184622
:1016000089F09CFF2A4604F10C01BDE8384089F0BE
:101610004BBF000038B5C5780B46102D044628BFD7
:10162000102510220021184689F088FF2A4604F16F
:101630000C01BDE8384089F037BF000008B543F021
:10164000A3FC30B9034A92F88C3643F0040382F8C5
:101650008C3608BDA855002038B591ED000AF7EE8C
:10166000000A0D4619F012F920B10B4801F03CFFB9
:10167000002038BDD5ED007A9FED087AF0EEE77ACC
:10168000F4EEC77AF1EE10FA03D5034801F03EFFFD
:10169000EEE70320EDE700BFA8250020000000349E
:1016A00010B5044607F002FF204610BD13B58B8B22
:1016B000B72B0C4607D0B3F5967F21D002B0BDE81A
:1016C000104047F0DBBA124912481E2201F046FFD3
:1016D000D4ED017A94ED007A0D48FCEEE77ABCEE89
:1016E000C77A17EE903A8DED017A9DF804109AB200
:1016F00001F0CCFB002814BF0020042002B010BD74
:1017000004480549022201F029FF0020F6E700BF46
:10171000D05B0020A8250020A45B002000B5244B4E
:10172000DFED246A007C03F5D06292ED007A03F2CB
:101730008462D2ED007AA3F580528BB092F9CA246C
:10174000002A03F2746218BFB0EE677A1168049140
:1017500003F26C62D2ED007A8DED057AFDEEE77A48
:1017600003F5CE6317EE902AD3ED007AF4EEE67A15
:10177000F1EE10FA58BFF0EE667AFCEEE77A00233D
:1017800003930693079317EE903A12B2ADF8202018
:10179000ADF82220ADF82430B7221A23CDE900326B
:1017A0003E2103AA40F002FE0BB05DF804FB00BF2F
:1017B000A855002000FF7F4770B5164C94F892267C
:1017C0008AB022B90AB0BDE8704042F0A3B8057CE7
:1017D0005FF00CFBD4F8F065D4F8F415D4F8EC35D0
:1017E000A4F50054CDE90513B4F84026ADF8262041
:1017F0000023CDE90733ADF8243068221C23CDE95E
:101800000306CDE90032212103AA284640F0CEFD8F
:101810000AB070BDA8550020F0B5464CB4F8EC34C1
:10182000DE078DB0054643D504F5B26304F5B66214
:10183000D3F800C01268CDF8252004F2A45304F2B6
:101840008C5E1F68DEF800E0CDF80CE004F5B363B1
:1018500003AA1E68CDF810C004F29C5306961868BF
:10186000079004F5B46362201968089104F2AC5340
:1018700002211B68CDF829302123CDE900308DF8F5
:1018800024101923C221287C059740F08FFD287C65
:1018900040F022FD0646287C41F022FC00F12103A5
:1018A0009E4205D2287C0DB0BDE8F0403FF090BFCD
:1018B000B4F8EC3499073AD504F5CF6304F5D36254
:1018C000D3F800C01268CDF8252004F28C636222A0
:1018D0001F68194BCDF810C01E68059704F2846389
:1018E00006961868079004F5D163287C196808915A
:1018F00004F2946304F274641B68CDF82930032168
:10190000212324688DF82410CDE90032C221192347
:1019100003AA039440F04AFD287C40F0DDFC044615
:10192000287C41F0DDFB00F121039C42BAD30DB0CD
:10193000F0BD00BFA8450020284C002005207047BE
:10194000024BD3F8F80503681B681847A855002018
:1019500030B5CD788BB0272D28BF27250C46272200
:101960000021684689F0EAFD2A4604F10C01684628
:1019700089F09AFD1C4BD3F8F81503F5C16291422A
:1019800030D1DDED057A9FED197AF0EEE77AF4EECD
:10199000C77AF1EE10FA25D59DF8262002F0410114
:1019A00041291FD111061DD402F01801182919D0A0
:1019B00003F20C610198086003F5C26102980860A7
:1019C00082F0040203F2146103980860C2F38002FB
:1019D00083F81C2603F5C36103F5C4630498079AD2
:1019E00008601A600BB030BDA8550020000000341C
:1019F00030B5194D95F8913685B00C464BBBCA7879
:101A00008DF80C30092A28BF09220C3101A8CDE934
:101A1000013389F049FD9DF808305A1F012A18D971
:101A200003F0F703122B14D0A5F58053B3F9AA24C1
:101A300012B9E279A3F8AA24227AE179074800F0E2
:101A4000B1F9227AE179054800F0E4F9012385F83B
:101A5000913605B030BD00BFA8550020F4530020DA
:101A6000F0B51B4BB3F9AA3489B005460E461446AF
:101A70003BB1D779BB4204D009B0BDE8F04045F096
:101A8000F3BBA27A637A43EA0223E27A43EA02438F
:101A90001D2B13D0212B08D01BB921462846FFF758
:101AA000A7FF224631462846E6E701A92046FFF770
:101AB0009DFD084801A901F0F9FFF2E701A92046C0
:101AC000FFF7A8FD034801A902F04EF8E9E700BFBF
:101AD000A8450020A825002013B5CA78072A4FF092
:101AE0000003044628BF07220C3168460093CDF856
:101AF000033089F0D9FCBDF900304BB901231C211A
:101B0000204684F80F3302B0BDE8104047F06EB8AD
:101B100002B010BD30B5CD7889B01E2D28BF1E256E
:101B20000C461E220021684689F008FD2A4604F171
:101B30000C01684689F0B8FC0248694602F064F876
:101B400009B030BDA825002000B589B0084601A91C
:101B5000FFF74CFD034801A901F0A8FF09B05DF8AB
:101B600004FB00BFA82500201FB508466946FFF703
:101B700051FD0348694601F0F7FF05B05DF804FB2D
:101B8000A82500202DE9F041CC7894B0262C28BF60
:101B9000262488462622002107460AA889F0CEFC82
:101BA00002AD224608F10C010AA889F07DFC284606
:101BB00007F0A6F99DF84A30022B06AC03D0032BA0
:101BC00044D0002B66D1DFED357ADDED106A9FED54
:101BD000346A9DED0F7A66EEA76ADDED0E7A27EE88
:101BE000067A67EE867A0023FDEEE66ABDEEC77AD6
:101BF000FDEEE77A17EE102A17EE901A00932046B2
:101C000016EE903A07F09CF994E80F0085E80F0073
:101C100097F80F3363BB012698F8083098F807202F
:101C20008DF8193000238DF818208DF81B3099227B
:101C30000423CDE90032387C8DF81A600323224654
:101C40002F2140F0B3FB14B0BDE8F081DFED137A33
:101C5000DDED106A9FED126A9DED0F7A66EEA76AC0
:101C6000DDED0E7A27EE067A67EE867A0123BBE772
:101C7000BDF8446086B90B483246294601F00EFC97
:101C80000028C8D0084A0621384642F011FE87F8DD
:101C90000F63C1E70226BFE70026BDE70000C84288
:101CA0008096184BA8250020FCF8090838B58A7AD8
:101CB0004B7A43EA0223CA7A43EA0243272B0546BA
:101CC0000C460CD81C2B10D91D3B0A2B0DD8DFE875
:101CD00003F01E0C0C0C1B0C0C0C0C121500452BED
:101CE0000FD0522B01D1FFF733FE21462846BDE825
:101CF000384046F09DB9FFF7EFFEF6E7FFF742FFE9
:101D0000F3E7FFF707FFF0E7FFF71EFFEDE7FFF749
:101D10002BFFEAE700207047C8207047012070477A
:101D200000207047002070470120704790F89C30D9
:101D30008B4286BF283150F82100002070470000F8
:101D400090F89C308B4286BF283150F8210000204B
:101D500070470000014B93F8A6047047A845002087
:101D6000C36A43F4E053C362036B43F4E053036379
:101D7000436B43F4E05343637047000013B54FF4E3
:101D80004470CDE9002107F089FB044628B1DDE964
:101D9000002146F06FFB024B2360204602B010BDCD
:101DA00098FA09082DE9F04FDFF8649085B00646EF
:101DB0000F46904600254FF4837A96F89C30ECB29B
:101DC000A34222D9204640F087FA8346204641F0BC
:101DD00087F9031D9B4514D399F9CB34ADF808302E
:101DE00094220623CDE90032422102AA20468DF832
:101DF0000A708DF80B80ADF80CA040F0D7FA0135D1
:101E0000DBE720463FF0E4FCF9E705B0BDE8F08FE2
:101E1000A84500202DE9F04FDFF8649085B0064614
:101E20000F469046002540F2011A96F89C30ECB21D
:101E3000A34222D9204640F04FFA8346204641F083
:101E40004FF9031D9B4514D399F9CB34ADF80830F5
:101E500094220623CDE90032422102AA20468DF8C1
:101E60000A708DF80B80ADF80CA040F09FFA013598
:101E7000DBE720463FF0ACFCF9E705B0BDE8F08FAA
:101E8000A8450020704700001FB500F5405303F23D
:101E9000746203F26C63002112681B68019100F503
:101EA000A25001A90292039302F01CF803F01AFC5D
:101EB00003F0C4F905B05DF804FB000070B586B00E
:101EC00006461322002101A810EE105A10EE904A87
:101ED00089F034FBA3238DF8043095238DF8053069
:101EE0005EF08CFF1322CDF80700CDF80B1006F53D
:101EF0008F5001A9CDF80F50CDF813403BF024FAD4
:101F000006B070BD2DE9F0418AB0044688461746F8
:101F10000021232201A8109D1E4689F00FFBA32358
:101F20008DF8043095238DF8053001238DF80630A7
:101F30005EF064FF2B68CDF81B306B68CDF80700AE
:101F4000CDF80B10CDF81F302322AB68CDF80F80F1
:101F500001A904F58F50CDF81370CDF81760CDF8B6
:101F600023303BF0F1F90AB0BDE8F08197207047CB
:101F700010B500F540530446D3F8F80503681B6814
:101F800098471A22C1B204F58F503BF09DFB04F52F
:101F90009070BDE810400FF0D7BD000037B500F5D8
:101FA000125104460122243139F06EFF012504F557
:101FB0000B51104A009500232031DA2037F0DCF96C
:101FC0000D4A0095002304F58F51FD2037F0D4F918
:101FD0000A4B1A68D20705D4094A1D6004F59B54C0
:101FE000083414600648012103B0BDE8304037F0E2
:101FF00015BA00BF70450B085CB80A08A025002080
:102000000022002000207047002070470069C0F3C4
:10201000401070470F299DBF302303FB0100503053
:102020000020704700207047012070477047000073
:102030000020704700207047002070470020704744
:102040000020704700207047002070470020704734
:10205000002070470020704770470000036800228E
:102060001B68184710207047002070477047000019
:10207000032070470120704770470000012070471F
:10208000002070477047000000F51350343070474F
:1020900000487047CC1E0A0808B500F54050D0F83B
:1020A000F80503681B689847C0B208BD034808607C
:1020B0000F2111704FF0FF321A6070475C360A082A
:1020C00000207047002070477047000016F0A4B948
:1020D0003BF0A0BA47F0F0B845F026BA05F0BEBC18
:1020E00006F0D6BC00F000BF00F0FABE00F018BF4A
:1020F00001F078BC00F0E6BE00F0ECBE00F056BF88
:1021000070B5234B036000F50055224BC5F84C3EDB
:1021100000F540530446986808B107F0CBF91E4B10
:10212000236095F81C3143B9D5F818512DB12846D4
:1021300014F0F6FF284607F0B9F904F59A500C3070
:102140005BF04EFD04F59850103049F01BFA04F690
:10215000E46504F68466B54204D0183D284614F0C0
:102160004FFCF8E70D4BC4F8C83804F628203EF0C1
:1021700079FA04F6FC103EF075FA04F65C103EF0B5
:1021800071FA04F513603EF06DFA204670BD00BF91
:1021900090370A08C4D20A0838B10A0898840A0895
:1021A00038B54C4B044640F8043B4AF0E9FA04F1D8
:1021B000100006F093FD04F1680038F0BFFE04F54E
:1021C00090700FF07BF804F58C6005F0B7FA04F21C
:1021D000845007F071F904F6C80015F063FF04F5A8
:1021E00066604AF055FA04F5736038F0C9FB04F5EF
:1021F0008F503AF0DDFF04F5975014304FF000FF98
:1022000004F59850103049F0A5F904F59A500C30B7
:102210005BF0D2FC04F59B50083039F09BF904F5D3
:102220009D501C304BF08AFC04F5805304F59F52FE
:102230000025104683F8E053274B10301A6034F025
:102240004DFC294604F5A25001F042FF04F5D5509B
:10225000083055F0C3FD04F5FD500C3058F0E4FC97
:1022600004F5035004305AF001FE04F50450283000
:102270005BF036FA04F5065001F08AFD04F50B50C8
:10228000203056F09FFA04F50C501449383037F0DE
:1022900071FC04F50D50103050F056F904F5105053
:1022A0000C305BF0A1FF04F5005304F5115083F8E6
:1022B00064540B4D3C305CF0B9F82B6813B10948FD
:1022C0005EF062FD2046084937F054FC2C60204641
:1022D00038BD00BF38B10A088C670020A43D0B0848
:1022E000DC5E00205C340A0850B00A0810B59FED8F
:1022F000225A9FED224A9FED222ADFED221A9FEDFE
:10230000221A9FED220A86B00446F0EE453AB0EE5E
:10231000453AF0EE452AF0EE450AF7EE004A543011
:102320008DED054A8DED042ACDED031A8DED021ACF
:102330008DED015A8DED000A55F0F0FA9DED015A30
:102340009DED054A9DED042ADDED031A9DED021A6F
:102350009DED000AF7EE004AF0EE453AB0EE453A40
:10236000F0EE452AF0EE450A04F59E7055F0D6FAD7
:10237000204606B010BD00BF00000000CDCCCC3D13
:1023800000007A450AD7A33CCDCC4C3DCDCC4C3E89
:10239000F0B500F50055224BB5F8A6241A7087B0A9
:1023A000044648F035FF48F0B3FC204601F060FCDD
:1023B00004F5805393F8BC2612F001020FD102A855
:1023C000019206F09DFD02A904F5A25002F04CFF17
:1023D00028B12368019ADB6C02A920469847114E68
:1023E0003368DB6A93F89C7037B195F866341BB993
:1023F0005EF0FCFCC5F86804336885F86674DB6A37
:1024000093F89C20084B5A7139F00AF838F05CFDBB
:1024100004F51750203007B0BDE8F04055F0CEBAB3
:10242000E8220020A4250020055E0020FFF7B0BFB1
:1024300010B50821044601F0D7F918B117F0DAFDFC
:1024400015F0FAFC0121204601F0CEF910B120462A
:10245000FFF71AFD0421204601F0C6F918B104F572
:102460008F503AF023FB1021204601F0BDF928B12E
:1024700004F58F50BDE810403AF0B2BB10BD00002B
:10248000FFF7D6BF102925D8DFE801F0090D111993
:102490001524242424241D2424242424210000F58C
:1024A00058500430704700F558502C30704700F5F4
:1024B00058502430704700F558500830704700F5E8
:1024C00058502830704700F557503C30704700F5A1
:1024D000585070470020704708B556F077FA044B03
:1024E0001B68DB6A93F89C10BDE8084056F04ABAB6
:1024F000A4250020FFF7F0BF2DE9FF410446FFF7B8
:102500004FFE874B236004F5125004F5005624302B
:10251000FFF7ECFE002304F51B50C6F8C8360C305C
:1025200047F0E0F8DFF85C827E4BC6F8CC3642F22A
:102530001C7542F61C27601947F062FA44F80580C2
:102540003035BD42F7D1601948F03AFD04F53850F6
:1025500030303EF0C9FA04F538503C303EF0C4FA51
:1025600004F539570023A6F8483E0C376E4BC6F8E1
:102570004C3E07F114005DF0F7FA04F53A5504F506
:102580003B58043508F128082846143543F094F8E0
:102590004545F9D104F540550723EB6000232B8214
:1025A0004FF4CB7006F080FFA860284614305DF031
:1025B000DBFA04F5415018305DF0D6FA5B4B1A682F
:1025C00002B91F605A4BC6F84C3E5A4B0393002683
:1025D0000294009604AB04F5415013E90C0040212D
:1025E000343005F091FE04F55750283006F088FC91
:1025F00004F55853C5F8F8354F4BC5F8FC354F4B2B
:10260000C5F800364E4BC5F804364E4BC5F80836B3
:1026100005F20C6300274FF07E521A60DF609F6066
:102620005F60494BC5F8243604F55858474BC5F848
:10263000283608F13008464BC5F82C3608F104005E
:1026400006F05EFC08F1140006F05AFC05F25C632B
:1026500040481F605F609F603F4B04F55A5218600E
:10266000103233464FF6FF774FF0140C9EB20CFB3E
:1026700006010133097C0029F8D1384B38491E8006
:102680000B6813B137485EF07FFB85F8913604F58F
:102690005A50012385F8923614300A605BF074FFBB
:1026A000314BC5F89436314BC5F8EC36304BC5F894
:1026B000F43604F55C502F4BC5F8FC36C5F8E846F7
:1026C000C5F8F046C5F8F846103006F019FC04F5D8
:1026D0005C502C3006F014FC04F55D50083006F018
:1026E0000FFC04F55B56244BC5F85C37A5F8607702
:1026F00006F1A40006F004FC4FF0FF330C36C5F8D9
:10270000C0371E4B1E491E60304637F033FA204654
:10271000A5F80877A5F8247704B0BDE8F08100BFDC
:1027200090370A0840340A08C4D20A082062002000
:1027300074FB0908FD20010804380A08E8340A0877
:102740004C380A0838380A0860380A08FC340A0885
:1027500010350A08782E0A08A05E00209E5E002030
:102760005C5E002070340A08A8340A08C120010801
:10277000C5200108C92001080000FFFFD85D002026
:10278000E08E0A0894340A0838B5054B1C682368A3
:102790000A461D68034B01462046A847002038BD65
:1027A000A4250020A825002010B55DF01DFE064CD4
:1027B000064B18602046FFF79FFE2046044A054955
:1027C000BDE8104086F08CB9A8250020A425002083
:1027D00010C000200121010838B52DED028B0D46F7
:1027E000F0EE608AB0EE408A144602F07BFF90ED76
:1027F000937AD0ED957A67EE877A90ED927A67EECC
:10280000A87AE7EE087AC5ED007AD0ED920AD0ED0D
:10281000937A90ED957A67EEA07A67EEA80AE7EED4
:10282000480ABDEC028BC4ED000A38BD30B52DED71
:10283000068B83B0F0EE409AB0EE60AA0D460446D7
:1028400002F050FFD0ED7F7AD0F80002B8EEE79AA0
:1028500018F0E8F807EE900AF8EEE78A79EEC9AAD0
:102860003AEE688AFDEEEAAAB0EE480A18F0BCF823
:10287000BDEEC00A5DB110EE103ADFED1D0A002B6F
:10288000CCBF38EE608A38EE208ABDEEC80AF8EE7A
:10289000C00A01AA6946B8EEEA0A2046FFF79CFF83
:1028A000144BDFED157A009903F5CF6269EEA79A14
:1028B000116003F27C620199116029EE279AA3F658
:1028C0007422C2ED009A2AEE27AAA3F5276268EEC9
:1028D000A78A82ED009AA3F68C12A3F6881382EDE4
:1028E00000AAC3ED008A03B0BDEC068B30BD00BF6B
:1028F00000A00C47A85500200AD7233C38B52DED81
:10290000028B0D46B0EE408AF0EE608A144602F06B
:10291000E9FED0ED937A9FED147AF0EEE77AF4EECB
:10292000C77AF1EE10FA1DD4D0ED957A90ED927A37
:1029300067EEE87AE8EE077AC5ED007A90ED937AD3
:10294000D0ED957A90ED926AC7EE876A0120C6EEC7
:10295000077A67EEA80AE6EE880AC4ED000ABDEC25
:10296000028B38BD0020FAE70000003430B52DEDB1
:10297000068B5F4CDFED5F8AB4F9E4345B4285B0CF
:1029800008EE103A054604F563603EF0B1F8B8EE83
:10299000C88AB4F9E43490ED00AA28EE288AF6EE4D
:1029A000009A98EE29AA04F5636008EE103A3EF00A
:1029B0009FF8B8EEC88AB4F9E83490ED009A28EE92
:1029C000288A04F63C6098EE299A08EE103A3EF008
:1029D0008FF8B4F9EA34D0ED009A04F63C600AEEC0
:1029E000903A3EF085F8B8EEC88AF8EEEAAAD8EE3A
:1029F000289A6A4602A990ED008A8DED00AA9AEE07
:102A0000A88A2846F0EE4A0AB0EE690A8DED038ADC
:102A10008DED019ACDED029AFFF770FF01AA03A98F
:102A2000F0EE490AB0EE480A2846FFF767FF02F0C9
:102A300059FED0F8000217F0F5FF04F5B35304F285
:102A4000DC44D4ED007A93ED030A30EE270A08EE59
:102A5000100A20EE280A17F0C7FFB8EEC88A30EE39
:102A6000480A17F0C1FFDFED247A9DED007AB5EE3C
:102A7000C00AF1EE10FAACBF70EE676AF0EE406A81
:102A8000B4EEE67AB4BF70EE277AF0EE407AF1EE5B
:102A900010FA2ADD9DED016AB4EEE76AF1EE10FA54
:102AA00023D5B5EEC00AF1EE10FA08DD77EE665ACE
:102AB00037EEC65AF4EEC55AF1EE10FA13D4B5EE5D
:102AC000C00AF1EE10FA10D537EE667A77EEC67AC4
:102AD000B4EEE77AF1EE10FACCBF0120002005B089
:102AE000BDEC068B30BD0120F9E70020F7E700BF01
:102AF000A84500200000C84200A00C4770B5364C25
:102B00002DED028B04F26C62A4F62433D3ED007A2F
:102B100092ED000ADFED318A30EE270AA4F58056E7
:102B200084B020EE280A054617F05EFFB6F9EA34B5
:102B300001EE103AB6F9E83404F2746200EE903A0D
:102B4000A4F53263D3ED007AB0EE408A92ED000A2C
:102B5000B8EEC11A30EE270AF8EEE00A0C2017F0A2
:102B600097FF20EE280A28468DED010AFFF7FEFEAA
:102B70009DED010A0146F0EE480A2846FFF756FE91
:102B80009DED010A03AA02A9F0EE480A2846FFF7C4
:102B900023FEB6F9E634002B0FDD07EE903A04F57C
:102BA000CE62F8EEE77A92ED007AB4EEE77AF1EED3
:102BB00010FA02DA94F830364BB99DED020A084853
:102BC00000F018FB9DED030A054800F0F5FB04B08A
:102BD000BDEC028B70BD00BFA85500200000C842AC
:102BE000A825002038B54C4C94F88C36054613F0D7
:102BF000010047D1A4F580529FED487AB2F9B8247C
:102C000007EE902AF8EEE77A04F26C6167EE877AB5
:102C100091ED000A13F0100FBFEE007AF7EE006A94
:102C200008BFB0EE667AA7EE270AC3F30012DFED05
:102C30003C7A81ED000AB5EEC00AF1EE10FA0AD531
:102C40001AB160F3041384F88C36B4EEE70AF1EE9F
:102C500010FA06DC0BE0B4EEE70AF1EE10FA06DD3E
:102C60002AB994F88C3643F0100384F88C369FED23
:102C70002C1ADFED2C0A2C2017F00AFF04F26C63EB
:102C800083ED000A94F88C369A07C3F3400032D4DF
:102C900025499FED227AB1F9BA2407EE902AB1F9BD
:102CA000E824B1F9EA1400EE902A01EE101AF8EEC9
:102CB000E77A04F27462190767EE877AF8EEE00AA1
:102CC00092ED007AB8EEC11A1AD577EE677AF4EE73
:102CD000E07AF1EE10FAC2ED007A03D560F3C30397
:102CE00084F88C3604F2746494ED000A3C2017F0EA
:102CF000CFFE84ED000A2846BDE83840FFF7FEBE4F
:102D000077EE877AF4EEC17AF1EE10FAC2ED007A2E
:102D1000E8DD43F00803E3E7A85500200AD7A33C09
:102D20000000B44300000000A84500200A207047BE
:102D300001207047094B93F83016024609B1FFF79E
:102D4000DDBE93F8911629B9A3F5805393F8F034BA
:102D5000DB0702D51046FFF745BF7047A855002096
:102D6000042070470120704730B52DED028B8BB0E9
:102D700004465EF03BF807AB054606AA05A9201DF0
:102D800019F0FAFB274A9FED288A136841F288312F
:102D9000EB1A8B421CD9156045F02AF9DDED067A55
:102DA00067EE887A054617EE900AFDF7ADFBDDED7C
:102DB000077A67EE887ACDE9020117EE900AFDF7EF
:102DC000A3FB1A4ACDE90001062128463EF0E0FAAD
:102DD000DDED067ADDED070A9FED150A60EE880A43
:102DE00027EE888A60EE800A204628EE000A00213D
:102DF000FFF71CFDDDED070A9DED060A09AA08A9EB
:102E00002046FFF7E9FC9DED080A0A4800F0F2F9B8
:102E10009DED090A074800F0CFFA0BB0BDEC028B1C
:102E200030BD00BF705D0020E02E654210380A08FA
:102E30000000C842A82500200020704701207047EC
:102E4000024B014618680268126810472862002089
:102E500008B50020FFF7F4FFC188472048F03CF890
:102E6000472047F0D5FE0120FFF7EAFFC188482040
:102E700048F032F8BDE80840482047F0C9BE0000DD
:102E80000220704701207047FFF7ACBE08B50B4623
:102E9000013BDBB2012B114611D85BB9472048F04A
:102EA0001BF8472047F0B4FE48F0DEF847F090FDED
:102EB000012008BD482048F00FF84820F2E7002024
:102EC000F7E7000008B546F067FDBDE8084046F0AA
:102ED00043BC0000002100F5A25002F089BB0000B5
:102EE00000F2845006F072BF10B5044607F05EF899
:102EF00090F921308BB190F8403373B194F9A83533
:102F00005BB1064B1B68DB6A93F89C302BB904F26B
:102F10008450BDE8104006F071BD10BDA42500200E
:102F200070B5044600F590700FF066FD94F8143407
:102F30001C4904EB0312D2F8C4010A68824210D083
:102F4000B02202FB034294F8585492F8F12145B99B
:102F5000022A06D9144E08603278012A02D9013AB1
:102F6000327070BDFDD104F54055D5F8F0252AB971
:102F7000D5F8F42512B905233370F2E7B02202FB2D
:102F8000034303F5FE730FCB05F5BD6585E80F0020
:102F9000236804F55751DB6C0022283120469847FE
:102FA0000023E9E7745D00200C2200207047000038
:102FB00037B5044648F02CF947F0AAFE04F5005551
:102FC0004721002047F0D6FF4821012047F0D2FFDB
:102FD000B5F8E41401EB810101EB8101490089B2EC
:102FE000472047F0FFFDB5F9E834B5F9EA140F4D75
:102FF000C91A01EB810101EB8101490089B2482026
:1030000047F0F0FD48F030F847F0E2FC04F53850A6
:1030100001A9303001953DF0FDFD04F5385001A9BE
:103020003C3001953DF0F6FD03B030BDCDCCCC3D3C
:10303000F0B52DED028B00F5005785B0B7F8E82408
:10304000B7F8EA3404466425482012FB05F613FB62
:1030500005F547F0B7FD04F5595304F51350383022
:10306000B0EE408ADFED230A93ED0E0A01900021B5
:1030700054F00EFE07EE906A38EE000AF8EEE77A9A
:103080000198B4EEE70AF1EE10FA25D98DED020AA7
:1030900007EE905A9DED027AF8EEE77AF4EEC77AE1
:1030A000F1EE10FA03D8CDED027A54F0E5FC482099
:1030B0009DED020A47F072FD97F8493E04F538503D
:1030C0003C3083B10C4B039303AA02A93DF0A6FD4B
:1030D00005B0BDEC028BF0BD0190CDED027A54F04D
:1030E000CBFC0198D4E702A93DF004FD012387F849
:1030F000493EEDE70AD7A33C0AD7A33C00F5595354
:1031000000F5005093ED0E7A00F59A6200F59B638E
:10311000D2ED007A93ED006A67EE867AF0EEC76A28
:10312000F4EEE76AF1EE10FA04D59FED180A482094
:1031300047F034BDDFED167AB5EEC07AF1EE10FA45
:1031400020EE270A10DDB0F8E834642213FB02F306
:1031500007EE903AF8EEE77AF4EEC07AF1EE10FA64
:1031600002D59FED0C0AE2E7B0F8EA34642213FBC3
:1031700002F307EE903AF8EEE77AF4EEC07AF1EE59
:1031800010FA02DD9FED040AD1E77047000000004D
:103190000000C84200A00CC600A00C4610B50446B2
:1031A00000F5595304F5005400F51350DFED100AF3
:1031B00093ED0E0A0021383054F06AFDB4F9EA04A8
:1031C000B4F9E8343221C21A1B1A4A434B4301EEC8
:1031D000102A00EE903A8020B8EEC11AF8EEE00A0C
:1031E00017F056FCBDE81040482047F0D7BC00BFA0
:1031F0000AD7A33C00F5005393F9C834012B03D040
:10320000022B03D0FFF714BFFFF778BFFFF7C6BF4D
:10321000F0B52DED028B00F500573223B7F8E454DA
:10322000DFED310A00F5175615FB03F5203600F5E2
:10323000595393ED0F0A83B000210446304654F0F1
:1032400027FD9FED2A1ADFED2A0ABF2017F020FC88
:103250004720B0EE408A47F0B5FC9FED241ADFED21
:10326000240A30EE080AC02017F012FC6B4207EE69
:10327000903AF8EEE77AB4EEE70AF1EE10FA26D9C2
:103280008DED000A07EE905A9DED007AF8EEE77A90
:10329000F4EEC77AF1EE10FA04D83046CDED007A9C
:1032A00054F0EAFB47209DED000A47F077FC97F8C1
:1032B000483E04F5385030307BB10E4B019301AAE3
:1032C00069463DF0ABFC03B0BDEC028BF0BD30466F
:1032D000CDED007A54F0D0FBD4E769463DF00AFC0E
:1032E000012387F8483EEEE70AD7A33C00A08C46AE
:1032F00000A08CC60AD7A33C00F55953D3ED0F7A32
:103300009FED127A00F5005000F2CC4300F2D44059
:1033100067EE877A90ED006A93ED007A27EE067AE1
:10332000F0EEE76AF4EEC76AF1EE10FA04D59FED0D
:10333000080A472047F032BCF5EEC07AF1EE10FAE9
:10334000CCBF9FED040A9FED040AF2E70AD7233CA5
:103350000000000000A08C4600A08CC610B50446FA
:1033600000F5595304F5005400F51750DFED110A2C
:1033700093ED0F0A0021203054F08AFCB4F9E434B4
:103380004FF6CE71322213FB02F213FB01F301EE72
:10339000102A00EE903AF120B8EEC11AF8EEE00AD9
:1033A000B1EE400A17F074FBBDE81040472047F02B
:1033B000F5BB00BF0AD7A33C00F5005393F9C9340D
:1033C000012B03D0022B03D0FFF722BFFFF794BFDE
:1033D000FFF7C4BFFEF7CCBD70B500F5005088B054
:1033E00090F9F1040C46D8B105210E4847F0CEFF04
:1033F000092106460B4847F0C9FF012103900948FF
:1034000047F0C4FF04AD00210346039A009128460B
:10341000314605F095FD95E80F0084E80F00012086
:1034200008B070BD785D002037B50C460022054617
:1034300011460F4847F0C2FF62680D48012147F06E
:10344000D5FFA2680A48052147F0D0FFE268084886
:10345000092147F0CBFF05F5135001240DF10701B9
:1034600031308DF8074037F085F9204603B030BD84
:10347000785D002037B503680191DD6C04460FF0DC
:10348000F9FA90F8F412019AB02303FB0101DC3140
:1034900020462B4603B0BDE8304018477FB50446B0
:1034A00004F5A25668460D4605F02AFD69463046E9
:1034B00001F01EFF48B929462046FFF7B5FF064632
:1034C00050B90026304604B070BD2946304601F0A0
:1034D000B9FD0028EFD1F4E795E80F0004F5575443
:1034E000283484E80F00EDE710B5074B1B6804464D
:1034F000D86A036801211B68984704F58F500121A1
:10350000BDE8104039F004BFA425002010B5074BDA
:103510001B680446D86A036800211B68984704F5B5
:103520008F500021BDE8104039F0F2BEA4250020E4
:1035300010B504465DF05AFC04F500540021C4F8AF
:10354000C806472047F0E6FC0021482047F0E2FC8F
:1035500047F08AFDBDE8104047F03ABA70B504461E
:1035600004F5005304F5405583F86424D5F8F83584
:103570008B420846164627D0C5F8F8150B685B68DD
:10358000984710B32046FFF7AFFFD5F8F80503685A
:103590001B6898473246C1B204F58F503AF094F850
:1035A00004F5395000210C3045F040FB04F5B253CE
:1035B000D3ED007A9FED077AF8EEE77A05F26C65B5
:1035C00067EE877AC5ED007A70BD2046FFF79EFF53
:1035D000DBE700BF0AD7233CF7B5044600F59F5050
:1035E000103033F005FC644B04F5415001223430B7
:1035F0009A71DA7104F58C6504F032FF04F53956DE
:103600000823C4F8743428460C3604F05DFD3046B7
:1036100042F098F8304645F04FFE06F0C7FC2023F4
:10362000036306F0C3FC07F087FD0223C4F8A4314E
:1036300004F5907004F5A2570DF0D4FE384600F062
:10364000BFFE04F58053002283F84927B4F9A43063
:1036500004F6C8001BB9B4F8A230A4F8A430B4F83A
:10366000A41016F073FD384600F0A4FF284601218F
:1036700004F004FB414B0093414B019302AB13E96F
:10368000060004F58F5039F037FE46F085F999228F
:10369000292147F0DDF846F07FF946F025F904F5D9
:1036A00000552046FFF784FC05F2BC4393ED007AF9
:1036B000DFED347AF0EEC76AF4EEE76AF1EE10FA65
:1036C00004F540574FD804F51353D3ED007ADFEDDE
:1036D0002E6AB0EEE76AB4EEE66AF1EE10FA42D86E
:1036E000DFED2A6A27EE267A67EEA67ABDEEC77A64
:1036F000FDEEE77A17EE103AC7F8F03517EE903A7C
:10370000C7F8F435D7F8F03543B9D7F8F4352BB905
:1037100004F5575128312046FFF75EFE1C4B1B680D
:10372000986A03684FF47A715B68984795F9EE14CC
:103730002046FEF7A7FE014610B904F558510431A2
:103740001F22204605F2C445FFF708FFD5ED007A99
:10375000F5EEC07AF1EE10FA0BDD204603B0BDE8BD
:10376000F040FFF7E5BE0B4A052130463DF010FE64
:10377000C8E703B0F0BD00BF055E0020A82500200B
:10378000D53301080000B442000034438096184B42
:10379000A42500206C380A0808B50A2922D8DFE8D9
:1037A00001F00D1911151D2121212121060000F51F
:1037B00057513C31FFF7D2FE012008BD00F55851AA
:1037C0000431F7E700F558512431F3E700F558517B
:1037D0002831EFE700F558512C31EBE700F558514F
:1037E0000831E7E70020E8E700F58F503AF0CABB60
:1037F00000207047002070470148032147F028BD92
:10380000785D002070B505462DED028B05F540541E
:103810005DF0E0FAD4F85436DFED227AC31A08EEF0
:10382000103AB8EE488A28EE278AF1EE047AB4EE10
:10383000E78AF1EE10FA33D504F234630FCB04F2C9
:10384000446686E80F0004F5CC63D3ED000A04F269
:103850005C6393ED000A05F5595068EE200A28EEE6
:10386000000A043005F00EFE04F2646393ED007A62
:10387000DFED0D7AD4F8483627EE277A07EE903A36
:10388000F8EEE77AE7EE087AFDEEE77A17EE903A7F
:10389000C4F84836012384F83036BDEC028B70BD85
:1038A0000023F8E7BD3786350000C84230B585B043
:1038B0006D460446284605F023FB294604F5A25030
:1038C00001F0D2FC50B104F54054002384F8923644
:1038D00095E80F0004F5BD6484E80F0005B030BD25
:1038E000F8B52DED028B00F54054054694F83036BE
:1038F000002B69D0D4F8F82500F55853243300F58F
:10390000575600F559579A4206F1280607F1040761
:1039100019D094F88C36DA0715D43946304605F0BC
:103920009FFC9FED2C7AF6EE007AE0EE077A04F227
:103930006C639FED297AFDEEE77AF8EEE77A67EEA1
:10394000877AC3ED007A3946304605F02BFD05F540
:10395000005704F5CE6383ED000A97F9CA34DFED12
:103960001F6A012B05BFD4F84836D4F8EC25D4F8EB
:1039700068369B1A07EE903AF8EEE77A04F284660E
:1039800087EEA67A86ED007AD4F8F80503681B68FE
:103990009847022818D094F88C369B0714D404F565
:1039A000CE63D3ED000A97F9CA349FED0D8A04F275
:1039B000746463B905F55A5595ED000A85F0D8FB96
:1039C00020EE080A84ED000ABDEC028BF8BD96EDEE
:1039D000000AF3E7A00CB3450AD7233C0000C84215
:1039E000E02E654273B5044604F50055FFF70AFF63
:1039F0002046FFF75BFF05F2C4462046FFF770FF45
:103A0000D6ED007AF5EEC07AF1EE10FA09DC244B1F
:103A10001E68F06A0368DB699847012816D102B076
:103A200070BD5DF0E3F9D5F8C83696ED007ADFEDAC
:103A30001D6AC01A07EE900A27EE267AF8EE677A1A
:103A4000F4EEC77AF1EE10FAE1D5E8E7F36A93F8FD
:103A50009C10E9B995F9EF34012B10D19FED120AB2
:103A6000472047F09BF89FED100A482047F096F852
:103A700047F0FAFA02B0BDE8704046F0A9BF47200F
:103A8000019147F029FA0199482047F025FAEFE71C
:103A900004F54054D4F8F80503689B689847E7E7B5
:103AA000A425002000007A440000000037B54B68D0
:103AB000054613B98A68002A51D005F540540A20FA
:103AC000C4F83C368B68C4F84036CA6892FBF0F202
:103AD000C4F838260B6993FBF0F3C4F86836B1F9E3
:103AE0001630DFED207AB1F9142007EE103AB1F963
:103AF0001830B8EEC77A87EE276A07EE103AB8EEAC
:103B0000C77A04F25C63C7EE276A07EE102AB8EEA4
:103B1000C77AC7EE275AC3ED005A04F5CC6383ED8C
:103B2000006A04F26463C3ED006A5DF053F9C4F8FF
:103B300054065DF05BF90221C4F858062846FFF7E9
:103B400053FE60B105F559531C330093D4F8383651
:103B5000D4F84026D4F83C162846FEF7D3F903B033
:103B600030BD00BF0000C84210B52DED028B0446E9
:103B700091ED018ADFED227A94F8713428EE278ADC
:103B800000F58C60242202FB0303F0EE480A93ED5B
:103B9000090A03F01BFDB4EE400AF1EE10FAF0EE54
:103BA000400A24D69FED177AF0EEC07AF4EE477AF9
:103BB000F1EE10FA1BDC04F5405303F5D161D1EDB1
:103BC000007A77EE807A04F55A52C2ED007A93F8C3
:103BD0008C0640070BD5F1EE407AC1ED007A00214A
:103BE000116093F88C266FF3820283F88C26B0EE76
:103BF000480ABDEC028B2046BDE81040FEF75EB9D6
:103C00000000C842FFFF7F7FB1F9002007EE902A35
:103C100000F54050F8EEE77A00F26C6310B5C3EDA2
:103C2000007AB1F9022007EE902AF8EEE77A00F266
:103C30007463C3ED007A00F5CE6300221A60B1F917
:103C4000002090F88C3647F6FF74121B18BF012233
:103C500062F3000380F88C36B1F9023090F88C26BC
:103C60001B1B18BF012363F3410280F88C2610BD93
:103C700010B500F54054D4F8580650B15DF0B6F8D0
:103C8000D4F85836C01A41F2873398428CBF0020CE
:103C90000120014B187110BD055E002070B52DED9F
:103CA000028B00F5005400F54053164603F26C6297
:103CB000D2ED008AB4F9EA2401EE102AB4F9E8241E
:103CC00003F2746300EE902A04F59C62D3ED007A4F
:103CD00092ED000ADA20B8EEC11AF8EEE00A30EEF2
:103CE000270A0D4616F0D4FEB4F9E824B4F9EA34F4
:103CF00007EE902AF8EEE77A9B1A30EE670A07EE95
:103D0000903A30EE000AF8EEE77AB7EE008A80EEDD
:103D1000277A04F2DC4337EE487A86ED007A93ED99
:103D2000000A38EE800A16F01FFEB4F9E43407EEFC
:103D3000103A30EE000AB8EEC77A0120C0EE077ADA
:103D400077EEC87ABDEC028BC5ED007A70BD00003D
:103D50007047000000207047704700000020704747
:103D60000020704700207047002070479FED010A37
:103D7000704700BF000000009FED010A704700BFC0
:103D800000000000704700000020704770470000EE
:103D900010B50446143000F019F804F12C0000F0BE
:103DA00015F804F174005DF02DF804F1F4005DF0F5
:103DB00029F84FF0FF33C4F85031204610BD000001
:103DC000014B1868704700BF7C5D00207047000001
:103DD000F0B52DED048B91B004466D46284605F0F4
:103DE0008FF894F8BC33002B72D004F57A730FCBA4
:103DF00085E80F0094F8F833D4EDEC8A94EDED8A61
:103E000094EDEE9A002B63D094F8D033002B5FD062
:103E10002D22002104A8D4F8C073D4F8C463D4F8C8
:103E2000C853D4F8CC4387F089FBA3238DF8103016
:103E300095238DF8113046238DF812305CF0DEFFAB
:103E40009FED250A9FED257ACDF8171068EE807A50
:103E5000CDF8130067EE877AFDEEE77A17EE903A19
:103E600068EE007A29EE000A67EE877AADF81B301B
:103E7000FDEEE77A20EE070A17EE903AADF81D3016
:103E800016F09CFDDDED017A9FED157ACDF82D70D1
:103E9000BCEEC00AF8EEE77A10EE103A67EE877AC9
:103EA000ADF81F3017EE903ACDF82130029BCDF8D7
:103EB0002530039BCDF82930CDF83160CDF8355051
:103EC000CDF839403AF038FA2D2204A939F03CFAFD
:103ED00011B0BDEC048BF0BDE02E65420000C8427D
:103EE0000AD7233C30B52DED028B8BB0044624223B
:103EF0000D4601A8002187F021FBA3238DF8043093
:103F000095238DF8053048239FED1F8A8DF80630E4
:103F10005CF074FFD4ED817A2B68CDF80F3067EE3A
:103F2000887A95ED020ACDF80B1017EE903AD4ED91
:103F3000827ACDF8133067EE887A6B68CDF8173047
:103F400017EE903ACDF80700CDF81B3016F00CFDB7
:103F500010EE103A94ED830ACDF81F3020EE080AD7
:103F600016F002FD10EE103ACDF8233094F80C3321
:103F70008DF827303AF0E0F9242201A939F0E4F96C
:103F80000BB0BDEC028B30BDE02E654230B587B082
:103F900014460D4618220021684687F0CFFAA32365
:103FA0008DF8003095238DF8013049238DF80230CB
:103FB0005CF024FFA3680393E36804936368CDF87F
:103FC00007100593CDF803008DF80B503AF0B4F9C3
:103FD0001822694639F0B8F907B030BD10B58EB077
:103FE000044602A804F08CFF02A9204601F03CF927
:103FF000002845D001F076FB694600F0CDFF1F2276
:10400000002106A887F09AFAA3238DF8183095238B
:104010008DF819304A238DF81A305CF0EFFEDDED93
:10402000037A9FED1B7A049BCDF82330F8EEE77AF4
:10403000059BCDF8273067EE877ACDF81B0017EE89
:10404000903ADDED007ACDF82B30F1EE677A17EE7D
:10405000903ACDF81F10204601A9CDF82F3000F07E
:104060000FFC78B1DDED017AF1EE677A17EE903A48
:10407000CDF833303AF060F91F2206A939F064F91F
:104080000EB010BD3AF058F9DFED027AEEE700BF4E
:104090000AD7233C5241C07F002303604360836002
:1040A000C360036143618361C361036270470000C1
:1040B00090F8F432B02202FB030390F8382393F80F
:1040C000D13012B1012B28BF0123184670470000E0
:1040D0002DE9F04F04468BB04FF0000A0D461CF05E
:1040E00083FD84F814A204F506704FF07E575BF050
:1040F0003BFD4FF47A73A4F8623284F86852C4F836
:104100004872C4F84C72C4F8507204F51B70002554
:1041100004F0F6FE04F52B790323C4F8803204F58D
:104120003476C4F89452C4F89852C4F89C52C4F837
:10413000A052C4F8A452C4F8A8524846FFF7ACFFF6
:1041400004F5487B3046FFF7A7FFC4F81453C4F8C2
:104150001853C4F81C535846FFF79EFFC4F8445345
:10416000C4F84853C4F84C53C4F85053C4F85453DB
:10417000C4F85853C4F85C53C4F86053C4F864538B
:10418000C4F86853C4F86C53C4F87053C4F88C5323
:10419000C4F89053C4F89453C4F8A853C4F8A45373
:1041A000C4F8A053C4F8B053C4F8B453C4F8B85317
:1041B000C4F8CC53C4F8C853C4F8C453C4F89C73AF
:1041C000C4F8C07304F5757004F09AFE04F57A70B3
:1041D00004F096FE04F58063C4F8FC531D6004F5FA
:1041E000816304F583601D605D609D6004F088FE5E
:1041F00004F22C4304F264481D605D609D606D4BC9
:10420000C4F83C3404F50D73C4F8403404F50E735F
:10421000C4F8443404F50F73C4F8483404F510733B
:10422000C4F84C3404F24523C4F8503404F5117337
:10423000C4F8543404F58B6340461D605D609D6096
:10424000FFF72AFF04F59160FFF726FF04F5976357
:1042500004F23C421D605D609D6004F2C44304F2C0
:10426000BC501D605D609D6004F59A631D605D60DB
:104270009D6004F2DC431D605D609D6004F2EC43D0
:104280001D605D609D6004F2FC431D605D609D608B
:1042900004F5A1631D605D609D6004F22C53C2F8BB
:1042A000E070C2F8E4701D605D609D6004F5A76376
:1042B0001D605D609D6004F244531D605D609D6003
:1042C00004F5AC631F605D6004F284531D605D60A3
:1042D0009D6004F5B2631D605D609D6004F5B5638B
:1042E0001D605D609D6004F00BFE04F2CC5324223F
:1042F0001D605D6004F2D45351461D605D6004F2A0
:10430000DC5340461D605D6087F018F904F2FC50F4
:10431000C8F82070C8F81070C8F80070FFF7BCFE2D
:1043200004F5C46304F5CA601D605D609D6004F21D
:104330002C631D605D609D6004F5C7631D605D605A
:104340009D6004F244631D605D609D6004F0D8FDD3
:10435000194B1A491C60204635F00CFC51462422AA
:10436000584687F0EBF8C4F84073C4F83073C4F8CB
:10437000207304F5257207CA04F5287383E8070043
:10438000484694EDAA1AD4EDA90A94EDA80A16F0AD
:1043900077FF3546494668466E4616F093FE0FCEC7
:1043A0000FC50FCE0FC533682B6020460BB0BDE89C
:1043B000F08F00BFAC3A0A08805D00205C390A0823
:1043C00010B5044688B001F017FA94F93232012B87
:1043D00002D1274804F072FD022B0AD1032384F88E
:1043E000323204A9012304F111008DF8103036F0A7
:1043F00083F994F8323284F8903204F23C4001F0B0
:10440000B1F994F93132642B30D1652304A904F257
:1044100031208DF8103036F0ADF904A9204634F083
:104420004BFD18B304238DF818300023CDE9013378
:1044300003930F230593694604A834F0BDFE059B42
:1044400028B108AA02EB8302009942F8581C0133F4
:10445000112B0593EFD95AF07BF89DED031ADDED92
:10446000020A9DED010A65215AF030F808B010BD2E
:10447000BC380A0870B500F5257600F528758CB0B3
:1044800004463146284618F029FBE0B996E80700B3
:1044900085E8070004F52B7194EDAA1AD4EDA90A5A
:1044A00094EDA80A0191084616F0EAFE02AD0199C2
:1044B00002A816F007FE0FCD04F534740FC40FCD1B
:1044C0000FC42B6823600CB070BD000013B540F220
:1044D000411200F50671044601A812F0DDFB04F25A
:1044E0003C4001F027FB20461CF05CFD01A812F0C7
:1044F000F5FB02B010BD0000F8B50B68C0F804323F
:104500004B68C0F808328B68C0F80C3201F10C0619
:1045100007460C4600F548750FCE0FC50FCE0FC5E8
:1045200033682B6004F1300207CA07F5457383E84E
:10453000070004F13C0207CA07F5517383E807003E
:1045400004F1480207CA07F5547383E8070054349E
:1045500094E8070007F5577383E80700384601F031
:104560005FFA3846BDE8F84001F042BA13B5044698
:1045700000F23C40019002F021FF04F5BE61019879
:10458000009102F02FFA0099204602B0BDE81040D9
:10459000FFF7B2BF4A78064BC2F340121A754A7849
:1045A000C2F380125A750A78C2F300129A757047E6
:1045B000055E002013B540F2F522044600F50671B1
:1045C00001A812F069FB002104F23C4001F026FD35
:1045D00094F8603223B120461CF09CFE84F86002FF
:1045E00001A812F07BFB02B010BD000038B590F8B6
:1045F0000C3305460C462BB1032B0BD095F86832D3
:10460000DB070CD405F5CA630FCB84E80F0095F8DF
:10461000600603E01CF01CFD0028EFD038BD002030
:10462000FCE7000000F23C4090ED380A70470000C3
:1046300000F23C4090ED390A7047000010B490F849
:104640000C230C462AB1032A0AD000205DF8044B43
:10465000704700F5B56007C884E807000120F5E75A
:104660005DF8044B1CF0DCBC90F88403431E5842F8
:104670005841704738B590F80C330D468BB900F2AD
:104680003C4001F0C9FA044610B90024204638BD68
:1046900001F016FAD5ED007A27EE800A85ED000AC2
:1046A000F4E7D0EDE07AC1ED007A90F87C43002C7D
:1046B000EBD090EDDE7ADFED086AB4EEE67AF1EE4B
:1046C00010FAF7EE006AB8BFB0EE667A67EE877A46
:1046D000C1ED007ADAE700BF0000003490F80C3337
:1046E000032B01D11CF01CBC0020704790F80C2358
:1046F000032A01D11CF042BD00F23C4001F0F0BEA3
:1047000030B590F80C3385B004460D468BB1032BC1
:1047100018D004F5257018F01BFA284601A98DED74
:10472000010ACDED020A8DED031A18F04BF80120B5
:1047300006E000F23C4001F019FA0028E9D100201F
:1047400005B030BD90F86032002BF8D01CF0FEFCB4
:10475000DFE700007FB590F80C2332B1032A4FF059
:10476000000309D0039304930CE000F23C4007B02F
:104770005DF804EB01F0D6BA03A903930493059303
:104780001CF0C4FB9DED030ADDED040A07B05DF8E3
:1047900004FB000007B590F80C3333B100F57F70CF
:1047A00003B05DF804EB18F029B900F23C4001F0C9
:1047B000B9FA68468DED000ACDED010A18F01EF930
:1047C00003B05DF804FB000090F80C03003818BF3C
:1047D0000120704708B590F80C23032A05D0BDE8E6
:1047E000084000F23C4001F085BA1CF08FFB01202C
:1047F00008BD000010B590F80C230C461AB1032A2E
:1048000007D0002010BDBDE8104000F23C4001F090
:1048100015BA1CF091FB012084ED000AF2E70000BC
:1048200090F80C33032B01D11CF070BC00207047B2
:1048300030B590F80C3385B005460C4623B1032BF8
:1048400009D0002005B030BD00F23C4005B0BDE805
:10485000304002F0F7B8002302A9029303931CF042
:104860003DFB0028EDD001A928461CF043FB0028A1
:10487000E7D0029B2360039B6360019BA360E1E799
:1048800090F80C231AB1032A05D00020704700F2DB
:104890003C4002F0FDB81CF02DBB000090F9323214
:1048A0003BB990F8683213F0010F14BF03200020C9
:1048B0007047032070470000F7B50446FFF7EEFF8E
:1048C0000546002862D0032839D194F860326BB3D2
:1048D00094F86832D8072BD501A920461CF04CFE6D
:1048E000BDF80430002B18BF002594F8146206F0C0
:1048F000FD06012E4AD10023032D019307D101A902
:1049000020461CF045FE20461CF044FC064604F2FE
:104910003C4002F049F908B994F809039DF80430C5
:10492000D90703D55A0701D59F0632D400252DE0BB
:1049300020461CF0ADFA002808BF0025D5E7002569
:10494000D3E713F0020F2EE094F9443223B99DF817
:104950000430DB092FD0E9E7002EF8D00EF08AF8FA
:10496000FFF7A6FB022807D99DF805309806DDD58C
:104970009DF80430D906D9D5FB6A93F89C30002BFA
:10498000E5D118E0DA0601D41B0718D5284603B094
:10499000F0BD0028FAD094F80923B4F96436002A4F
:1049A000CFD013F0010FF1D1154B1F68FB6A93F8BC
:1049B0009C30002BC8D19DF804309C07E2D405F050
:1049C000F5FA05F0F1F90028B0D10EF053F8FFF731
:1049D0006FFB0228AAD90EF04DF890F8F432B022FD
:1049E00002FB030090ED3B7AF0EE007AB4EEE77A3A
:1049F000F1EE10FA9AD59DF80530DB09C6D195E79E
:104A0000A42500202DE9F04790F8603292B00446CA
:104A1000002B00F0948020461CF0BAFE2046FFF7E1
:104A20004BFF03287BD104F54878002741462046F8
:104A30000097019702971CF07FFB694620461CF007
:104A400071FB009BC4F80432019BC4F80832029B3E
:104A5000C4F80C32204600F0E3FF204600F0C8FF07
:104A600015F0C8FA054620461CF02AFA0028A8BF0F
:104A7000C6B203AA4FF0FF312046BCBF95F8EB94B5
:104A800095F8EC640397A8BFB146049705971CF00E
:104A900061FA03A818F05CF84FF00C0A0AFB095001
:104AA00084EDD10AC4EDD20A84EDD31A04F5517114
:104AB00000F55C7018F05CF804F557770AFB0655B2
:104AC00084EDC50AC4EDC60A84EDC71A3A464FF014
:104AD000FF31204605F500751CF050FA95E80700F7
:104AE00006AE86E807003946304618F0A7F804F508
:104AF0002B72414609A816F075FA314609A816F03E
:104B0000F3F909A9204684EDD40AC4EDD50A84ED51
:104B1000D61A1CF03DFD09A92046FFF73BFD94F88D
:104B20006636002B3AD109A804F0EAF909A9204613
:104B30001CF09AFA90B3012384F866362EE0D0F880
:104B400064321BB95CF052F9C4F86402154B1B685F
:104B5000D86A03685B68984788B15CF047F9D4F875
:104B60006432C01AB4F86232984204D920461CF06C
:104B7000D1FB84F8600294F860327BB14BE75CF0C3
:104B800035F9D4F86432C01A41F287339842E4D838
:104B900039F0D2FB39F012FA0028DED112B0BDE8AC
:104BA000F08700BFA425002090F80C3323B1032B1D
:104BB0004FF0000007D0704790F93222032A04D149
:104BC0000A70012070470870FBE718467047000024
:104BD00073B50D460DF107010446FFF7E5FF0646E4
:104BE00028B19DF807302BB1032B09D000263046A1
:104BF00002B070BD04F5CA630FCB85E80F00F6E77D
:104C0000294620461CF024FA94F86062EFE7000081
:104C10007FB50E460DF103010446FFF7C5FF0546BB
:104C200018B90025284604B070BD9DF8033083B143
:104C3000032B16D004F5257017F08AFF01A9304622
:104C40008DED010ACDED020A8DED031A17F0BAFDC4
:104C5000E8E7314604F23C4000F088FF0028E9D143
:104C6000DFE794F86032002BDBD0314620461CF0A1
:104C70006DFADFE737B50D460DF107010446FFF782
:104C800093FF28B19DF8073023B1032B0FD00020EC
:104C900003B030BD04F5BE631B682B6004F2F4530F
:104CA00004F5BF641B686B602368AB60F0E72046C7
:104CB00029461CF037FA94F86002E9E710B504467B
:104CC000FFF7ECFD18B1032807D0002010BD04F257
:104CD0003C40BDE8104000F073BF94F86032002BF8
:104CE000F3D020461CF0D4F80028EED094F814320B
:104CF00003F0FD03012BE9D194F80C03C31E5842C5
:104D00005841E3E710B50446FFF7C8FD80B103281A
:104D100010D194F8600250B15CF068F8D4F86432B5
:104D2000C01A44F62063984294BF0020012010BDB1
:104D30000120FCE70020FAE708B50246FFF7AEFDC8
:104D4000032804D110461CF023FC012008BD0020DC
:104D5000FCE7000030B585B004460191FFF730F85C
:104D60000199054610B9002005B030BD0191FEF74C
:104D7000F7FF01990028F6D02846FEF7F5FF002836
:104D8000F1D0B4F864365907EED494F80933002B07
:104D9000EAD00B4A1268D26A92F89C506DB103A90E
:104DA0002046FFF7C9FF30B19DF80E309A07DBD5DA
:104DB000C3F38000D8E72846D6E71846D4E700BFFB
:104DC000A42500202DE9F04190F80C338CB0002789
:104DD000032B06460C46154600970197029719D1FA
:104DE0001CF06EF86A4680464FF0FF3130461CF0EA
:104DF000C5F8B8F1FF3FA760676027600DD115F0D7
:104E0000F9F82B4690F8EC14224614F023F80CB075
:104E1000BDE8F0814FF0FF38EBE715F0EBF82B46DB
:104E200022465FFA88F114F015F895ED000A6846FD
:104E300017F0CAFE03A920468DED051A8DED030A71
:104E4000CDED040A17F0FAFE06F52B7206F548714F
:104E500003A816F0C7F8214603A816F045F884ED1C
:104E6000021A84ED000AC4ED010A95ED007ADFED27
:104E7000037AA7EE271A84ED021AC8E70AE81C4154
:104E800037B5054600F5067140F6033201A811F06A
:104E900003FF2846FFF702FD044640B103280AD06D
:104EA000002401A811F01AFF204603B030BD2846A7
:104EB0001CF092F8F5E728461CF08EF80446F0E75F
:104EC00008B50246FFF7EAFC10B1032806D008BD7A
:104ED000BDE8084002F23C4000F03CBEBDE808409E
:104EE00010461CF061BB00000B4610B411462BB1FC
:104EF000032B09D000205DF8044B70475DF8044B8C
:104F000000F23C4000F03CBE5DF8044B1CF0ACB835
:104F100013B50446FFF7C2FC0A460146204601923B
:104F2000FFF7E2FF70B9084B019A1B68DB6A93F840
:104F30009C0038B194F80C13204602B0BDE8104034
:104F4000FFF7D2BF02B010BDA425002037B504463C
:104F50000D4640F2B25200F5067101A811F09CFE18
:104F6000294620461CF09EF894F80C33032B054686
:104F700010D148B104F583612046FFF7C9FF84F8DA
:104F80002804204600F07CFD01A811F0A7FE284669
:104F900003B030BD0025F7E770B590F87C32DB0731
:104FA00086B004460D460CD402F0BEFF437C24229A
:104FB00002FB0300D0ED0B7AF1EE677AC5ED007AC3
:104FC0003BE002A803F09CFF01A92046FFF758FC34
:104FD000E8B90DF04FFD94F94432022B0646E3D1B7
:104FE000FFF766F80228DFD996F8F4029FED147AED
:104FF000B02303FB0066D4F87032D6F8E0209B1A89
:1050000007EE903AF8EEE77A67EE877AD6E702A9DC
:105010002046FFF77DFF0028DBD0D4F87022039BE9
:10502000DFED076A9DED017A9B1A07EE903AF8EEE4
:10503000E77AA7EEE67A85ED007A06B070BD00BF8C
:105040000AD7233CF0B50C4687B000F5067106463A
:1050500040F6863201A811F01FFEA36853B9E36839
:1050600043B9636833B9002701A811F037FE384609
:1050700007B0F0BD204604F04BF80028F3D094E8C8
:105080000F0002AD85E80F000021284604F002F869
:1050900007460028E7D096F87C32DB0704D439F0C5
:1050A0004BF9192138F0E0FE95E80F0006F51B7C5E
:1050B0008CE80F0096F87C3243F0010386F87C32CE
:1050C000304600F0DDFC42F093FF462143F0AEFD98
:1050D00042F08EFF452143F0A9FD054BA2681B68F5
:1050E000DB6A1A61E2685A6162689A61BCE700BFD4
:1050F000A425002038B5144B1B68DD6A2B680446D4
:105100005B6828469847F0B12B690BB96A69D2B140
:10511000C4F874326B69C4F87832A969002204F5C6
:105120001B7003F0F3FE94F87C3223F0030343F08A
:10513000030384F87C3242F05BFFBDE83840034A49
:1051400006213CF025B938BDA4250020E4380A0822
:1051500010B588B004460593FFF7A0FB0328059B14
:105160004FF000000AD10690079006A802900B9815
:1051700001900A98009020461BF0F2FF08B010BD85
:1051800038B50446FEF71CFE0546D0B194F80C3342
:10519000032B03D095F84E41204638BD20461BF026
:1051A0004BFFFF280446F5D001462846FEF7DCFDFC
:1051B0000028EFD021462846FEF7D2FD0028E9D08E
:1051C000EAE70446E8E7000008B590F80C33032B43
:1051D00005D014F00FFF90F9EB04C0B208BD1BF02E
:1051E0006FFE431CF9D1F4E708B590F80C3383B196
:1051F000032B03D1BDE808401BF05ABE37F00AFB71
:1052000040F6ED424FF4801137F0BCFA4FF0FF301A
:1052100008BD1846FCE7000090F80C33032B01D1C1
:105220001CF002BC7047000090F80C33032B01D136
:105230001BF08CBD704700001BF012BE10B5044679
:105240001EF080FC2046FEF7C3FD2046BDE810405E
:10525000FEF7C4BE90F80C330BB1032B01D11CF048
:105260005FBC00207047000030B500F57573044640
:105270000D460FCB85E80F0094F8E40330BD000025
:105280007FB5054668460E4603F03AFE95F87C3237
:10529000DB0703D40024204604B070BD69462846CD
:1052A000FFF7E2FF04460028F4D0694605F51B70BD
:1052B00004F012F886ED000AC6ED010AEBE70000E3
:1052C000D0F880330B6090F87C037047D0F88833B7
:1052D0000B6090F88503704730B500F5677304469E
:1052E0000D460FCB85E80F0094F8AC0330BD0000ED
:1052F00030B500F5836304460D460FCB85E80F00FB
:1053000094F8280430BD000010B500F22C4203468A
:105310000C4607CA84E8070093F8380410BD000063
:105320002DE9F0432DED028B8BB005460E46174656
:10533000FFF726FF014680462846FFF70BFD04468F
:10534000002848D0FEF73CFD4146FEF70FFD86EDF4
:10535000000A95F93032002B3ADD0DF08BFBFEF799
:10536000A7FE012834D90DF085FB90F8F432D5ED75
:10537000DE7ADFED5D8A96ED000AB02202FB0300C3
:1053800095F93032D0ED3B0A07EE103AF4EEE87AA8
:10539000B8EEC77AF1EE10FAB7EE008AB8BFF0EEB9
:1053A000487A37EE201A20EE270A70EEC70A40F23C
:1053B000B63015F06DFBD5EDDE7AF4EEE87AF1EE5D
:1053C00010FAB8BFF0EE487A80EE277A86ED007AC0
:1053D00001233B7003E095F8083333B93870204659
:1053E0000BB0BDEC028BBDE8F08395F80C334FF0A9
:1053F0000009CDF80490CDF80890CDF80C9043B199
:10540000032B10D0CDF81090CDF81490CDF8189053
:105410007CB902233B703246414605F23C4001F024
:1054200087FB0446DBE701A928461BF0F9FD04468B
:10543000E8E795F80C33002BEBD004A92846FFF7DA
:1054400063FF04460028E4D001A904A817F0A6FBD6
:1054500007A8CDED080A8DED091A8DED070A17F0A2
:10546000B1FF04A8B0EE408A17F0ACFF95F93032D6
:10547000002B30DD07EE903AF8EEE77A4FF47F70BC
:1054800070EE670A37EE801AF5EEC00AF1EE10FAF8
:1054900048BFDFED160AF4EE410AF1EE10FAB0EE65
:1054A000480AC8BFB0EE601A15F0F2FAB0EE408AB2
:1054B000D5EDDE7A9FED0C7AF4EEC77AF1EE10FAB4
:1054C000B7EE007AB8BFF0EE477A88EE277A03236A
:1054D00086ED007A7DE7B5EEC08AF1EE10FA48BF9E
:1054E0009FED028AE4E700BF0000003400000000E6
:1054F00010B50446FFF768FE84F80D032046FFF759
:1055000063FE84F80E032046FFF75EFE84F80F0367
:105510002046FFF769FE04F55A7184F8100320460F
:10552000FFF78CF884F8740300F0CAFA04F561728E
:1055300084EDDE0A04F560712046FFF7F1FE04F504
:10554000627184F87C032046FFF794F804F56371D8
:1055500084F885032046FFF7C1F804F5677184F8E5
:1055600098032046FFF7CCF804F56C7184F8AC037F
:105570002046FFF77FFB04F5707184F8BC032046DA
:10558000FFF746FB04F5757184F8D0032046FFF75A
:105590002DF804F57A7184F8E4032046FFF718FB30
:1055A00084F8F8032046FFF7D5F804F5806384ED0E
:1055B000FF0A2046C3ED000AFFF7ECF804F20443AB
:1055C00083ED000A04F2144204F581612046FFF7DE
:1055D000F9FB04F583612046FFF79AFC04F22C41A5
:1055E00084F828042046FFF7F5F884F8380410BD45
:1055F00037B50D46044600F0FFF81DB914F0FAFC6B
:1056000013F0FCFA4FF4BE7204F5067101A811F014
:1056100043FB94F869322BB92046FFF76BFD012359
:1056200084F86932224B1D68A86A03689B69984711
:105630002046FEF71FFF2046FEF798FF204600F0A9
:1056400051FA2046FFF7DEF9286B30B10368D4ED3C
:10565000D20ADB6894EDD10A9847D4F8100208B159
:105660005CF032FB204600F07DF82046FFF724F97D
:1056700094F8903284F80C0383420ED084F89002A0
:1056800098B10C4D0C4B032808BF1D4642F0B0FCEE
:105690000A4A2B4606213BF07BFE2046FFF728FFF7
:1056A00001A811F01BFB03B030BD054DEEE700BFB4
:1056B000A42500202B0C0A08DB380A08FC380A084D
:1056C000E0380A08D0EDDE7A9FED057AF4EEC77A6D
:1056D000F1EE10FAB7EE000AA8BFB0EE670A704705
:1056E00000000034014B1868704700BF805D002047
:1056F0004FF0FF30704700000120704770470000F6
:10570000002070470020704770470000704700007D
:10571000002070470020704700207047002070472D
:10572000002070470020704700207047012070471C
:105730000368D3F894301847002070470020704762
:1057400000207047002070470020704700207047FD
:1057500000207047002070470020704700207047ED
:10576000704700007047000008B514F043FC90F843
:10577000EC0408BD08B514F03DFC90F8EB0408BD3E
:1057800030B52DED028B9FED1A1ADFED1A0A91ED5F
:10579000000A87B005462D200C468DED011ACDED8F
:1057A000000A15F075F99DED011ADDED000AF0EE25
:1057B000408A2E2094ED010A15F06AF99DED011A38
:1057C000DDED000AB0EE408A2F2094ED020A15F0BC
:1057D0005FF903A905F52570CDED038A8DED048AE7
:1057E0008DED050A35F0AAF807B0BDEC028B30BD8F
:1057F000C2B8323EC2B832BE10B504465BF0F6FA0B
:10580000D4F8F4321BB1C21AB2F57A7F12D30A4A25
:105810001268D26A92F89C2002B15BB9C4F8F40213
:1058200094F8314214F0E6FB80F8E24404F0BEFB49
:1058300080F8254010BD00BFA42500202DE9F043CD
:105840002DED028B91ED007AD1ED037A87B08DEDCD
:10585000047AB0EEC77AB5EEC07AF1EE10FADDE95F
:105860001087DDF84C90CDED057A0C4615461E46A6
:1058700006DCF0EEE77AF5EEC07AF1EE10FA02DD22
:1058800004A817F00DF96B20B7EE001AFFEE000A1E
:105890009DED050A15F0FCF86C2089ED000AB7EEC5
:1058A000001AFFEE000A9DED040A15F0F1F804A8B5
:1058B00088ED000A17F07CF8B7EE008A002852D075
:1058C0000023C9F8003088ED008AD4ED067A67EE2F
:1058D000A77AF4EEC87AF1EE10FA4ADB00233360BF
:1058E00085ED008ADFED3F0A96ED000A7C20B7EED9
:1058F000001A15F0CDF886ED000A95ED000A7D201E
:10590000B7EE001AFFEE000A15F0C2F885ED000AA6
:10591000D4ED067A129BDFED346AF1EE677AC3EDBF
:10592000007A96ED007AF0EEC77AF4EEE67AF1EEC0
:1059300010FA2BD503AB02AA01A9204615F000FDF1
:105940009DED018AB0EE480A83F0F0F985ED000A7A
:10595000B0EE480A83F040FB87ED000A07B0BDECCB
:10596000028BBDE8F08304A817F00EF80028A7D139
:10597000ABE738EE670A14F0BDFF86ED000A94ED40
:10598000087AC7EE007AC5ED007AABE794ED076AB6
:10599000C6EE077AC7ED007A96ED007AB0EEC77AC8
:1059A000B4EEE67AF1EE10FAC4D495ED007ADFEDAC
:1059B0000F6AB0EEC76AB4EE666AF1EE10FAB9DCAF
:1059C000B4EE477AF1EE10FAB4D6B0EEE77AB4EE60
:1059D000667AF1EE10FAADDCF4EE677AF1EE10FAC9
:1059E000BCD7A7E70000000000000034FFFF7F7F66
:1059F0001FB500F51773039300F51673029300F5B6
:105A00001573019300F51473009300F5127200F5FD
:105A1000137300F54871FFF711FF05B05DF804FB43
:105A20009FED156A90ED817ADFED146AD0ED837AEF
:105A300027EE067A67EE867A27EE267A67EEA67A52
:105A4000BDEEC77AFDEEE77A80ED7E7A90ED827A40
:105A500027EE067A17EE903A27EE267A002BB8BF8B
:105A600003F50C43BDEEC77AB8BFA03380ED7F7A53
:105A7000C0F80032704700BFE02E65420000C84207
:105A80001FB50E4B1B680446B3B1684603F038FAE5
:105A900069462046FFF72CFC20B16A4600212046CB
:105AA000FEF774FA94F87C32DB0705D504F51B7217
:105AB00001212046FEF76AFA04B010BD50600020B4
:105AC00008B502F031FABDE8084001F0BFBD0000A2
:105AD00010B580F8F81204465BF088F9C4F8FC02AF
:105AE00010BD000010B590F8F832044653B15BF0D9
:105AF0007DF9D4F8FC32C01AB0F57A7F84BF002358
:105B000084F8F83294F8003353B15BF06FF9D4F8AD
:105B10000433C01AB0F57A7F84BF002384F80033C1
:105B200010BD000000F5B6700B4607C883E80700FB
:105B3000012070470023C0F89C30C0F89830C0F8AE
:105B40009430C0F8A830C0F8A430C0F8A030C0F835
:105B5000AC30704770470000024B0B604FF07C5335
:105B600013607047000048427047000008B50B46BC
:105B700000F12801184616F06FFA012008BD000058
:105B800010B500F5C0700C460FC884E80F00204621
:105B900003F0A6F930B1FFF7A5FD00F51B700FC8A3
:105BA00084E80F00204603F09BF980F00100C0B2AA
:105BB00010BD000010B5044603F078FC204610BD6F
:105BC00010B5D0F8783104465BB15BF00FF9D4F82A
:105BD0007831C01A41F28833984294BF00200120E6
:105BE00010BD0120FCE7000013B50093036801928B
:105BF000D3F890309847DDE90021044628B90448DD
:105C0000044B0068C06A11F025FA204602B010BDAE
:105C1000A42500201C3A0A0813B504460191FEF79A
:105C2000CFF82368019A1B6D014608B190F84E1118
:105C3000204602B0BDE810401847000030B585B0DE
:105C4000002301930293039303680D46DB6D01A9C2
:105C50009847044620B1039B2B60204605B030BD19
:105C600002F062F9417C01F02DFE04460028F4D0D8
:105C700002F05AF901F08CFDB1EE400A85ED000A00
:105C8000EBE7000090ED007ADFED0F7AB0EEC77A17
:105C9000B4EEE77AF1EE10FA14D590ED017AB0EE99
:105CA000C77AB4EEE77AF1EE10FA0BD590ED027AEE
:105CB000B0EEC77AB4EEE77AF1EE10FA4CBF0120ED
:105CC00000207047002070470000003410B5FEF738
:105CD00077F8044658B190F84E11FEF741F830B10C
:105CE00094F84E112046BDE81040FEF73DB8002064
:105CF00010BD000038B50D460CF0BCFE0446FEF7A2
:105D0000D7F9022881BF94F8F402B02303FB0040C6
:105D100000F5827089BF07C8002085E807000120D0
:105D200038BD00002DE9F0432DED028B8FB00368E4
:105D30000025DB6C0395049505950695029502A94F
:105D400004469847064638B1FFF7BAFEDDED027A01
:105D500027EE800A8DED020A0CF08CFEFEF7A8F902
:105D60000746002E50D0DDED027AD4ED6A6A94ED3C
:105D70006B7A23680B9527EE877A67EEA67A8DED0E
:105D8000097ACDED0A7A0C950D959B6C0BA92046EE
:105D900009AD98470BA9284616F070FD012F8DED2F
:105DA000030ACDED040A40F2B3800CF063FE90F8D4
:105DB000F432DFED5B7AB02505FB030090ED3C8A01
:105DC00028EE278AB0EE480A82F0B0FFF0EE408A53
:105DD000B0EE480A83F000F9CDED0B8A8DED0C0A88
:105DE0000CF048FE90F8F43205FB030090ED3B0AFE
:105DF0000BA816F063FD09AD8DED050ACDED060A81
:105E000005A896BB03C885E00128CED89DED020AFF
:105E1000B5EEC00AF1EE10FA7FDD07AED4F8AC2182
:105E2000D4F8A83107923046089316F065FD236830
:105E30000B950C950D959B6C0BA920469847DDEDB5
:105E4000077A9DED0B7A77EE877A9DED0C7ACDED92
:105E5000077ADDED087A77EE877A09ABCDED087A1F
:105E600096E8030083E8030049E0236993ED000A04
:105E7000B7EE008A38EE408A16F020FD04F5C879A6
:105E80008DED090A4846B0EE480ACDED0A0A16F033
:105E900015FD0BA92846CDED0C0A8DED0B0A16F069
:105EA000EDFC04F5D07603AFC4ED650A314684ED10
:105EB000640A384616F0F2FC04F5CC788DED090A38
:105EC0004046B0EE480ACDED0A0A16F0F7FC0BA9E1
:105ED00028468DED0B0ACDED0C0A16F0CFFC97E8A5
:105EE000030084ED660AC4ED670A86E803004946AC
:105EF000404616F0C3FC8DED090ACDED0A0A9DED72
:105F0000090ADDED0A0A0FB0BDEC028BBDE8F08393
:105F1000DDE9030185E80300F1E709950A95EEE75D
:105F200035FA8E3C10B590F84213044603F058FC45
:105F30007C23C0B203FB0044D4F8A00010BD0000D5
:105F4000044B026F1B68DB6A5A60426F9A60826F73
:105F5000DA607047A4250020F0B58FB0044614F035
:105F600049F8002302930393049390F8EB1401ABD8
:105F700002AA054612F010FF04F19407D8B39DED74
:105F8000010AB5EEC00AF1EE10FA34DD02A816F0EF
:105F90002BFE04F1B00684ED2C0AC4ED2D0A84ED2D
:105FA0002E1A3946304616F02FFE04F17C01304699
:105FB00016F0DEFD04F1880105A88DED050ACDED92
:105FC000060A8DED071A16F0D3FD08A88DED080A14
:105FD0009DED010ACDED090A8DED0A1A16F0F4FDCA
:105FE0000BA904F128008DED0B0ACDED0C0A8DED07
:105FF0000D1A15F051FA95F8EB040C2303FB005031
:10600000394600F55C7016F0B3FD84ED2C0AC4ED42
:106010002D0A84ED2E1A0FB0F0BD00002DE9F047D7
:10602000824B00251F682DED028BC0F89C50C0F8F4
:106030009850C0F89450C0F88450C0F88050C5679C
:10604000C0F89050C0F88C50C0F88850C0F8B850D4
:10605000C0F8B450C0F8B0500446F86A03688AB07B
:106060005B680E46984704F12809002854D05AF07E
:10607000BDFE42F20F7398424ED8FB6A9FED6C8AC8
:1060800093ED010A84ED1C0AD3ED020AC4ED1D0A4A
:1060900093ED031A484684ED1E1A15F0F1F841F00D
:1060A000A7FFD4ED1E7A67EE887A054617EE900AB0
:1060B000FAF72AFAD4ED1D7A67EE887ACDE9040161
:1060C00017EE900AFAF720FAD4ED1C7A67EE887A78
:1060D000CDE9020117EE900AFAF716FA554ACDE912
:1060E0000001062128463BF053F994ED1E8AB0EEDC
:1060F000480A82F01BFE84ED6B0AB0EE480A82F07B
:106100006BFF84ED6A0A5AF071FEC4F87C010AB094
:10611000BDEC028BBDE8F087A6B194ED1C0AB4EE8D
:10612000400AF1EE10FA0DD6D4ED1D0AF4EE600A25
:10613000F1EE10FA06D694ED1E1AB4EE411AF1EE05
:1061400010FA52D713F056FF90F8EC344FF00C0AC7
:106150000AFB030303F50073074693E8070007AE45
:1061600086E807004FF01508B2EE028AF2EE068AC2
:10617000304617F027F9B4EEC80AF1EE10FA38D518
:1061800008F1FF3818F0FF083CD1304617F01AF933
:10619000F1EE047AB4EEE70AF1EE10FA43DD9DED7C
:1061A000090ADDED087A9DED078A20EE000AA7EEC8
:1061B000A70A83F027F9F0EE400AB0EE480A82F011
:1061C000D7FFDDED090A84ED1D0A9DED080AF1EE09
:1061D000600AB1EE400A82F0CBFF84ED1C0A9FED0D
:1061E000161AD4ED1D0A94ED1C0A484615F048F81D
:1061F0007BE7304617F0E6F8B4EEE80AF1EE10FA65
:10620000BEDCC2E7384612F017FC384612F0F6FC46
:1062100097F8EC340AFB037303F5007393E8070067
:1062200086E80700A4E725676567D8E7A42500206E
:10623000E02E6542283A0A08000000000021FFF71E
:10624000EDBE000037B5044608461546019117F02B
:10625000B9F8B7EE007AC7EE007AB4F8DC300198EE
:106260000133A4F8DC3094ED367A37EE277A84EDEA
:10627000367AB0EE007AF4EEC77AF1EE10FA06D56F
:10628000B6EE007AF4EEC77AF1EE10FA0DDC9FED6F
:106290000E7AF4EEC77AF1EE10FA13D59FED0B7A71
:1062A000F4EEC77AF1EE10FA0CDDB0EE670A16F0E4
:1062B0008BFC012085ED000AC5ED010A85ED021A6F
:1062C00003B030BD0020FBE700247449BD3786359C
:1062D00070B52DED028B00F1280600F134058AB06F
:1062E00029460446304616F0EBFCB6EE008A20EE56
:1062F000088A2846B0EE480A16F066FC07A9304620
:10630000CDED080A8DED091A8DED070A16F046FC51
:1063100030468DED010AB0EE480ACDED020A8DED52
:10632000031A16F051FC07A928468DED070ACDED9A
:10633000080A8DED091A16F031FC04A901A88DEDAB
:10634000040ACDED050A8DED061A16F0CDFC324695
:1063500001A920468DED070ACDED080A8DED091A39
:10636000FFF770FF58B95AF041FD0121C4F87801D8
:106370002046FFF753FE0AB0BDEC028B70BD2A46E3
:1063800004A92046FFF75EFF0028ECD004F140028C
:1063900007A92046FFF756FF0028E4D0EBE70000EE
:1063A00030B52DED028B0D4683B091F842130446B3
:1063B000284603F015FAC1B27C2000FB0151903150
:1063C00004F1280014F0ECFD68468DED000ACDEDD7
:1063D000010A16F013FBDFED1C7AB4EEE70AF1EECA
:1063E00010FA05D59FED190A03B0BDEC028B30BD44
:1063F000684616F055FB684616F0DAFA0028F1D127
:10640000284694ED488A03F05FFBF0EE400AB0EEB8
:10641000480A14F03BFA80B9284603F055FB84ED96
:10642000480AB0EE408A82F081FC84ED490AB0EE61
:10643000480A82F0D1FD84ED4A0A04F5927168465B
:1064400016F084FAD0E700BF00000034000000001E
:106450009FED0C7AB4EEC70AF1EE10FA0BD4DFED23
:106460000A7AB4EEE70AF1EE10FA07DCC0EE077A1A
:10647000B0EE670A7047F7EE007AF9E7F2EE047AB9
:10648000F6E700BFF3665F3F58A00B4108B51C302C
:1064900016F0B4FAF1EE007AB4EEE70AF1EE10FA73
:1064A0009DBFF1EE027A37EEC00ADFED047A9FED70
:1064B000040A98BF20EE270A08BD00BFCDCC4C3E91
:1064C000CDCCCC3D08B5836993F9000038B10CF010
:1064D000D1FAFDF7EDFD012894BF0020012008BD91
:1064E000F8B52DED028B054603F060FD03F05CFC72
:1064F0000446B8B3FFF7F6F890F8093393B328468B
:10650000FFF7E0FF064668B30CF0B4FA90F8F432F7
:10651000B02707FB030090ED3B7AF0EE087AB4EE6B
:10652000E77AF1EE10FA1DD495ED1E8A0CF0A2FA6E
:1065300090F8F432DFED1E7A07FB030090ED3C0A81
:1065400098EE270A14F026FADFED1A7AB0EEC00AA8
:10655000B4EEE70AF1EE10FA08DC5AF047FC3446D4
:10656000C5F86801BDEC028B2046F8BD05F5B67094
:1065700016F028FFB0EE408A0CF07CFA90F8F43266
:106580009FED0D7A07FB0303D3ED3B7A67EE877A25
:10659000B4EEE78AF1EE10FADFD55AF027FCD5F811
:1065A0006841001BB0F5FA6F8CBF00240124D9E7C5
:1065B000E02E654200003442CDCC4C3F10B50A4B72
:1065C0001B68DB6A93F89C3004465BB95AF00EFCFA
:1065D000D4F87C31C01A44F61F6398428CBF002067
:1065E000012010BD0020FCE7A4250020F8B52DED0A
:1065F000068B04460CF03EFA054603F0D7FC06462F
:1066000006F00EFA002840F0AB802046FFF768FF46
:10661000002800F0A8803046FFF784FCD4F8E8306A
:10662000984200F01A813046FFF77CFCD4F8E8303D
:10663000DFED8F7AC31A08EE903AF8EE688A30469A
:1066400068EEA78AFFF76EFC94F8BC30C4F8E80047
:10665000F3B9304603F0BAFBD0B104F1280796F83D
:1066600042233946304603F033FAD4ED1D0AB0EE2A
:10667000401A384694ED1C0A14F002FE0023C4F8B8
:106680009030C4F88C30C4F88830012384F8BC30D2
:1066900020463146FFF784FE95F8F40205EB00151D
:1066A000B0EE408AD5F8A030C4F8EC3004F1B00068
:1066B000D4ED129A16F086FE6368DFED6E7A93EDE4
:1066C000007AB4EEE77AF1EE10FA68EE299AB0EEAD
:1066D00040AA01D5C3ED007A2046B0EE4A0AFFF782
:1066E000B7FE636820EE299A93ED000A29EE009A1E
:1066F000FFF7CCFE29EE009A204684ED249AFFF79E
:106700005DFF38B1D4ED247AB2EE007A67EE877A75
:10671000C4ED247AF0EE007AF4EEE78AF1EE10FA96
:1067200010D5DFED557AB4EEE7AAF1EE10FA09D5EF
:10673000DFED527A69EEA79AD4ED2A7AE9EEA87ACB
:10674000C4ED2A7A9FED4E0A94ED397ADFED4D7A49
:10675000B0EEC88A28EE008AA7EE278A84ED398A2F
:10676000BDEC068BF8BDFEF7BDFF90F80933002B9A
:1067700073D02046FFF7A6FE00286ED095F8F422CD
:1067800005EB0213D3F8A010D4F8EC308B4264D0A0
:10679000B02606FB025292ED3B7AF0EE087AB4EE98
:1067A000E77AF1EE10FA58DBCB1AC4F8EC1008EED9
:1067B000903A95F8F4329FED341A94ED1E0ADFED0D
:1067C000337A06FB0353D3ED3C9A69EE819AF8EED7
:1067D000688A39EEC00A68EEA78A14F045F9B0EE6F
:1067E000409A82F0F9FB94F8BC30B0EE408AF3B1E5
:1067F000F3EE047AF4EEE78AF1EE10FA17DC95F87E
:10680000F40206FB005595ED3B7AF2EE027AB4EE07
:10681000E77AF1EE10FAFFF649AFDFED1D7AB0EE40
:10682000C99AB4EEE79AF1EE10FAFFF63FAF9FED8A
:10683000198AD4ED1D0A94ED1C0AB0EE691A04F110
:10684000280014F01DFD012384ED248A84ED238AA1
:1068500084ED228A84F8BC3028E7BDEC068B04F175
:1068600088009FED0D0ABDE8F84016F001BA00BFA0
:10687000BD378635CDCC4C3DC2B8B23E0AD7233C9D
:10688000CDCC4C3ECDCC4C3F35FA8E3C6F12833A8A
:106890001904863F00000000EC51783F30B50C230E
:1068A00003FB010101F1C003144693E807008BB01C
:1068B00004AD85E8070094E8070083E80700284650
:1068C000FFF7E0F907AB58B194E8070083E8070049
:1068D0009DED070ADDED080A9DED091A0BB030BDEC
:1068E00095E80700F2E70000F0B52DED028BD0F837
:1068F00030318B60D0F83431CB6085B004460D4622
:1069000001F012FB06460CF0B5F8A36993F90030CC
:10691000022B07464BD1FDF7CBFB022847D997F84E
:10692000F432B02202FB0373D3F8E01000222846B1
:1069300002F0ECFAD4ED500A94ED4F0A284602F02A
:10694000A1FD94F8443163B35AF050FA9FED228AC6
:1069500097F8F4128DED018A01AA064638460BF02D
:106960000DF9D4F838019FED1D0A361A07EE906A2A
:10697000F8EE677A4FF4876027EE800AB6EE001AC9
:10698000F0EE480A14F084F8DDED017A30EE270AC3
:1069900004F584708DED010A15F090FF284602F091
:1069A00071FD94F8440105B0BDEC028BF0BD707C24
:1069B000242303FB006696ED0B8AFEF793FED0EDD1
:1069C0009C7A9FED077AF8EEE77AE8EE077AFDEE1B
:1069D000E77A17EE901AA9E7000000006F12833AD9
:1069E0000000C842F8B5036F0B60436F4B60836FC4
:1069F0008B6000F14C050E46074601F10C040FCDEB
:106A00000FC40FCD0FC42B68236007F1B00207CA73
:106A100006F1300383E8070007F1940207CA06F184
:106A20003C0383E8070007F11C0207CA06F148038C
:106A300083E8070006F160013846FFF755FF86F846
:106A40007000F8BD30B589B0044668460D4602F0C6
:106A500057FA69462046FFF793F818B900242046F4
:106A600009B030BD04A802F04BFA204604A9FFF794
:106A70003BFF04460028F1D004A9684602F05AFC06
:106A800085ED000AC5ED010A85ED021AE7E7000071
:106A90001FB500230C4601A9019302930393FFF74E
:106AA000D1FF08B1039B236004B010BD30B585B0A1
:106AB00001AD00230C462946019302930393FFF78F
:106AC000C1FF034618B195E8030084E803001846A7
:106AD00005B030BDF8B506460F461546FDF770F90E
:106AE000044690B13946FDF73BF970B1204639466E
:106AF000FDF73AF9044640B1FDF762F93946FDF772
:106B000035F985ED000A2046F8BDFEF7EBFD90F85B
:106B1000083343B13046FFF7D5FC044618B1D6F828
:106B200064312B60EFE7D6F864312B600024EAE78C
:106B300070B52DED048B1646FFF7CCFF054670B3FC
:106B4000FEF7D0FD90F930424CB30BF093FFFDF708
:106B5000AFFA012823D9E4B207EE904AB8EE678A6B
:106B60000BF088FF90F8F43296ED009AB02202FB09
:106B70000300D0ED3B8AFEF7A3FF38EE281A78EE2B
:106B8000C80A40F2614029EE000A13F081FFB0EE1E
:106B9000408AFEF795FFC8EE007AC6ED007ABDEC9C
:106BA000048B284670BD000008B503F0FFF9BDE86E
:106BB000084003F0F9B8000010B5044616F0B0F82C
:106BC00050B904F10C0016F0ABF828B904F1180024
:106BD000BDE8104016F0A4B8012010BD38B500F192
:106BE000280504462846FFF7E7FF28B12046012183
:106BF000BDE83840FFF712BAD4ED107AB7EE007A4C
:106C0000F4EEC77AF1EE10FA06D5BFEE007AF4EE94
:106C1000C77AF1EE10FA12DC2046FFF759FB28463E
:106C2000FFF7CAFF0028E1D1D4ED107AB2EE047A62
:106C3000F0EEE77AF4EEC77AF1EE10FAD6DC38BD62
:106C400010B5044616F0BEFB2046BDE8104016F015
:106C500023B800002DE9F04F2DED028BA3B00027E3
:106C60000446B0EE408A0A970B970C97FFF7BEFCDC
:106C700013F0C0F904F1F00B05465E464FF0000832
:106C800004F1280A95F8F131022B5FFA88F1A8BFC8
:106C900002238B423AD92846019111F0EBFD01996C
:106CA00080B310AB13AA284613971497159712F0C8
:106CB000D1F89DED100AB5EEC00AF1EE10FA21DD13
:106CC00013A815F091FF1CA950468DED1C0ACDEDBF
:106CD0001D0A8DED1E1A14F007F916A88DED160A7F
:106CE000B0EE480ACDED170A8DED181A15F06CFFBD
:106CF0001CA930468DED1C0ACDED1D0A8DED1E1A26
:106D000015F082FF08F101080C36BBE795F8EC148A
:106D10000C2303FB015101F50071504614F0E4F817
:106D200084ED070A94ED450AC4ED080A30EE088A9E
:106D300084ED091A84ED458A0BF09CFE0646FEF7A9
:106D4000D1FC90F8093302932046FFF7BBFB80B1DA
:106D50003046FDF7ADF902280BD996F8F4226169A7
:106D6000B02303FB026391F9001093F802018842FB
:106D700061DA94ED457ADFEDCC7AB4EEE77AF1EEA4
:106D800010FA62D494ED598AFEF7A0FF38B1FDF7EE
:106D900017F890F84E11FCF7E9FFB0EE408A236C2B
:106DA000626BA16A1E93B0EE480A1CA81D921C914A
:106DB00015F00AFF04F5B6710AA88DED0A0ACDEDAB
:106DC0000B0A8DED0C1A15F01FFF5AF00FF8002377
:106DD000019084F82C312046FFF774FB00286BD01B
:106DE00096F8F422B02101FB0262D2F8E430C4F834
:106DF000303196F8F43201FB0363D3F8E830C4F87D
:106E0000343159F0F3FF0123C4F83801C4F83C7160
:106E1000C4F8407184F84431D4F81831002B5ED1A5
:106E2000019BC4F818310AAB93E8070004F5847499
:106E300084E8070009E006EB0212D2F8A0200192D4
:106E40000199D4F818218A4204D123B0BDEC028BF9
:106E5000BDE8F08F03F5827393E8070094F82C31B6
:106E60000DF1280C8CE807001BB904F5847383E846
:106E700007000123604684F82C3104F5B67115F043
:106E80008DFE1CA904F14C008DED1C0ACDED1D0AF0
:106E90008DED1E1A14F056F8B5EEC00AF1EE10FA98
:106EA0008DED1C0AD8BF9FED810ACDED1D0A8DED39
:106EB0001E1A84ED590A8EE794ED457AD4ED4F7A87
:106EC000DDED0A6AE6EE877ADDED0B6AC4ED4F7AF6
:106ED000D4ED507AE7EE267AC4ED507A9CE7D4EDF3
:106EE000457A734B0D97F5EEC07AF1EE10FA0E97D6
:106EF0000F93AAD99FED6F7A94F82C3167EE877AB9
:106F0000B7EE007AC7EE278A1BB9029B002B00F070
:106F1000C380E36804F584710AA893ED008A15F034
:106F20003DFE28EE888A8DED1C0A1CA8B0EE480AAA
:106F3000CDED1D0A8DED1E1A15F046FE16A90DA801
:106F40008DED160ACDED170A8DED181A15F05CFEC1
:106F50000DA8FFF775FE0DA815F0FCFE20B159F045
:106F600045FFC4F8780170E701231822002116A814
:106F7000039384F0E3FA182200211CA884F0DEFABF
:106F80009FED4A8A05F20E530DF170084FF000098B
:106F90004FF0FF37059395F8F131022B1A465FFA4F
:106FA00089F1A8BF02228A4240F296808B42049166
:106FB0006BD9059B13F80930002B66D0B0EE680A38
:106FC000584615F055FEDDE90331002B66D00C2242
:106FD00022AB02FB0933A3F11802049220465A4661
:106FE0000693FFF75BFC069B03ED060A049BC3EDCB
:106FF000010A83ED021A4046FEF744FE002844D100
:107000004046FFF71DFE404615F0A4FE00283CD187
:107010000C2303FB09F222AB134407920DA9A3F141
:10702000300240460492069315F05EFE069B03ED87
:107030000C0A049B0DA9C3ED010A83ED021A404618
:1070400015F03EFE22AB079A03EB890303ED1A0A03
:1070500016AB981816F0B6F97A1C04D0B4EEC08AB4
:10706000F1EE10FA03DD4FFA89F7B0EE408A22AB59
:1070700003EB870353ED1A7AF5EE407AF1EE10FA3E
:10708000F7EE007A48BFB0EE678A09F1010908F10E
:107090000C080BF10C0B7EE7029B66E79BE80700F0
:1070A00088E80700A7E700BFCDCC4C3E00000000F9
:1070B000000080BF0AE81C41CDCC4C3ECDCC4C3FFB
:1070C000CDCC4C3D920A06BF920A063FC2B8B23EF2
:1070D000728A0E3C5B8218397B1C3FF440AF84F807
:1070E0001C712046FFF7FCF960B12046FFF7EAF972
:1070F000002840F0348122AA0C2303FB072300223E
:1071000043F8282C16AA07EB470895F8EB3402EB56
:10711000880895F8F0219A4240F23C812B4493F87C
:107120000C35002B00F0368195F8EC3495F8F12100
:107130009A4240F22F812B4493F80E35002B00F039
:1071400029810C2322AA4146504603FB072713F04E
:10715000F9FE07ED0C0A47ED0B0A07ED0A1A404647
:1071600015F0DEFD002840F02181404615F0F2FDCB
:10717000002840F01B815FED307A94ED387A28EEDC
:10718000278A5FED327AA7EE278A04F1B00084EDFA
:10719000388A16F017F9A3685FED377A93ED007A15
:1071A000B4EEE77AF1EE10FAB0EE408A00F1028117
:1071B0002046B0EE480AFFF74BF9404615F004FDB3
:1071C000A3688DED130ACDED140A8DED151A93ED1C
:1071D000000A13A815F0F8FC204684ED1F0AC4ED40
:1071E000200A84ED211AFFF7E9F928B1B2EE000A6E
:1071F00004F17C0015F03CFD029BB3B33046FCF774
:1072000057FF012831D996F8F402B02303FB00663A
:1072100096ED3B7AF0EE087AB4EEE77AF1EE10FAEA
:1072200023D595F8EC040C2303FB005595ED807AEB
:10723000F1EE0C7AB4EEE77AF1EE10FA15DBD4ED4C
:107240001D7A1FED607AF4EEC77AF1EE10FA0CDDCC
:107250001FED637AF4EEC77AF1EE10FA05D5B6EEBB
:10726000000A04F17C0015F003FD5FED687AB4EECE
:10727000E78AF1EE10FA22D51FED6B0A404615F0B1
:10728000A3FC10A88DED100A94ED450ACDED110A6E
:107290008DED121A15F098FC13A904F1A0008DEDE4
:1072A000130ACDED140A8DED151A15F0ADFCD4EDD1
:1072B0002B7A94ED457A77EE877AC4ED2B7A94EDAC
:1072C0002B7AF1EE047AB4EEE77AF1EE10FA4FF091
:1072D00000053BDB12F08EFE5FED827A94ED2B1AF7
:1072E00094ED280A21EE271A40F2C530F1EE410A4A
:1072F0008DED031ACDED020A13F0CAFB9DED031AC2
:10730000DDED020A84ED280A40F2C63094ED290A28
:1073100013F0BEFB9DED031ADDED020A84ED290A90
:1073200040F2C73094ED2A0A13F0B2FB04F1A00139
:1073300084ED2A0A04F1940015F066FCC4F8A85004
:10734000C4F8A450C4F8A050C4F8AC5018220021CE
:1073500004F1F00084F0F2F8C4F8145160E5E36839
:10736000F7EE000A93ED000A13F090FA00283FF4BC
:10737000C2AE94ED1C0AB0EEC00A81F02DFE0C23C3
:1073800022AA03FB072353ED0A7A27EE800A03EDB6
:107390000A0AB7E60C2322AA03FB0727002347F8B3
:1073A000283C47F82C3C47F8303CD8E62046FFF70D
:1073B00015FCD4E5C3ED007AFAE600BF2DE9F04DE7
:1073C0002DED048B9EB0044612F014FE00F59F6371
:1073D000D3ED007A90ED7F8AF4EE487AF1EE10FA60
:1073E00048BFB0EE678ADFED5C7AB4EEE78AF1EE73
:1073F00010FA0DDD1822002104F1F00084F09EF84F
:107400000023C4F814311EB0BDEC048BBDE8F08D30
:107410002046FEF7A1FD2046FEF75AFFB0EE480ACF
:107420002046FFF717FC2046FFF7D8FBFEF75AF976
:1074300014AD00F5347204F1280114A813F0D2FD44
:107440000FCD04F14C060FC60FCD0FC62B6833606D
:1074500004F1740204F1780304F1700104F14C00AA
:1074600013F06EFF94ED1E8AB0EE480A81F05EFCC8
:1074700084ED6B0AB0EE480A81F0AEFD204684ED43
:107480006A0AFEF75DFDFEF72DF904F5C071FDF700
:107490002FFF59F0ABFCD4F8B031C31A632BB2D92B
:1074A000C4F8B00136F048FF9FED2C9A054659F01C
:1074B000A5FCD4ED1C7A67EE897A074617EE900A90
:1074C0000E46F9F721F8D4ED1D7A67EE897A8246E7
:1074D00017EE900A8B46F9F717F894ED1E0A20EE86
:1074E000090A41EC180B13F03FFAD4F8740110EEBE
:1074F000108AF9F709F8CDE91201D4F87001F9F70B
:1075000003F8CDE91001D4F86C01F8F7FDFFCDE9DF
:107510000E01D4F8E400F8F7F7FFCDE90C01D4F838
:10752000E000F8F7F1FFCDE90A014046F8F7ECFF7B
:107530000B4B01930B4B0093CDE908018DED068BAE
:10754000CDE904ABCDE90276074B084A0849284645
:1075500036F034FB57E700BFCDCC4C3EE02E654201
:107560008D3A0A08973A0A08543A0A085E3A0A0815
:10757000E0380A0808B52DED048BB0EE609AF0EE05
:10758000408A00F011F9B0EE408A89EE280A81F0B5
:1075900059FEDFED0B7A20EE270A81F0EBFDDFEDDF
:1075A000097A38EE278ADFED087A28EE278AF7EE87
:1075B000007A37EEC00A28EE000ABDEC048B08BD45
:1075C00041D3423E33938843A1D81943FFF7D2BF3A
:1075D00008B52DED048B9FED189AF0EEE07AF4EEED
:1075E000C97AF1EE10FAF0EE408AB0EE608A1ED44D
:1075F00000F0DAF8DFED117A9FED117A70EE277A5C
:107600009FED100AE8EEC77A9FED0F7A27EE800A09
:10761000C8EE007A87EE270AB4EEC90AF1EE10FA36
:1076200005DBBDEC048BBDE8084081F0EBBEBDEC92
:10763000048BB7EE000A08BD000000343393884382
:10764000F4FDD43B48A18F43CDCC9C3F427CD0ED90
:10765000257A242101FB020292ED0B0AD2ED090AE0
:1076600030EE270AFFF7B4BF38B52DED088BDFEDFC
:1076700021AA9FED21AA9FED21BA0546B0EE409ABE
:10768000F0EE609AB0EE408A1524013CA4B25CB3DF
:10769000F0EE490A2846B0EE480AFFF76BFFF0EE1D
:1076A000490A70EE698A284638EE2A0AFFF762FF17
:1076B000B0EEE87A70EE697AB4EECA7AF1EE10FABA
:1076C00077EEE87A10D468EEAA8A40F2631088EE6A
:1076D000A70AB0EE4B1A38EE400AF0EE4A0A13F051
:1076E000D7F9B0EE408AD0E7B0EE480ABDEC088B7F
:1076F00038BD00BFCDCCCC3D0AD7233C0024744913
:10770000002343608360C360036143618361C3619D
:10771000002380F82030704790F82020531CDBB203
:10772000062B80F8203000EB820288BF002382ED18
:10773000010A88BF80F82030704700004FF0FF3307
:1077400010B543610E4BC0F8A8300023044680F802
:10775000C830A830FFF7D4FF0A4BC4F8A83004F5AE
:10776000867058F001FA084B08491C60204632F038
:1077700001FAD4F89030C4F89430204610BD00BF10
:10778000B43C0A08C43C0A08845D00205C3D0A0839
:1077900008B5A83038F09EFEDFED027A20EE270A09
:1077A00008BD00BF00007A4490ED3C0ADFED057A89
:1077B000B0EEC07AB4EEE77AF1EE10FA48BF90ED81
:1077C0003D0A70470000003473B5D0F8A430044679
:1077D0000E4663B159F00AFBD4F8A430C01A42F245
:1077E0000F73984203D894ED280A02B070BD114B74
:1077F0001D687DB195F84E112846FCF7B5FA48B1E1
:1078000095F84E1101AA2846FCF7A4FA10B19DED97
:10781000010AEAE7242101FB064494ED0A0ADFEDA0
:10782000067AB4EEE70AF1EE10FA58BFB0EE670A36
:10783000DBE700BF7C5D002000000C4208B561B1B1
:107840000378022B02D9064859F09EFA5A1C02709E
:1078500000EB83004160012008BD0846FCE700BF43
:107860007C3B0A082DE9F84305460E469146002464
:1078700000F13C082B78A34211DD00234A46314633
:1078800001200FF07DF8242363430746002158F8B8
:1078900003000FF085F8874204D00134EAE70020A6
:1078A000BDE8F8830120FBE7054B1B682BB141695C
:1078B0004A1C02D0184636F065BB0020704700BF56
:1078C0005060002002290BD8242303FB010191F80A
:1078D000390030B191F83A0018B191F83B00704787
:1078E000002070472DE9F047044659F07FFAD4F89C
:1078F000F86042F21073861B9E4288BFC4F8F800FD
:1079000000274FF0240942F2107A237CFDB2AB42EB
:107910001CD929462046FFF7D5FF70B109FB054861
:1079200098ED0D0AD8ED097AD4ED250A30EE270A34
:107930002046FFF799FE88ED0C0A564504D909FB4D
:107940000540303032F0EEFA0137DEE7617C204648
:10795000FFF73AFF84ED3D0ABDE8F08770B50446B5
:1079600086B059F043FAD4F89830C31AB3F57A7F49
:1079700005464FD3344B94ED257A1B68DFED336A0F
:10798000DB6AD4ED247A93F89C60B0EEC76AB4EE5B
:10799000E66AF1EE10FA32D5B0EEE76AB4EEE66AC6
:1079A000F1EE10FA2BD502A801F0AAFA96BBFDF76A
:1079B00099FE02A9FDF79CFC60B3DDED037A9FED13
:1079C000247AF8EEE77A67EE877AC4ED257AC4F870
:1079D0009850FDF787FEFDF753FA2046FFF782FF28
:1079E00040F006FB0546D4F89400F8F78DFD194ADF
:1079F000CDE900010621284639F0CAFC0AE037EE3D
:107A0000676AF7EE005AB0EEC66AB4EEE56AF1EEC8
:107A100010FA01DC06B070BDB0EEE76AB4EEE66ABB
:107A2000F1EE10FAF6D4002ECFD02046903080ED43
:107A3000007A32F077FA40F0DBFA074A012106B00B
:107A4000BDE8704039F0A4BCA4250020000000343B
:107A50000AD7233CBD3B0A08983B0A08F0B52DED38
:107A6000048B85B004464FF4537200F5867103A869
:107A70000FF012F9D4ED227AD4ED236A9FED796AE2
:107A8000637C37EEE67A2422B0EEC77AB4EEC67A8B
:107A9000F1EE10FAC1BF9FED747A67EE877A9FED21
:107AA000737AE6EE877A02FB03430025C4ED237A5E
:107AB00093F839602378E9B28B4206D904EB81034D
:107AC000013558685BF01EFBF4E7DFED698A9FED36
:107AD000698A9FED699A0027237CFDB2AB4264D985
:107AE000242303FB054393F83920002A5BD0D3ED10
:107AF0000C7AF4EEE87AF1EE10FA0BDBF4EE677A2A
:107B0000F1EE10FA06D6F0EEE77AF4EE487AF1EEEE
:107B100010FA04DD242303FB05435A6A1A63242365
:107B200003FB0543D3ED090AD3ED0D7A93F8382012
:107B300070EEA70AA2B993ED0C0A2046FFF746FDA6
:107B4000D4ED257A30EE670AB4EE400AF1EE10FA71
:107B500016D7242303FB0545002385F83A3022E09D
:107B6000012A09BFD3ED0C7A93ED0B0A77EEE00AF8
:107B7000D4ED3B7A04BF80EE897A87EE270AE3E7EB
:107B8000F0EEC07AF4EE487A2423F1EE10FA03FB0B
:107B90000545E1DC012385F83A30D4ED237A37EE50
:107BA000800A85ED0B0A013796E7627C2046114674
:107BB000FFF788FE48B1242101FB024292ED0B0A37
:107BC000D16904F1A80038F065FC94F99C10277C79
:107BD000002907DBB94205DACAB211462046FFF791
:107BE00071FE68B900226274D5B2AF4209D9294644
:107BF0002046FFF767FE01320028F5D0657400E0EB
:107C000062742046FFF7AAFE2046FFF74DFE10B132
:107C100020465CF08FFA637C242505FB034393F830
:107C20003930B34216D036F087FB4FF6FF7136F08D
:107C3000A9F978B1607C05FB004494F83930002B39
:107C400014BF00220422019236F076FB019A122121
:107C500036F02AF903A80FF041F805B0BDEC048B0B
:107C6000F0BD00BF0AD7233C0AD7A33C48E17A3FC6
:107C700000000034FFFF7F7F002019462DE9F04F00
:107C80000446007C0F4687B004F13A03002201212C
:107C9000D5B2A84203F1240305D903F8231C03F845
:107CA000241C0132F4E76F4B1E68F06A03685B68BE
:107CB000984740B140F09CF96B4A062107B0BDE8F7
:107CC000F04F39F065BB40F093F9684A062139F06E
:107CD0005FFB002303A904F18800039332F0E0FC6A
:107CE0000A2559F083F880462046FFF7B7FE59F081
:107CF0007DF8A0EB0800B0F5FA7F02D95C4801F0EE
:107D0000DDF8B06A03680A215B689847617C204609
:107D1000FFF7D8FD0028E7D0B06A036864215B68EC
:107D2000013D984715F0FF05DBD1524B05951B88A7
:107D30008DF80650CDE90355ADF80430052559F00E
:107D400055F880462046FFF789FE59F04FF8A0EB22
:107D50000800B0F5FA7FD1D8617C2046FFF7B2FD6C
:107D60000028EFD094F810B00DF10C08A14601AA3C
:107D70004FF0000A5FFA8AF18B4516D92046FFF7CB
:107D8000A1FD50B1D8ED007A99ED097A137877EE1C
:107D9000877A0133C8ED007A13700AF1010A08F1FD
:107DA000040809F124090132E4E7B06A0368642198
:107DB0005B68013D984715F0FF05C0D1A9464FF01B
:107DC0002408237C5FFA89F6B34226D906AB3344F4
:107DD00013F8143C33B908FB064686F83B3009F12A
:107DE0000109EEE7002FFAD007EE903A06AA02EB5F
:107DF0008602F8EEE77A12ED030AD4ED250A204652
:107E000080EE270AFFF730FC08FB064002A930305D
:107E10008DED020A32F044FCE1E7617CDFF85C9012
:107E20002046FFF7D1FC002684ED3D0A4FF02408E0
:107E3000237CF7B2BB420FD908FB074393F83B30D2
:107E400043B140F0D5F87B1C4A46062139F0A0FA30
:107E50000135EDB20136EBE70DB907484FE707B042
:107E6000BDE8F08FA4250020D83B0A08033C0A088F
:107E7000193C0A0878F70908553C0A08333C0A08F7
:107E800008B5037C022B02D9034858F07DFF5A1C29
:107E90000274184608BD00BF743C0A0838B5057C5A
:107EA00002460024E1B28D4206D91046FFF70AFDD2
:107EB00001340028F6D138BD281E18BF0120FAE78A
:107EC00070B50D4609780729044606D8027E437E20
:107ED00022B901228A401343437670BD002BFCD0A7
:107EE00000262278F3B29A42F7D904EB830329469D
:107EF00058680368DB6898470136F2E737B50D46E6
:107F00000192FFF7CBFF0199044630B90448054BB5
:107F100000682A46C06A0FF09DF8204603B030BDC5
:107F2000A425002027510B08014B1868704700BF9B
:107F3000845D002010B50446006810B103685B68DA
:107F40009847204610BD000013B500220B680A6058
:107F500001A901935BF026FC044601A8FFF7EAFFA4
:107F6000204602B010BD000013B500220B680A6065
:107F7000022201A901935CF011FE044601A8FFF75B
:107F8000D9FF204602B010BD13B500220B680A606D
:107F9000012201A901935CF001FE044601A8FFF74C
:107FA000C9FF204602B010BD13B500220B680A605D
:107FB00001A901935CF0F2FD044601A8FFF7BAFFA6
:107FC000204602B010BD000010B50446006810B194
:107FD00003685B689847204610BD00002DE9F04F0C
:107FE0008FB0D0F800310893344B354D1B680593A2
:107FF0000446586803689B68984794F99D3006903A
:10800000002BA2BF012606FA03F3069305F1D80A56
:108010002B68089A1A420BD000274FF0010BB94683
:10802000069A0BFA07F3134206D10137202FF7D136
:108030000C355545ECD12DE0F9B26B682A7A0991DF
:1080400020460793FFF70EFC0999804628B3CDE937
:108050000A990B9B0D930DA9079BCDE90B9920461F
:10806000984701462046FFF7E9FB0DA8FFF762FF9E
:108070000CA8FFF75FFF0BA8FFF7A6FFB8F1000FF2
:1080800002D00AA8FFF7A0FF2378032B02D0237C9D
:10809000032BCAD10FB0BDE8F08F059B58680422AE
:1080A0000368CDE90182074A00921B680A461E4612
:1080B00001462B7A0BA8B047CBE700BFA4250020D0
:1080C0004C3E0A08801A060070B5D0ED247A9FED68
:1080D000837AF0EEE77AF4EEC77A0123F1EE10FA34
:1080E0008AB00446037609D49030002309A905908C
:1080F000099332F0D5FA059831F014FF0026E663B3
:108100002666C4F88460762231462046FFF7AAFB33
:10811000054600286CD0CDE90666079A099200232F
:1081200009A92046CDE907335AF07EFB01462046D7
:10813000FFF784FB09A8FFF7FDFE08A8FFF7FAFE8A
:1081400007A8FFF741FF15B106A8FFF73DFF237809
:10815000032B00F09580237C032B00F09180762286
:1081600000212046FFF77EFB054600284FD0002364
:10817000CDE90633079A0992002309A92046CDE9E3
:1081800007335BF039FB01462046FFF757FB09A890
:10819000FFF7D0FE08A8FFF7CDFE07A8FFF714FFF2
:1081A00015B106A8FFF710FF2378032B68D0237CB6
:1081B000032B65D094F99D10002937DA2046FFF78C
:1081C0000DFFD4F80031DA046CD40025637EEB4057
:1081D000DB07EAB26CD40135082DF7D1237823B13F
:1081E000237C13B16368002B4AD13D4800F066FE42
:1081F0003C4B1B68596804220B68CDE901023A4ADE
:1082000000921E680246762307A8B04785E7354BE3
:108210001B68596804220B68CDE90102324A0092BA
:108220001E680246762307A8B047A3E77722C9B2A3
:108230002046FFF717FB054620B30023CDE90633A0
:10824000079B0993002209A92046CDE907225CF08B
:10825000A5FC01462046FFF7F1FA09A8FFF76AFEE0
:1082600008A8FFF767FE07A8FFF7AEFE15B106A83E
:10827000FFF7AAFE2378032B02D0237C032B9DD18A
:108280000AB070BD174B1B68596804220B68CDE912
:108290000102154A00921E6894F89D20772307A8D2
:1082A000B047CDE7637E002B8FD1012363768CE747
:1082B0003820059201F0F2F8064618B1059A2146D9
:1082C0005CF00AFD31462046FFF7B8FA2378032B0D
:1082D000D6D0237C032B7FF47EAFD1E7000000349F
:1082E000883C0A08A4250020801A060090F8603512
:1082F000934207D902F5A77250F8220010B1036823
:108300009B6A1847002070472DE9F34105466E46E9
:1083100086E80C00134B45F8043B04460F4600F575
:10832000C87828462C3500F0CFFCA845F9D196E84E
:10833000030004F26453C4F85C7583E80300089BEF
:10834000C4F86C350849204631F014FC074B1A6814
:1083500012B1074858F018FD20461C6002B0BDE875
:10836000F08100BF54410A081C400A08885D0020C3
:10837000603F0A082DE9F041A2B00C4607A930F091
:108380009BFD002855D000210D220CA80591ADF8C9
:1083900018100B9183F0D2F82B4B611C1F68C9B2E7
:1083A0000BAD0129F86A0A9546D1284B062205A98A
:1083B0000EF050FE264B019305AB009300241122D2
:1083C0002946244BF86A8DF819400EF043FE04AAA2
:1083D0000DF10F0128468DF83C40049432F03EF830
:1083E00038B31D49DFF86C80482210A883F05CF890
:1083F000062610AC2268531E049AC2F3513202EBD7
:10840000831223798DF82430A368019305AB009380
:108410000892434611222946F86A0EF01BFE0021FD
:10842000B7EE000A07A830F0F7FE013E04F10C0495
:10843000E0D122B0BDE8F0810091084B062205A9E9
:108440000EF008FEB6E700BFA4250020192E0A088A
:10845000913F0A088B3F0A087CF70908843F0A0805
:108460002DE9F04F90F8606585B00446002E59D193
:108470007F2380F870350DF10F0104232A308DF829
:108480000F3032F049F904F5C87504F5A768271DC7
:108490005FFA86FA1822FF21284683F04FF885F804
:1084A0005FA097F92690B9F10A0F5CD03DDCB9F1D5
:1084B000040F0FDCB9F1020F0FDD442000F0EEFFD6
:1084C000834620B13B462A4621465CF06BFFC8F844
:1084D00000B002E0B9F1090F39D0D8F8000050B16E
:1084E000696EC5F8609031B12C4B43F8261031F01D
:1084F0004FFD31F045FD58F8040B0AF101095FFA10
:1085000089F940B103689B68984784F860955146A3
:108510002046FFF72FFF0136092E05F1680507F108
:108520002C07B5D105B0BDE8F08FB9F1150F28D0F3
:10853000B9F1190FD1D1482000F0B0FF83460028CF
:10854000C5D03B462A4621465EF000F9BFE73820F9
:1085500000F0A4FF83460028B9D03B462A462146B6
:108560005DF086FBB3E7302000F098FF83460028DB
:10857000ADD0CDF800A03B462A4621465EF068F813
:10858000A5E7782000F08AFF834600289FD03B466D
:108590002A4621465DF0D4FB99E700BF8C5D0020A0
:1085A00090F860358B4283BF682303FB010090F88D
:1085B000DD0100207047000090F860358B4283BFDA
:1085C000682303FB010090ED6A0A9FED010A7047E2
:1085D0000000000090F860358B4206D901F5A771C4
:1085E00050F8210008B15DF07DB89FED010A704799
:1085F0000000000010B490F860458C420A4614D97F
:1086000001F5A77450F824407CB1E468246A64063C
:1086100003D55DF8044BFFF7DDBF682101FB0203C2
:1086200093ED6A0A5DF8044B70479FED010AF9E784
:108630000000000090F860358B420BD901F5A7715E
:1086400050F8210038B1C3681B6A1A4214BF0120D8
:10865000002070470020704770B590F86035934255
:1086600004460E46154601D8002070BD02F5A773DA
:1086700050F823000028F7D003689B69984700282A
:10868000F2D0682202FB0544D4F8AC313360ECE749
:1086900070B590F86035934204460E46154601D8F1
:1086A000002070BD02F5A77350F823000028F7D012
:1086B00003689B6998470028F2D0682202FB0544B2
:1086C000D4ED6C7AF4EE677AF1EE10FAE8D6C6EDE6
:1086D000007AE6E770B590F86035934204460E469E
:1086E000154601D8002070BD02F5A77350F823008D
:1086F0000028F7D003685B6998470028F2D0682209
:1087000002FB0544D4F8B4313360ECE790F86035EF
:1087100093420ED902F5A77350F823305BB168235A
:1087200003FB020292F8EC0130B1D2F8E8310B60A1
:1087300070470020704718467047000008299DBF09
:108740002C2303FB01004068002070472DE9F04F07
:108750004B4B2DED028B1B68DB6A93F89C3089B084
:108760000446002B00F08680DFF82CB19FED458A8F
:108770004FF0000994F860355FFA89F5AB4279D97A
:1087800005F5A77354F8230000285DD003685B6BE0
:108790009847682303FB0543074693F8DC3183427F
:1087A00052D2032861D8DFE800F04F025259364E0A
:1087B0004FF000083FF01CFC94F86025AA4284BFEB
:1087C000682202FB05424FF0680105F1010301FB3D
:1087D00005458CBFD2F8A82118EE102A8246D5F89C
:1087E000B001CDE90632F7F78FFE079ACDE9040113
:1087F0001046F7F789FE069B0096CDE902015A461E
:108800000421504638F0C4FD0123204A84F8713514
:1088100085F8DC71D372D4F86C354BB3002255B2B5
:108820005957481C03D0414502F10102F7D194F990
:108830007035AB4208DBD4F86835D4F8640542469D
:108840003146984784F8705509F1010992E72C23C5
:1088500003FB05430E4E93F92D80ABE72C2303FB5E
:1088600005430C4E93F92E80A4E70026B046A1E7FD
:108870001D46DCE709B0BDEC028BBDE8F08F00BF00
:10888000A425002000000000A53F0A08055E002086
:10889000EE5D0B089C3F0A08B43F0A0890F860356B
:1088A0008B4207D901F5A77150F8210010B1036878
:1088B000DB6918470020704708299CBF682303FB29
:1088C000010000F5C870704790F86035934207D9F1
:1088D00002F5A77250F8220010B103685B6A1847CE
:1088E0000020704790F860358B420DD901F5A773D1
:1088F00050F8233043B1682303FB0101012081EDCF
:10890000730A81F8C801704700207047F8B5002449
:1089100002460E4625462C2792F86035E1B28B427E
:1089200010D901F5A77352F823304BB107FB01238F
:108930009B689E4204D11046FFF7D4FF2843C5B27E
:108940000134E9E72846F8BD2DE9F04F002493B043
:1089500005460E46174621462F2206A8059405F522
:10896000A76982F0EBFD05F12A0A4FF02C0B05F503
:10897000F8730BFB04F259F8040B1AF90210E5B274
:1089800030B951B90134092CF3D14FF0010813E08B
:10899000682262439A58914212D01548154B0068DC
:1089A00001930135EDB20095134BC06A324639464A
:1089B0000EF050FB4FF00008404613B0BDE8F08FBA
:1089C00005A9332203935CF06FFF039B804605A942
:1089D0000028D7D1064801910135EDB20068009515
:1089E000054BC06A324639460EF034FBE4E700BF5F
:1089F000A4250020EA3F0A08DC3F0A082DE9F04FD1
:108A0000DFF88090DFF880A0DFF880B08DB00646F8
:108A1000002796F86035FCB2A3422ED9682505FBE5
:108A2000046595F8E43133B395F8E51119BB4FF0BF
:108A300001082022444404A889F8198082F07EFDB0
:108A400007EE904A4AF21043F8EEE77A03AA4C2167
:108A5000ADF8283050462423CDED037A3AF0AEFB32
:108A60003FF0C6FA9BF80030054A0094042138F024
:108A70008FFC85F8E5810137CBE70DB0BDE8F08FBD
:108A8000F43F0A08055E0020DD600020E822002097
:108A90002DE9F04F2F4B1E6885B0044646B1D0F843
:108AA0005C15304635F06EFA10B1304634F00AFAF3
:108AB00058F09CF94FF0000801904FF02C0A4FF04D
:108AC000680B94F860355FFA88F5AB4239D904EB4E
:108AD0008507D7F8380588B30AFB05430BFB054922
:108AE00093F92A20D9F8F0118A4227D132B30268CB
:108AF000D2689047D7F838050268126B904799F80A
:108B0000DD2112B1019BC9F8E031BEB1D4F85C158A
:108B1000304635F037FA88B158F070F9CDE90210D7
:108B200002460B46D7F8380529465DF003FCDDE91F
:108B30000232D7F8380529465DF07AFC08F10108C1
:108B4000BFE72046FFF702FE204605B0BDE8F04F24
:108B5000FFF754BF506000202DE9F0474FF00008A8
:108B60002DED028B04468946B0EE408A4746012629
:108B70004FF0680A94F860355FFA88F5AB421AD96D
:108B800029FA05F3DB070AD505F5A77354F8230086
:108B900078B10368B0EE480A9B6B984706400AFB21
:108BA000054508F1010895F8DC319F4238BF1F46A2
:108BB000E0E70646F3E727B97F23A4F87035034BB7
:108BC000DF72BDEC028B3046BDE8F087055E002009
:108BD00090F860358B4207D901F5A77150F8210054
:108BE00010B10368DB6B1847002070470B46114635
:108BF00090F860259A4207D903F5A77350F823002F
:108C000010B103681B6C18477047000070B504462C
:108C10000E46002594F86035E9B28B4205D93246FC
:108C20002046FFF7E3FF0135F4E770BD2DE9F84377
:108C300090F860550246002400F12A062C2700F522
:108C4000F8784FF06809E1B28D420FD907FB04F3C1
:108C500009FB04F0F35658F80000834209D11BB118
:108C60001046FFF79DFC10B10134ECE70120BDE890
:108C7000F8830020FBE7000010B590F860258A42D9
:108C8000044617D9682202FB010393F8DC31022B5A
:108C900003D004D9032B18BF0023184610BDFFF7DB
:108CA00097FF48B92046FFF7C1FF00280CBF0623F5
:108CB0000123F2E70023F0E70623EEE7014B1868F3
:108CC000704700BF885D002010B50349044630F0AE
:108CD00051FF204610BD00BFD4410A0810B504461C
:108CE000203049F061FB044B04491C60204630F001
:108CF00041FF204610BD00BFB05D002070430A0850
:108D00002DE9F3410022B7EE000A0221054630F0BA
:108D10009BFB28465DF06AFD49F0C0FB234B1E68B3
:108D20000446F06A03685B6A98470B4602210246D4
:108D30000091204649F04EFBB5F94A70002F13DD33
:108D4000D6F82C80D8F8003040465B68BCB2984713
:108D500028B198F84D3013B1C92FA8BFC824B06A04
:108D6000036821465B68984795F949002022002155
:108D700011F0CCFEC4B24CF051FA4CF0EFF970B9DE
:108D8000B06A036801345B68E4B205219847072C98
:108D9000F1D9074802B0BDE8F04157F0DDB8072C23
:108DA000F7D885F8494002B0BDE8F081A42500203D
:108DB000D4420A0810B504465DF0E6FC2046BDE842
:108DC00010405DF011BD00002DE98048284BDFF810
:108DD000A490DFF8A4A0DFF8A4B01446012293B059
:108DE00005460E461A704FF0000857F0FFFFD9F8FD
:108DF00000300393A0EB080241F287339A42074602
:108E00001FD9CDE9005603985346342205A9C06AFC
:108E10000EF020F9214605A8049457F08DF8CDE90D
:108E2000005603985B46342205A9C06A0EF012F979
:108E300004943FF0DDF8049B05AA022138F08EFA75
:108E4000B8463FF0D5F83EF06FFB3FF0D1F840F068
:108E500033FA0A2105A80DF005FF039B986A036801
:108E600005215B68984705A80DF008FFBDE700BF26
:108E7000B45D0020A425002075BA0A0891720B0881
:108E80000FB400B595B016AA002152F8043B039226
:108E900005A83C220193049182F050FB054A019BF6
:108EA000402104A856F0F0FF039A034804A9FFF7F5
:108EB0008BFF00BFEC420A0802430A080FB407B553
:108EC00004AA034852F8041B0192FFF77DFF00BF7C
:108ED00014430A08014B1868704700BFB05D0020BA
:108EE00008B50449102282F0CFFAB0FA80F04009A8
:108EF00008BD00BFB85D00201022002182F01EBB1B
:108F000010B50446FFF7F8FF204610BD0378416016
:108F100023F00D03022A037008D0032A0AD0012A85
:108F200003D1DBB243F0010303707047037843F0D1
:108F30000803F9E7037823F0050343F00503F3E79B
:108F400073B504460E4615460193FFF7D5FF20463C
:108F5000C4E90265069A0199FFF7D8FF02B070BD17
:108F60000078420704D4030704D400F001007047DE
:108F70000320704702207047F0B587B004461546BD
:108F8000FFF7EEFF88420F46064605D163682B6067
:108F90000126304607B0F0BD00230328019301D01D
:108FA000032913D132F06AFF08B90026F1E7012343
:108FB00001AA214632F09EFD0028F6D0DDED017AAF
:108FC0009FED337A67EE877ACDED017A032E32D8A2
:108FD000DFE806F0020916246468032FE5D8DFE80D
:108FE00007F02C2E3C49FCF77DFB90F87C32DB0728
:108FF000DBD56468FCF776FBD0F870321C44ECE7F4
:1090000002A8FFF779FFFCF76DFB02A9FCF770F9E6
:1090100006460028BDD06468039BEFE7D4ED017AD3
:109020009DED017AF8EEE77A77EE877AFDEEE77A42
:1090300017EE904AD1E70024CFE72C60A8E7FCF7B1
:1090400051FB90F87C6216F00106AED0FCF74AFBAB
:10905000D0F87032E41A2C609BE702A8FFF74CFFAF
:10906000FCF740FB02A9FCF743F90646002890D024
:10907000039BEFE707EE904A9DED017AF8EEE77A61
:1090800077EEC77AFDEEE77AC5ED007A80E700BF9C
:109090000000C84273B501AA05460E46FFF76CFFF3
:1090A000044620B1019932462846FFF72FFF20469B
:1090B00002B070BD13B5144601AAFFF75DFF48B1B9
:1090C000DDED017A9FED047AF8EEE77A67EE877AB4
:1090D000C4ED007A02B010BD0AD7233C07EE900A17
:1090E0009FED090AF8EEE77A08B527EE800A7FF0CF
:1090F0001DFEDFED067AB4EEE70AF1EE10FAD8BFF6
:10910000B0EE670A08BD00BF50E0EF300AD7233C3D
:1091100010B50446806811F07DFE20B1E068BDE81E
:10912000104011F08BBE10BD0D4B83424FF0000379
:109130008B4106DA00F1255000F5311000F5E050C2
:109140007047084B98424FF0FF3371EB0303BEBFEB
:1091500000F1564000F5130000F52440704700BFB1
:1091600000D2496B002EB69490EA010F01D4401A48
:109170007047C317401A63EBE1710D4B83424FF008
:1091800000038B4106DA00F1255000F5311000F59F
:10919000E0507047074B98424FF0FF3371EB0303E9
:1091A000BEBF00F1564000F5130000F524407047A3
:1091B00000D2496B002EB69470B52DED028B84B0B1
:1091C000044668460D46FFF797FEFCF78BFA6946A2
:1091D000FCF78EF8064608B3A368029ADFED128A00
:1091E00003999B1A07EE903AF8EEE77A67EEA87AB1
:1091F000C5ED007AE068FFF7B7FF08EE100AA06837
:10920000024402EBD272B8EEC88A5010FFF766FF34
:1092100028EE288A28EE000A85ED010A304604B0BF
:10922000BDEC028B70BD00BFF67C8E3F37B50023CE
:109230000C4601AA022105460193FFF79DFE10B9D5
:10924000002003B030BD21462846FFF7B5FF0028B7
:10925000F6D0DDED017AF8EEE77AC4ED027AF0E7B8
:1092600038B52DED028B0C460246C168E068FFF769
:109270007BFF9568A46808EE100A601900EBD070B7
:109280004010641BFFF72AFF07EE904AF8EEE77ADA
:10929000F8EEC80A87EE807ABDEEC70A10EE103AE3
:1092A0005B4200EE103AB8EEC00A7FF061FFDFEDDE
:1092B000087A30EE270ABDEC028BB5EEC00AF1EE5B
:1092C00010FA44BFDFED037A30EE270A38BD00BF45
:1092D000DB0FC93FDB0FC94030B52DED028B0B46CC
:1092E00085B08C68D0E90251D868FFF73DFF08EEE1
:1092F000100A601900EBD0704010FFF7EFFE641BFE
:1093000007EE904AF0EE400AB8EEC88A9FED060AD2
:10931000F8EEE77A28EE008A27EE800A68EE200A47
:1093200005B0BDEC028B30BD8262363C82B002B02B
:10933000FFF7D2BFF0B52DED028B0D4689B08C68DA
:109340000646D0E90271E868FFF70EFF08EE100A42
:10935000E01900EBD0704010FFF7C0FE73686A6838
:109360009FED0E1A9B1A07EE903AE41BB8EEE77ACF
:10937000F0EE400A07EE904A9FED090AB8EEC88A5F
:10938000F8EEE77A28EE008A27EE011A27EE800A27
:1093900068EE200A09B0BDEC028BF0BD0AD7233C71
:1093A0008262363C10B52DED028B84688A680B46CC
:1093B000111B08EE901AC168D868FFF7D5FE224449
:1093C00002EBD27208EE100A5010FFF787FEB8EEDB
:1093D000C88AF8EEE88A28EE000A20EE000AA8EE15
:1093E000A80A80F00FF8BDEC028BDFED027A20EEC8
:1093F000270A10BD8262363C094B984206DDC0F157
:10940000D64000F5930000F5A4407047054B984204
:10941000BEBFC0F1144000F5360000F5385070476B
:1094200000E9A43500175BCAF8B52DED028BDFED1E
:10943000148A076820EE280A0646FDEEC07A0D461B
:1094400017EE904A04EBD47007EB6000B0EE608A30
:10945000FFF744FE28EE288A3819C8EE007AFFF795
:10946000CBFF306017EE900AF7F778FD2B68C01835
:1094700041EBE371FFF758FEBDEC028B2860F8BDAD
:1094800002AAB34200F10C010830FFF7CDBF000083
:109490000148FFF731BD00BFB85D002001218842BF
:1094A00038BF08467DF004BDFFF7F8BF08B17DF076
:1094B00003BD7047FFF7FABF00214FF0FF3310B52F
:1094C00000220363044601600171C0F80510417277
:1094D00080F8251000F13C0300F50B70D9709A60FC
:1094E000DA601A615A619A61DA611A625A629A62A2
:1094F000DA631A645A649A64DA641A655A659A657A
:10950000DA65DA661A675A677C339842E6D12146F3
:1095100004F5167007F026FC044B1A6822B90449BA
:109520001C60204630F026FB204610BDC85D0020A0
:10953000D4450A0873B5D0F83C32019199420446EB
:1095400013D0D0F84032994218D0D0F844328B4230
:1095500016D102200AE0D4F8343253B3D4F83832AA
:109560004BB34FF0030002B070BD002094F82230DE
:109570008342F8D8431C84F82230F4E70120F5E751
:10958000D0F83062002EE6D194F841233546B6007B
:109590009AB1A319C3F83012A319019AC3F83C2257
:1095A00094F82230AB429CBF6B1C84F822302846D2
:1095B000D9E70126E8E70226E6E704F50C7001A9E1
:1095C000304431F07BF9E7E738B504460D4631F019
:1095D000EBF8291D201D31F0E7F805F1080104F131
:1095E000080031F0BBF905F1140104F1140031F069
:1095F000B5F905F1200104F1200031F0AFF905F1D2
:109600002C0104F12C0031F063F805F1300104F174
:10961000300031F06BF905F13C0104F13C0031F010
:109620009DF9AB6BA3636B6B636338BD2DE9F043AE
:10963000A1B00023002500F13C0706468DF8075035
:1096400003930493059306930793089309930A934E
:109650000B931093119312931393149315931693E2
:10966000179318931C931D931E9300F50F78B9461A
:1096700058F8043BF3B1F26E934223D0D6F8E820B9
:10968000934221D0D6F86421934213D10221EBB248
:1096900099420FD0C1EB411109EB8104214601A889
:1096A000FFF792FF39462046FFF78EFF01A93846A3
:1096B000FFF78AFF0135032D07F17C07D8D121B0D0
:1096C000BDE8F0830021E2E70121E0E72DE9F04762
:1096D00006460F461546804604464FF0000A3946B6
:1096E0003046FFF727FF626FBA425FFA8AF90ED160
:1096F000C3B2022B0BD87C2202FB0A66012086F83B
:109700003E0086F83F3085F80090BDE8F0870AF10A
:10971000010ABAF1030F04F17C04E0D100243946B8
:109720003046FFF707FFD8F86C205FFA84F912B9CA
:10973000C3B2022B22D90134032C08F17C08EED1EC
:1097400000244FF07C0906F13E0A39463046FFF707
:10975000F1FE034609FB04F05FFA84F81AF80020D2
:1097600012B9DBB2022B12D90134032CEDD196F8D9
:109770002300042814D9194857F006FB7C2000FB6D
:109780000464012084F83E0084F83F30BBE70644BF
:10979000012086F83E0086F83F3085F80080B4E767
:1097A00006F54371002251F8043BBB42D4B208D104
:1097B000A04202D8631C86F8233003342C700020AA
:1097C000A3E73BB9421C06EB800086F82320C0F8D3
:1097D0000C73F2E70132052AE5D1F0E710440A08DC
:1097E000C9B200EB8101D1F83C3253B1026F934210
:1097F0000AD0D0F8EC20934208D0D0F868219342E8
:1098000006D04FF0030070470020704701207047DA
:109810000220704759B190F82030032B07D05A1C12
:1098200080F8202000EB8300416101207047002078
:10983000704700002DE9F8430F469146044600F5B5
:10984000BA7894F83E5035B97C344445F9D10025B6
:109850002846BDE8F88300234A46394601200DF02A
:109860008FF800210646E06E0DF09AF88642EBD1A3
:10987000EEE700002DE9F043DFF87C8085B0044678
:1098800000F50F7600257C27B14656F80C3CD9F838
:1098900000209342E9B206F1040619D1C3B1204673
:1098A000FFF79EFFC0B207FB004090F83E307BB947
:1098B00003A9A9F10C00039331F000F83EF098FBE6
:1098C00056F8043C009342462B46012137F060FDD8
:1098D0000135032DD8D104F16C0504F5F074296825
:1098E00021B9AB6813B128462FF002FB7C35A542A5
:1098F000F5D105B0BDE8F0832C440A0838B504461C
:109900001546FFF76DFFC0B2022808D87C2303FB81
:10991000004029465030BDE8384031F00FB838BD1E
:1099200038B504461546FFF75BFFC0B2022808D8D9
:109930007C2303FB004029465C30BDE8384030F012
:10994000FDBF38BD37B50D4604468DED010AFFF762
:1099500047FF022D07D8C0B27C2303FB004001A9BA
:10996000683030F09DFE03B030BD000038B50546CC
:10997000FFF736FFC4B2022C13D8C4EB4414A40082
:109980003C3504F10800284400212FF0B1FA04F11D
:10999000340104F1300029442844BDE8384030F057
:1099A0008DBF38BD70B505460E461446FFF718FF4B
:1099B000C3B2022B0DD87C2000FB035394E80700B0
:1099C000443383E8070031462846BDE87040FFF77E
:1099D000CDBF70BD37B504461546FFF701FFC0B2D5
:1099E000022809D87C2303FB00400DF10701403019
:1099F0008DF8075030F0D8FE03B030BD10B500210F
:109A00000446FFF7B3FF20460121FFF7AFFF2046D2
:109A10000221BDE81040FFF7A9BF00001FB590F973
:109A20002C30044623B390F921300BB36846FFF77E
:109A300067FAFBF757FE6946FBF716FCC0B1DDED90
:109A4000037A9FED0C0AF8EEE70ADDED027AF8EEF4
:109A5000E77A0123C0EE800A84F83D3387EE800A5E
:109A600007F0C2FBDFED047A20EE270A84ED0A0A34
:109A700004B010BD8096184B35FA8E3C024690F922
:109A8000210058B192F8400340B1114491F92C02E1
:109A900020B192F92400033818BF0120704700005C
:109AA00038B590F8223005465BB100242346E1B278
:109AB0002846FFF7E3FF08B10133DBB20134032C82
:109AC000F5D1184638BD000090ED0A0A7047000035
:109AD00038B50C46D1ED066A11460546FFF780FE03
:109AE000C3B27C2000FB0353D4ED087AD3ED260AE1
:109AF00094ED076AD3ED255A93ED245A26EE600AB9
:109B000067EEA00AA5EEA70AF0EE607AE5EE867A87
:109B1000B7EE007AA6EEE67A67EEE60AB1EE400A04
:109B2000E5EE070A7FF024FB9FED071ADFED070A39
:109B300040F61C0010F0ACFFD5ED0A7ABDE83840C5
:109B400030EE270A10F090BFDB0F4940DB0F49C011
:109B50002DE9F04190F822308B4204460D4602D2A6
:109B60000020BDE8F081FFF73BFEC0B204F13C06E7
:109B7000C0EB401006EB8000083013F023FCDFED53
:109B8000157AB0EEC00AB4EEE70AF1EE10FAE7D4A7
:109B900029462046FFF724FEC5B27C2000FB05477E
:109BA0003B6F002BDCD0032DDAD000FB056030309A
:109BB000D7F86C8030F0B4F8D7E91B32934201D16A
:109BC000984505D07C2000FB0544C4F86C80C7E7AD
:109BD0000120C6E7000000342DE9F74F04460E4689
:109BE000174600F50F7A4FF0000B5AF8049B5FFA06
:109BF0008BF8B9F1000F26D041462046FFF73EFF13
:109C000008B341462046FFF7EBFD7C23C0B203FBBF
:109C1000004090F83E505DB908F101031B4ADBB2E9
:109C20003946304656F030F9284603B0BDE8F08F8B
:109C30005AF8102C914506D0154A3946304656F050
:109C400023F90025F0E70BF1010BBBF1030FCCD199
:109C50004FF0000894F822305FFA88F18B420DD95A
:109C600020460191FFF774FF054620B9019920466F
:109C7000FFF704FF20B908F10108EBE70125D3E75E
:109C8000044A3946304656F0FFF8CDE754440A08F6
:109C900069440A088E440A082DE9F0412DED048B31
:109CA00090F842139FED348ADFED348A9FED349AA9
:109CB00082B00646FFF794FD06F13C07C5B27C2052
:109CC00000FB057554354FF0000896F822205FFA26
:109CD00088F39A424ED919463046FFF7CFFE10B9A5
:109CE00008F10108F1E719463046FFF779FDC4B2E3
:109CF0007C2000FB0474D4ED157AF0EEE77AF4EEE4
:109D0000C87AF1EE10FA04F154040ED5D4ED017ABC
:109D1000F0EEE77AF4EEC87AF1EE10FA05D50020FD
:109D200002B0BDEC048BBDE8F0812946204613F05B
:109D300061FBB4EEE80AF1EE10FAF0DC29462046A9
:109D400012F070FEB4EEC90AF1EE10FAE7DC21461B
:109D5000284612F0A3FD68468DED000ACDED010AFC
:109D600012F04CFEDFED077AB4EEE70AF1EE10FADE
:109D7000B6DDD4E70120D3E700000034DB0FC93F94
:109D8000920A863F00004843022910B5044608D8CD
:109D9000FFF726FD7C23C0B203FB004494F83D008E
:109DA00010BD0020FCE7000013B590F842130191AC
:109DB0000446FFF7E9FF30B10199204602B0BDE843
:109DC0001040FFF75BBE02B010BD0000F7B590F980
:109DD00021500446002D73D090F84053002D6FD0D1
:109DE00090F84213FFF7D0FF94F83D33064613B9BD
:109DF0002046FFF713FE002594F82020EBB29A428C
:109E000007D904EB83030135586903689B689847B9
:109E1000F2E756F0EBFF0027224604F5BA7140F254
:109E2000F315D2F89C30C31AAB428CBF0023012338
:109E300082F83D307C32914247EA0307F1D194F930
:109E40002430032B07D194F83C33002B3BD0D4F8BB
:109E50003803002849D167B1236B013309D034F0AE
:109E60006BFA216B34F08EF818B134F065FA33F0E8
:109E70003DF994F92C32002B3AD194F92D32CBBB19
:109E800094F92E3213B1022384F8423394F842132A
:109E90002046FFF779FF8642054611D034F04CFA90
:109EA0004FF6FF7134F06EF850B1002D14BF002250
:109EB0000422019234F040FA019A032133F0F4FFB6
:109EC000284603B0F0BD012384F83C330420FFF79B
:109ED000E5FA054610B1214606F0DAFF94F9243080
:109EE000C4F83853032BB2D0B5E706F0DFFFB2E772
:109EF0000023C9E70123C7E738B590F921300446AC
:109F0000D3B190F84053BDB1FFF76AFCC0B202284C
:109F100012D87C2303FB0044D4ED1A7A9FED087A13
:109F2000F4EEC77AF1EE10FA06D4B7EE087AF4EE42
:109F3000C77AF1EE10FA00DD0025284638BD00BFD3
:109F4000ABAA2A3F70B5D0F8085315F40035044683
:109F50000E460DD190F840335BB90A78072A07D82E
:109F6000012303FA02F290F83F33134380F83F33A2
:109F700070BD94F82020EBB29A42F9D904EB830328
:109F8000314658690368DB6898470135F1E70000FE
:109F900038B505466C242B591BB1002128192EF029
:109FA000A7FF7C34B4F5F07FF5D138BD014B1868BC
:109FB000704700BFC85D00202DE9F04FB24BD3F8C9
:109FC00000800446D8F8040003688DB09B68984769
:109FD000002507464FF0010909FA05F33B4240F01E
:109FE00092820135202DF7D1D8F804000368DB6890
:109FF0009847002507464FF0010909FA05F33B424F
:10A0000040F0C3820135202DF7D1D8F80400036851
:10A010009B689847002507464FF0010909FA05F3A8
:10A020003B4240F0F1820135202DF7D1D8F80400F1
:10A0300003689B689847002507464FF0010909FA15
:10A0400005F33B4240F01C830135202DF7D1D8F8B1
:10A050000400DFF840B203689B689847002504902D
:10A06000049A0123AB40134240F046830135202D72
:10A07000F6D1D8F80400DFF81CB20368DB68984713
:10A0800000250490049A0123AB40134240F005845C
:10A090000135202DF6D1D8F804000368DB68984715
:10A0A000002507464FF0010909FA05F33B4240F04D
:10A0B000BF840135202DF7D1D8F804000368DB6890
:10A0C0009847002507464FF0010909FA05F33B427E
:10A0D00040F0ED840135202DF7D1D8F80400036855
:10A0E0009B689847002507464FF0010909FA05F3D8
:10A0F0003B4240F01B850135202DF7D1D8F80400F4
:10A1000003689B689847002507464FF0010909FA44
:10A1100005F33B4240F04A850135202DF7D1D8F8B0
:10A12000040003689B689847002507464FF0010923
:10A1300009FA05F33B4240F079850135202DF7D12E
:10A14000D8F804000368DB689847002507464FF0FD
:10A15000010909FA05F33B4240F0A4850135202DA1
:10A16000F7D14A4B089308AF0425D8F804000368D8
:10A170009B689847002683460123B34013EA0B0FE0
:10A1800040F0CB850136202EF6D1D8F804000368C4
:10A19000DB689847002683460123B34013EA0B0F80
:10A1A00040F001860136202EF6D1013D15F0FF0565
:10A1B00007F10107D9D1D8F8040003689B689847D4
:10A1C0004FF00109074609FA05F33B4240F02F869C
:10A1D0000135202DF7D1D8F804000368DB689847D3
:10A1E000002507464FF0010909FA05F33B4240F00C
:10A1F0005A860135202DF7D1D8F8040003689B68F2
:10A200009847002507464FF0010909FA05F33B423C
:10A2100040F085860135202DF7D1D8F80400036879
:10A22000DB689847002507464FF0010909FA05F356
:10A230003B4240F0B0860135202DF7D1144B0793F7
:10A24000D8F8040003689B689847002583460123DB
:10A25000AB4013EA0B0F41D000275FFA85F9D4F821
:10A26000083313F4803A31D107AB4946DB5D0493E0
:10A270001A462046FFF7DEFA049B0646002800F047
:10A28000C686CDE908AA07E0A42500200C0D0E0F14
:10A2900020212223801A0600099B0B930022012112
:10A2A0000BA8CDE9092204F06FFF01462046FFF715
:10A2B000B1FA0BA8FDF73EFE0AA8FDF73BFE09A880
:10A2C000FDF782FE16B108A8FDF77EFE94F8233054
:10A2D000052B00F048810137042FC0D10135202D16
:10A2E000B5D1D8F804000368DB6898470025834699
:10A2F0000123AB4013EA0B0F38D000275FFA85F932
:10A30000D4F8083313F4803A28D107AB4946DB5D13
:10A3100004931A462046FFF78DFA049B0646002850
:10A3200000F08486CDE908AA0022099B0B93114610
:10A330000BA8CDE9092204F027FF01462046FFF7CC
:10A3400069FA0BA8FDF7F6FD0AA8FDF7F3FD09A8C9
:10A35000FDF73AFE16B108A8FDF736FE94F8233053
:10A36000052B00F000810137042FC9D10135202DC4
:10A37000BED1D8F8040003689B689847002682463F
:10A380000123B34013EA0A0F31D010255FFA86F992
:10A39000D4F8083313F0080B20D12A46494620464A
:10A3A000FFF748FA0746002800F04F86CDE909BBC1
:10A3B0000A9B002201210BA8CDE90A2301F048FCE9
:10A3C00001462046FFF726FA0BA8FDF7FDFD0AA877
:10A3D000FDF7FAFD17B109A8FDF7F6FD94F8233053
:10A3E000052B00F0C0800135EDB2142DD0D101361F
:10A3F000202EC5D1D8F8040003689B689847002632
:10A4000082460123B34013EA0A0F34D014255FFAC1
:10A4100086F9D4F8083313F4001B24D12A464946A0
:10A420002046FFF707FA0746002800F02186CDE90D
:10A4300008BB099B0B93002201210BA8CDE909223F
:10A4400002F018F801462046FFF7E4F90BA8FDF7E3
:10A4500071FD0AA8FDF76EFD09A8FDF7B5FD17B15E
:10A4600008A8FDF7B1FD94F82330052B7BD001350A
:10A47000EDB2182DCDD10136202EC2D1D8F804006E
:10A480000368DB689847002682460123B34013EA3D
:10A490000A0F34D014255FFA86F9D4F8083313F480
:10A4A000001B24D12A4649462046FFF7C3F9074638
:10A4B000002800F0ED85CDE908BB0022099B0B9335
:10A4C00011460BA8CDE9092201F0D4FF0146204630
:10A4D000FFF7A0F90BA8FDF72DFD0AA8FDF72AFD4F
:10A4E00009A8FDF771FD17B108A8FDF76DFD94F8F7
:10A4F0002330052B37D00135EDB2182DCDD10136E3
:10A50000202EC2D12FE0D4F8083313F0010A25D150
:10A510005FFA85FB1E2259462046FFF78BF9064657
:10A5200020B3CDE908AA099A0B9200230822012141
:10A530000BA8CDE9093303F0C7FA01462046FFF71F
:10A5400069F90BA8FDF7F6FC0AA8FDF7F3FC09A8CA
:10A55000FDF73AFD16B108A8FDF736FD94F8233053
:10A56000052B7FF43EAD0DB0BDE8F08FD8F8041098
:10A5700004220B68CDE90102B84A0092D3F800A08A
:10A580005A461E2309A8D047CDE7D4F8083313F064
:10A59000010A24D15FFA85FB1E2259462046FFF7A7
:10A5A00049F9064608B3CDE908AA099B0B93062290
:10A5B00000210BA8CDE9091103F086FA01462046D7
:10A5C000FFF728F90BA8FDF7B5FC0AA8FDF7B2FCC8
:10A5D00009A8FDF7F9FC16B108A8FDF7F5FC94F8F9
:10A5E0002330052B7FF40EADBDE7D8F8041004220C
:10A5F0000B68CDE90102994A0092D3F800A05A46AF
:10A600001E2309A8D047D0E7D4F8083313F4805AA2
:10A6100021D15FFA85FB0D2259462046FFF70AF942
:10A620000646F0B1CDE909AA0A9B0022CDE90A232A
:10A63000012108220BA804F0B5FA01462046FFF7D5
:10A64000E9F80BA8FDF7C0FC0AA8FDF7BDFC16B1A0
:10A6500009A8FDF7B9FC94F82330052B7FF4E3AC8F
:10A6600081E7D8F8041004220B68CDE901027B4A87
:10A670000092D3F800A05A460D230AA8D047D3E78A
:10A68000D4F8083313F4801A21D15FFA85FB2C2209
:10A6900059462046FFF7CEF80646F0B1CDE909AAA3
:10A6A0000A9B0022CDE90A23012108220BA804F00D
:10A6B000A7FB01462046FFF7ADF80BA8FDF784FC89
:10A6C0000AA8FDF781FC16B109A8FDF77DFC94F8F6
:10A6D0002330052B7FF4B8AC45E7D8F804100422EA
:10A6E0000B68CDE901025D4A0092D3F800A05A46FA
:10A6F0002C230AA8D047D3E7D4F8083313F4807783
:10A700003FD15FFA85F90C2249462046FFF792F8BF
:10A710000646002800F08480CDE90677079B0A935F
:10A720004FF0000A692249462046CDF81CA0FFF7E9
:10A7300081F80746002800F08180CDE908AA099B2E
:10A740000B9300221A2309920BA901220AA801F0F7
:10A7500007F801462046FFF75DF80BA8FDF734FC2B
:10A7600009A8FDF731FC17B108A8FDF72DFC0AA8D0
:10A77000FDF72AFC07A8FDF727FC16B106A8FDF790
:10A7800023FC94F82330052B3FF4EDAED4F80833C6
:10A7900013F480777FF46AAC5FFA85F90C2249469E
:10A7A0002046FFF747F80646002859D0CDE906773E
:10A7B000079B0A934FF0000A682249462046CDF8CD
:10A7C0001CA0FFF737F80746002857D0CDE908AAA4
:10A7D000099B0B9300221A2309920BA901220AA8B4
:10A7E00000F0BEFF01462046FFF714F80BA8FDF766
:10A7F000EBFB09A8FDF7E8FB17B108A8FDF7E4FBA0
:10A800000AA8FDF7E1FB07A8FDF7DEFB16B106A8D5
:10A81000FDF7DAFB94F82330052B7FF427ACA2E692
:10A82000D8F8041004220B68CDF800B0CDE901027D
:10A830004A461F6807A80C23B8476FE7D8F80410EA
:10A8400004220B68CDF800B0CDE901024A46D3F8E6
:10A8500000A009A86923D04771E700BF801A06004D
:10A86000D8F8041004220B68CDF800B0CDE901023D
:10A870004A461F6807A80C23B84799E7D8F8041080
:10A8800004220B68CDF800B0CDE901024A46D3F8A6
:10A8900000A009A86823D0479AE7D4F8083313F436
:10A8A00080773DD15FFA85F90C2249462046FEF7B4
:10A8B000C1FF0646002800F08180CDE90677079B9E
:10A8C0000A934FF0000A692249462046CDF81CA0A1
:10A8D000FEF7B0FF074600287ED0CDE908AA099B05
:10A8E0000B9300221A230BA90AA8099200F038FF43
:10A8F00001462046FEF78EFF0BA8FDF765FB09A871
:10A90000FDF762FB17B108A8FDF75EFB0AA8FDF78B
:10A910005BFB07A8FDF758FB16B106A8FDF754FB33
:10A9200094F82330052B3FF41EAED4F8083313F40B
:10A9300080777FF4ADAB5FFA85F90C22494620465B
:10A94000FEF778FF0646002855D0CDE90677079B2D
:10A950000A934FF0000A682249462046CDF81CA011
:10A96000FEF768FF0746002853D0CDE908AA099BE7
:10A970000B9300221A230BA90AA8099200F0F0FEFB
:10A9800001462046FEF746FF0BA8FDF71DFB09A870
:10A99000FDF71AFB17B108A8FDF716FB0AA8FDF78B
:10A9A00013FB07A8FDF710FB16B106A8FDF70CFB7B
:10A9B00094F82330052B7FF46BABD4E5D8F8041062
:10A9C00004220B68CDF800B0CDE901024A461F68A9
:10A9D00007A80C23B84772E7D8F8041004220B68C4
:10A9E000CDF800B0CDE901024A46D3F800A009A88D
:10A9F0006923D04773E7D8F8041004220B68CDF818
:10AA000000B0CDE901024A461F6807A80C23B847E9
:10AA10009DE7D8F8041004220B68CDF800B0CDE90A
:10AA200001024A46D3F800A009A86823D0479EE750
:10AA3000D4F8083313F0200A24D15FFA85FB1C22D6
:10AA400059462046FEF7F6FE064608B3CDE908AAA9
:10AA50000022099B0B9311460BA8CDE9092203F0B4
:10AA600031FC01462046FEF7D5FE0BA8FDF762FA41
:10AA70000AA8FDF75FFA09A8FDF7A6FA16B108A81B
:10AA8000FDF7A2FA94F82330052B7FF412AB6AE5A8
:10AA9000D8F8041004220B68CDE90102B84A0092EC
:10AAA000D3F800A05A461C2309A8D047D0E7D4F811
:10AAB000083313F0200A24D15FFA85FB1E22594681
:10AAC0002046FEF7B7FE064608B3CDE908AA0022E5
:10AAD000099B0B9311460BA8CDE9092203F0F2FB69
:10AAE00001462046FEF796FE0BA8FDF723FA0AA8BA
:10AAF000FDF720FA09A8FDF767FA16B108A8FDF7D7
:10AB000063FA94F82330052B7FF4E4AA2BE5D8F8F8
:10AB1000041004220B68CDE90102994A0092D3F88F
:10AB200000A05A461E2309A8D047D0E7D4F808331E
:10AB300013F0200A25D15FFA85FB1C2259462046D6
:10AB4000FEF778FE064610B3CDE908AA099A0B92E3
:10AB50000023022201210BA8CDE9093303F0B2FB47
:10AB600001462046FEF756FE0BA8FDF7E3F90AA8BA
:10AB7000FDF7E0F909A8FDF727FA16B108A8FDF7D7
:10AB800023FA94F82330052B7FF4B5AAEBE4D8F828
:10AB9000041004220B68CDE90102794A0092D3F82F
:10ABA00000A05A461C2309A8D047CFE7D4F80833A1
:10ABB00013F0200A25D15FFA85FB1E225946204654
:10ABC000FEF738FE064610B3CDE908AA099A0B92A3
:10ABD0000023022201210BA8CDE9093303F072FB07
:10ABE00001462046FEF716FE0BA8FDF7A3F90AA8BA
:10ABF000FDF7A0F909A8FDF7E7F916B108A8FDF7D8
:10AC0000E3F994F82330052B7FF486AAABE4D8F857
:10AC1000041004220B68CDE90102594A0092D3F8CE
:10AC200000A05A461E2309A8D047CFE7D4F808331E
:10AC300013F0400A21D15FFA85FB0C2259462046C9
:10AC4000FEF7F8FD0646F0B1CDE909AA0A9B0022FD
:10AC5000CDE90A23012106220BA800F047FD014699
:10AC60002046FEF7D7FD0BA8FDF7AEF90AA8FDF7C1
:10AC7000ABF916B109A8FDF7A7F994F82330052B15
:10AC80007FF45BAA6FE4D8F8041004220B68CDE9C6
:10AC900001023B4A0092D3F800A05A460C230AA8AE
:10ACA000D047D3E7D4F8083313F0400A20D15FFA35
:10ACB00085FB0C2259462046FEF7BCFD0646E8B14E
:10ACC000CDE909AA00220A9B11460BA8CDE90A2367
:10ACD00000F00CFD01462046FEF79CFD0BA8FDF799
:10ACE00073F90AA8FDF770F916B109A8FDF76CF918
:10ACF00094F82330052B7FF431AA34E4D8F80410FB
:10AD000004220B68CDE901021D4A0092D3F800A08D
:10AD10005A460C230AA8D047D4E7D4F8083313F0D6
:10AD2000800A26D13B78F1B21A462046CDE90413B9
:10AD3000FEF780FDDDE90413814618B3CDE909AAC9
:10AD40000A9B0022CDE90A2301210C220BA803F063
:10AD500087F901462046FEF75DFD0BA8FDF734F9A3
:10AD60000AA8FDF731F9B9F1000F02D009A8FDF7E3
:10AD70002BF994F82330052B7FF404AAFFF7F3BBDB
:10AD8000801A0600D8F80400B84AD0F800E0009213
:10AD90004FF0040CCDE9019C0A46DEF800A0014604
:10ADA0000AA8D047CCE7D4F8083313F0800A26D19C
:10ADB0003B78F1B21A462046CDE90413FEF73AFD7E
:10ADC000DDE90413814608B3CDE909AA0A9B0022F4
:10ADD000CDE90A2300210C220BA803F041F901461A
:10ADE0002046FEF717FD0BA8FDF7EEF80AA8FDF7C1
:10ADF000EBF8B9F1000F02D009A8FDF7E5F894F8D7
:10AE00002330052B7FF4CEA9FFF7ADBBD8F80400A3
:10AE1000964AD0F800E000924FF0040CCDE9019C76
:10AE20000A46DEF800A001460AA8D047CEE7D4F8CB
:10AE3000083313F4004A20D15FFA85FB0C225946EF
:10AE40002046FEF7F7FC0646F0B1CDE909AA0A9BB9
:10AE5000002201210BA8CDE90A2302F077FF014669
:10AE60002046FEF7D7FC0BA8FDF7AEF80AA8FDF7C1
:10AE7000ABF816B109A8FDF7A7F894F82330052B15
:10AE80007FF4A6A9FFF76FBBD8F8041004220B6863
:10AE9000CDE90102754A0092D3F800A05A460C236E
:10AEA0000AA8D047D3E7D4F8083313F4004A20D1D6
:10AEB0005FFA85FB0C2259462046FEF7BBFC06468E
:10AEC000F0B1CDE909AA00220A9B11460BA8CDE9F1
:10AED0000A2302F03BFF01462046FEF79BFC0BA82D
:10AEE000FDF772F80AA8FDF76FF816B109A8FDF78B
:10AEF0006BF894F82330052B7FF47BA9FFF733BB65
:10AF0000D8F8041004220B68CDE90102574A0092D8
:10AF1000D3F800A05A460C230AA8D047D3E7D4F8A8
:10AF2000083313F4007A20D15FFA85FB30225946AA
:10AF30002046FEF77FFC0646F0B1CDE909AA0A9B40
:10AF4000002201210BA8CDE90A2303F087FC01466A
:10AF50002046FEF75FFC0BA8FDF736F80AA8FDF7C0
:10AF600033F816B109A8FDF72FF894F82330052B14
:10AF70007FF450A9FFF7F7BAD8F8041004220B6841
:10AF8000CDE90102394A0092D3F800A05A46302395
:10AF90000AA8D047D3E7D4F8083313F4007A20D1B5
:10AFA0005FFA85FB302259462046FEF743FC0646F1
:10AFB000F0B1CDE909AA00220A9B11460BA8CDE900
:10AFC0000A2303F04BFC01462046FEF723FC0BA8A6
:10AFD000FCF7FAFF0AA8FCF7F7FF16B109A8FCF77F
:10AFE000F3FF94F82330052B7FF425A9FFF7BBBAB4
:10AFF000D8F8041004220B68CDE901021B4A009224
:10B00000D3F800A05A4630230AA8D047D3E7D8F88F
:10B01000041004200A68CDE9016014480090D2F8B9
:10B0200000A009A84A46D047FFF736B9D8F804105F
:10B0300004200A68CDE901600C480090D2F800A015
:10B0400009A84A46D047FFF76FB9D8F80410042280
:10B050000B68CDE90102054A0092D3F800B04A46D8
:10B060002B460AA8D847FFF7A3B900BF801A0600ED
:10B07000D8F8041004220B68CDE901020C4A0092B2
:10B08000D3F800B04A462B4609A8D847FFF7D1B9F4
:10B09000D8F8041004220B68CDE90102044A00929A
:10B0A000D3F800B04A462B4609A8D847FFF705BA9F
:10B0B000801A060073B50446FEF77EFF94F823302D
:10B0C000052B32D0002594F83F33EB40DA07E9B284
:10B0D00016D40135082DF6D194F82330052B24D051
:10B0E00094F8203013B194F82230F3B9104B114981
:10B0F0001B68986903681B6802B0BDE87040184778
:10B10000D4F808339B030CD42C200191FEF7C6F928
:10B11000064610B1019903F019FC31462046FEF7AE
:10B1200079FB94F82330052BD3D102B070BD00BF5A
:10B13000A4250020A8440A082DE9F04F90F92130F9
:10B1400089B00446002B00F00481012300F50C7542
:10B1500080F84133024600F50F712B462E46D06E23
:10B16000002859D0002384F8413394F94030642BEF
:10B170005BD094F9BC30642B00F08D8094F93831A9
:10B18000642B00F08A80D4F830722FBB01A92046CE
:10B190002DF092FE00B30C230593012306978DF842
:10B1A0001830714B07936946BDF80430049704A822
:10B1B000ADF810308DF800702DF0FEFF9DF90010F5
:10B1C00051B1022908DC38B1C9B27C2303FB01412B
:10B1D0006C3128462FF08AFB94F841B3BBF1000F85
:10B1E0005DD0E36E6367D4F8E830C4F8F030D4F88B
:10B1F0006431C4F86C3194F8233003F1C30204EBDA
:10B2000082020021042B7CD852F8040B1061013318
:10B2100042F8041CDBB2F5E753F8040B0028A1D177
:10B220008B4202F17C029AD19FE7002066238DF8C1
:10B2300010307C2303FB004004A940302FF09AFA21
:10B2400004A920462DF038FE00289CD004238DF858
:10B2500018300023CDE90133039331230593694668
:10B2600004A82DF0A9FF059B28B108AA02EB8302D0
:10B27000009942F8E01C0133332B0593EFD953F0CA
:10B2800067F99DED031ADDED020A9DED010A6621C5
:10B2900053F01CF977E70120C8E70220C6E7012731
:10B2A000A94655F8043B23B1AB600137042FF7D111
:10B2B00097E7AA46B8465FFA88F3022BF5D8DAF882
:10B2C000002055F8043C9A4205D104A95046CDF817
:10B2D00010B02FF00BFB5AF8043B08F101020BB938
:10B2E0009046E8E704A906EB88000193CDF810B07A
:10B2F0002FF0FCFA019BAB6001A948462FF0F6FA4B
:10B30000D3E794F8413313B92046FEF78FF994F848
:10B3100022300BB3154B1B68986A036864215B6885
:10B3200098472046FEF752FD94F83E3003B9E36695
:10B3300094F8BA300BB9C4F8E83094F836310BB948
:10B34000C4F86431FAF7CEF9FAF756FA0123A4F8F3
:10B35000403309B0BDE8F08F2046FFF7ABFE94F80C
:10B360002230002BE0D0D5E70CE40A08A425002009
:10B3700070470000012070470120704743689868BB
:10B380007047000010B5054B03600446806A10B199
:10B3900003685B689847204610BD00BF68490A08EB
:10B3A000406803685B6A184733B46C46406884E8B9
:10B3B0000C0003689D6A94E80C00AC4602B030BCF7
:10B3C0006047000010B50446FFF7DCFF2046FEF79B
:10B3D0006DF8204610BD000040680BF003BA000075
:10B3E000406801230BF0FEB940680BF0D7B90000AC
:10B3F00040680A220BF07CB940680BF091B900005C
:10B4000040680BF013BA000090F82E2022B190F89B
:10B410002D10002201F06EB97047000073B504468C
:10B4200005250026A06A8DF8076003680DF1070264
:10B43000DB680121984778B19DF807300C2B09D0C3
:10B44000102B05D0092B07D184F8303002B070BD25
:10B450001523F9E71423F7E7013DE3D12846F5E783
:10B4600010B4806A03681C690822A44601235DF8B1
:10B47000044B31216047000010B4806A03681C69E6
:10B480000122A44600235DF8044B322160470000EE
:10B49000F0B50446806A036885B05B699847054645
:10B4A000002800F08480A06A03685B6998470368FD
:10B4B0009B689847A06A03689B69984760B93D4BB1
:10B4C0003D491B68986903681B6898472B682846A4
:10B4D000DB689847002667E02046FFF7CDFF00288D
:10B4E000F4D02046FFF79AFF0028EFD0A06A036847
:10B4F0000121DB6A98472046FFF7B2FF30B92D4B98
:10B500002E491B68986903681B68DEE7A06A036818
:10B51000DB69984730B9274B29491B68986903684C
:10B520001B68D2E7A06A94F83010012784F82E70C7
:10B5300003685B6A9847A06A03689B6A984704F1AE
:10B540002D020146204601F023F906460028BDD011
:10B55000A06A94F82D10036801919B6A984701999D
:10B560000246204601F018F994F82C302BB194F8DB
:10B570002D103A46204601F023F994F82F2094F834
:10B580002D10204601F03EF92B682846DB689847CD
:10B59000A06A029403681D6A0A4B039304AB13E983
:10B5A0000C0042F21071A847304605B0F0BD0646C7
:10B5B000FAE700BFA4250020D4480A08FA480A0880
:10B5C00019490A08BDB6010870B5002586B0CDE955
:10B5D000005500230446806A8DF8085005930393B4
:10B5E000049303686A469E6810210923B047A0B1FE
:10B5F0009DF8003013F0010615D194F83130013375
:10B60000DBB2052B84F8313007D12046FFF734FF39
:10B610002046FFF725FF84F83160A06A03681B6BA2
:10B62000984706B070BD9DF8083084F831501B076C
:10B63000F3D4BDF901309FED1F6A06EE903ABDF9D3
:10B64000033007EE103ABDF90530F8EEE66A07EE72
:10B65000903ACDED036AF0EEE66AB8EEC77AF8EEFE
:10B66000E77AF4EEC66AF1EE10FA8DED047ACDEDCC
:10B67000057A0DD5B0EEC77AB4EEC67AF1EE10FABF
:10B6800006D5F0EEE77AF4EEC67AF1EE10FAC4D4FD
:10B690009FED090A03A811F0EBFAB2EE040A03A821
:10B6A00011F0E6FA94F82D200A2303A9204601F0B0
:10B6B0000FF9B2E7000000349A99193EFFF784BFF2
:10B6C00010B5044B044640F8043BFCF77DFC2046D3
:10B6D00010BD00BF80490A0810B50446FFF7F0FF0F
:10B6E0002046FDF7E3FE204610BD0000F7B50368D5
:10B6F0000F4616461BB90024204603B0F0BD0024B7
:10B70000046008200193FDF7C9FE054620B1124BE5
:10B710000360019B4360019401A8FCF755FC002DD8
:10B72000E9D03420FDF7BAFE04460028E3D000F04B
:10B73000E1FE0A4BA562236084F82C7084F82F6028
:10B740002046FFF7A5FE05460028D5D123682046F0
:10B750005B6898472C46CFE780490A0868490A0881
:10B760002DE9F74F046806460D4690469946002C91
:10B770006CD00B68002B49D0236820465B6A984741
:10B7800003689B689847012328680DEB030200219A
:10B790000BF028F898B39DF80130EA2B2FD1DFF891
:10B7A000F0B04FF0060A28680023802206210AF034
:10B7B000F5FF20B3DBF80070B86A03680A215B6804
:10B7C0009847002328681A4606210AF0E7FFB0B11F
:10B7D000B86A03680A215B689847012328680DEB63
:10B7E000030206210AF0FEFF48B19DF8014014F063
:10B7F00040042FD00AF1FF3A1AF0FF0AD3D1306883
:10B8000003685B6A98470368DB68984700241DE07B
:10B81000022223460F2128680AF0C0FFB86A036895
:10B8200001215B689847306803685B6A9847036842
:10B83000DB689847336834604A46414601A8019363
:10B84000FFF754FF044601A8FCF7BEFB204603B0F7
:10B85000BDE8F08F224623460F2128680AF09EFF9C
:10B86000B86A036801215B68984702232146306863
:10B870000DEB03020AF0B6FF04460028C8D0B869F1
:10B88000024903681B689847B9E700BF40490A08A6
:10B89000A425002090F82C10002200F02BBF0000FF
:10B8A00070B504468CB00426013E76B2731C4AD0B3
:10B8B000A06A15236A465D210AF094FF0028F3D0A0
:10B8C000A06A152306AA5D210AF08CFF0546002810
:10B8D000EAD0152206A968467FF0D6FD0028E3D1FC
:10B8E0009DF8003084F82E309DF8073084F8303011
:10B8F0009DF8143084F83A309DF813309DF81020EC
:10B9000084F83B309DF80F3043EA0223A3879DF86B
:10B91000013084F82F309DF8083084F83130039BD3
:10B920009DF80C20C3F30F2363869DF80B3043EA88
:10B930000223A386049BC3F30F23E386019BC3F377
:10B940000F23238707E0054B05491B6898690368A7
:10B950001B689847002528460CB070BDA425002020
:10B96000B4490A082DE9FF4104460023806A8DF896
:10B9700007300368DFF868815B6A984703689B6853
:10B980009847A06A03680A219B6C9847A06A0A221C
:10B9900004210AF0ADFE0425013D6DB26B1C32D0CE
:10B9A00000234B21A06A82220AF0F8FED8F800603A
:10B9B0000746B06A036802215B689847002FEBD006
:10B9C00001231A464B21A06A0AF0E8FE0746B06A36
:10B9D000036802215B689847002FDDD0A06A01232D
:10B9E0000DF1070240210AF0FDFE0028D4D09DF899
:10B9F0000720322A10D0002DCED1B0693649036815
:10BA00001D683223A847A06A03685B6A98470368E9
:10BA1000DB68984700255BE02046FFF741FF0028E0
:10BA2000F1D0A06A0123172251210AF0B7FE0028A5
:10BA3000E9D05222A06A012311460AF0AFFE002885
:10BA4000E1D0A06A012338224C210AF0A7FE002889
:10BA5000D9D0A06A03685B6A98470368DB68984797
:10BA6000A06A05210AF05CFEA36A04F12C02996821
:10BA7000204600F08DFE054650B3A36A94F82C10C2
:10BA80009A68204600F088FE94F8442094F82C1020
:10BA9000204600F0B7FE94F845302BB194F82C10F6
:10BAA0000122204600F08CFEA06A036802219B6CF4
:10BAB0009847A06A029403689E6A084B039304ABFC
:10BAC00013E90C0044F21B11B04755F08FF92064C4
:10BAD000284604B0BDE8F081DC490A084DBC0108E5
:10BAE000A425002070B5858F90F93B60AD03B5FBB0
:10BAF000F2F2A2F5804404FB04F2D51190F83A204A
:10BB00000498D201624306FB05225212A03002F5CE
:10BB10008012424312134A43DB0003EB623000B24F
:10BB200070BD000010B5448E53005C43B0F938304E
:10BB3000C91A838FD31AB0F93620B0F934005343B1
:10BB400004F500449B10C3EBC13300EB24400449CF
:10BB500093FBF0F04FF400420EF0C8FF00B210BDAE
:10BB60000080FFFF10B52DED028B8AB0044608233C
:10BB7000806A05AA42210AF035FE18B1BDF81A20E4
:10BB8000D30719D4A06A0AF051FE55F02FF9236C9F
:10BB9000C31AFA2B0CD92064002382224B21A06AFD
:10BBA0000AF0FCFD0123A06A1A464B210AF0F6FDBB
:10BBB0000AB0BDEC028B10BDBDF9141094F9303001
:10BBC0000093920894F92E300392C9102046FFF793
:10BBD00089FFBDF9161094F93130039A009308EEED
:10BBE000900A94F92F30C9102046FFF77BFFBDF96A
:10BBF0001810039A491008EE100A2046FFF792FF2A
:10BC000007EE900AF8EEE88AF8EEE77AB8EEC88A0E
:10BC1000B3EE000A07A8CDED097ACDED078A8DEDC8
:10BC2000088A11F039F8B2EE040A07A811F020F8DA
:10BC300055F0DCF894F82C2020640A23204607A94C
:10BC400000F046FEA06A0AF0F1FDB1E7FFF78ABFF7
:10BC5000F7B503680D4616461BB90024204603B00D
:10BC6000F0BD002707604820CDE90073FDF716FC02
:10BC7000044650B100F03EFC0E4B2360019BA362D2
:10BC8000019784F8446084F8455001A8FCF752F904
:10BC90006846FCF74FF9002CDFD02046FFF762FE24
:10BCA00005460028DAD1236820465B6898472C4671
:10BCB000D4E700BF144A0A0810B5044B044640F804
:10BCC000283BFCF737F9204610BD00BF144A0A088C
:10BCD00010B50446FFF7F0FF2046FDF7E7FB2046CE
:10BCE00010BD000090F82C10002200F003BD0000F1
:10BCF000F8B504460D4617461E4600F0FBFB094BFF
:10BD000023602B68A362002200232A6084F82D7030
:10BD100084F82E6023656365A365E3652366636627
:10BD20002046F8BD2C4A0A08F8B51C4609331646C9
:10BD3000DB086A46A2EBC30300AF9D46806AA31CE2
:10BD40006A460AF04FFD054628B122460DF1020170
:10BD500030467FF0A9FB2846BD46F8BD2DE9F341EA
:10BD600006460F46144655F041F8114BD3F80080B3
:10BD70000546D8F82800036801215B68984701232D
:10BD80000DF1070207213046FFF7CEFF60B19DF8A5
:10BD90000730DA0702D4B7EB531F05D055F026F869
:10BDA000431BA342E5D3002002B0BDE8F08100BFF1
:10BDB000A42500202DE9F041DFF8608292B004460E
:10BDC00002AF002646F02002A06A0023D2B2502122
:10BDD0000AF0E4FC002800F00C810325013D6DB25F
:10BDE0006A1C00F00681D8F80030986A03684FF4A6
:10BDF00096719B68984701230DF106025521204654
:10BE0000FFF792FF002800F0F4809DF8063013F051
:10BE1000E00F40F0EE80DB07E0D502230DF10602D3
:10BE200052212046FFF780FF002800F0E280BDF895
:10BE3000063001365BBA202E27F8023BC2D1BDF88E
:10BE400024309DF826109FED6D7ADFED6D6A9FED31
:10BE50006D6A43F30B0207EE902A1B0903F470632B
:10BE6000BDF82620F8EEE77A0B4343F30B03C4ED4D
:10BE70000C7A07EE903A02F470639DF82820F8EEF1
:10BE8000E77A134343F30B03C4ED0D7A07EE903AC0
:10BE90009DF92230F8EEE77AC4ED0E7A07EE903A7B
:10BEA0009DF92930F8EEE77A67EE877A07EE103AC7
:10BEB000B8EEC77A9DF92A30C4ED0F7A27EE267ABC
:10BEC000DFED517A84ED107A07EE103AB8EEC77ABA
:10BED0009DF92B30E7EE267AC4ED117A07EE903A01
:10BEE000F8EEE77A9DF9233067EEA67ADFED476A30
:10BEF000C4ED127A07EE903A9DF92C3007EE103A15
:10BF0000B8EEC77A9DF92E3027EE267AF8EEE77A5A
:10BF100084ED147A67EE867A07EE103A9DF9303098
:10BF2000C4ED137A07EE903AF8EEE77A9DF92D30DA
:10BF300067EEA67AB8EEC77AC4ED167A27EE267AAF
:10BF400007EE903A84ED157AF8EEE77A9FED307AB5
:10BF50009DF92F3067EE877AC4ED177A07EE903A95
:10BF60009DF93130F8EEE77A06EE903A67EE877A7F
:10BF7000F8EEE66AC4ED187ADFED267ABDF93830BE
:10BF8000E6EE877A07EE103A9DF93230C4ED197A61
:10BF9000B8EEC77AF3EE077AE7EE067A07EE103AC4
:10BFA000DFED1D6AC4ED1A7AB8EEC77A27EE267A5D
:10BFB00084ED1B7A9DF9333007EE103AB8EEC77A5C
:10BFC0009DF9343027EE267A84ED1C7A07EE103A7C
:10BFD0009DF9353007EE903AB8EEC77AF8EEE77A79
:10BFE00027EE267A67EEA67A84ED1D7AC4ED1E7AD6
:10BFF00000E0002012B0BDE8F08100BFCDCC4C3E87
:10C000000000803B0000003B0AD7233C0000003DBD
:10C010000000803817B7D1B80AD7A33AA42500206A
:10C0200073B501230E460DF1070206210446FFF702
:10C030007BFE18B90025284602B070BD9DF8073078
:10C04000013B012B0CD80023A06A1A4606210AF0F6
:10C05000A5FB0028EED0062200212046FFF77EFE39
:10C06000A06A0023324606210AF098FB0546002804
:10C07000E0D0262231462046FFF770FEDBE70000C5
:10C0800013B501230DF1070207210446FFF74CFE0B
:10C0900010B9002002B010BD9DF807301B070CD569
:10C0A0000023A06A1A4606210AF078FB0028F0D087
:10C0B000062200212046FFF751FEA06A0023072236
:10C0C00006210AF06BFB0028E3D01322072120464B
:10C0D000FFF744FE0028DCD0A06A002305220621D9
:10C0E0000AF05CFB0028D4D0172205212046FFF778
:10C0F00035FE0028CDD001212046FFF791FFC9E78A
:10C10000F7B50446806A5B4F03685B6A984703682B
:10C110009B689847A06A03680A219B6C9847A06AAD
:10C120000A2204210AF0E4FA0525013D6DB26B1CD8
:10C1300000F09680A06A0023B6227E210AF02EFB32
:10C140000028F2D03B68986A036818215B686E4645
:10C1500098470123324600212046FFF7E5FD0028DD
:10C16000E3D09DF80030332BDFD12046FFF722FECD
:10C17000002875D0A06A0023802250210AF00EFB0F
:10C1800000286DD02046FFF77BFF002868D0A06A0A
:10C19000002386222E210AF001FB002860D0A06A2D
:10C1A0000023242204210AF0F9FA002858D0A06ABA
:10C1B0000023022206210AF0F1FA002850D01422AE
:10C1C00002212046FFF7CAFDA06A002307220521AD
:10C1D0000AF0E4FA002843D001212046FFF720FFAF
:10C1E00000283DD0A06A036803219B6C9847A06A91
:10C1F00003685B6A98470368DB689847A06A172161
:10C200000AF08EFAA36A04F12C029968204600F025
:10C21000BFFA054608B3A36A94F82C109A68204622
:10C2200000F0BAFA94F82E2094F82C10204600F072
:10C23000E9FA94F82D302BB194F82C100122204605
:10C2400000F0BEFAA06A03689F6A0B4B009401934A
:10C2500096E80C0042F21071B847284603B0F0BDD2
:10C26000A06A03685B6A98470368DB689847002503
:10C27000F3E700BFA425002071C4010810B586B003
:10C280000C236A4631210446FFF74EFD002800F0DA
:10C29000DF809DF801309DF80020DFED717ADFED41
:10C2A000715A1B0403EB02239DF8022003EB026387
:10C2B0001B1206EE903A9DF804309DF803201B04F3
:10C2C00003EB02239DF8052003EB02631B1207EE2C
:10C2D000103A9DF807309DF806201B0403EB02235B
:10C2E0009DF8082003EB02631B1206EE103A9DF83E
:10C2F0000A309DF809201B0403EB0223F8EEE66ADE
:10C30000B8EEC77A9DF80B2066EEA76A27EE277A6B
:10C31000B8EEC66ADFED547A03EB02631B1226EE19
:10C32000276A07EE903AF8EEE77A67EEA57AF5EE1F
:10C33000C07AF1EE10FA40F38D80DFED4C5A77EEC3
:10C34000E57AD4ED134A94ED0F5A94ED1C4AD4EDDE
:10C350001D3A94F82C20F7EE005A74EEA54AF0EE40
:10C36000632AA4EEA75A0A2303A9D4ED107AD4EDC8
:10C370000C4A77EEA57A2046E7EEA64AD4ED1A7A63
:10C3800075EE677A94ED145AF0EE646AD4ED174AAC
:10C39000E5EE276AB0EE655AA7EEA45AC6EE854AC6
:10C3A00094ED115AD4ED0D6A35EE255AE5EE076A83
:10C3B00094ED157AE7EE876A94ED187AB0EE655A37
:10C3C000A7EE875A86EE857A94ED125AD4ED0E6A5E
:10C3D00035EE255AE5EE066A94ED166A94ED195A83
:10C3E000E7EE866AB0EE656AA7EE856AF0EE657ADA
:10C3F00086EE863A94ED1B6AF0EE646AE6EE447AC5
:10C40000E6EE476A86EEA75AF0EE476AE4EE646A03
:10C41000C6EEA75AD4ED1E6AD4EE262AE6EE636A6B
:10C42000B2EE046A27EE667A65EE066AA2EEA47A98
:10C43000CDED036A65EE866ACDED046AC7EE276A24
:10C4400076EE837A67EE867ACDED057A00F040FAD3
:10C4500006B010BD44BFDFED055A77EEA57A70E750
:10C4600047ABE73B5B9E803AF61BEB3B85EBCB4152
:10C47000FFF704BF30B51346026885B00D461AB900
:10C480000024204605B030BD002101607C200193CE
:10C490000392FDF703F8044620B1019B2A4603A945
:10C4A000FFF726FC03A8FBF745FD002CE8D020464B
:10C4B000FFF726FE05460028E3D1236820465B6887
:10C4C00098472C46DDE7000010B5044B044640F8C1
:10C4D000283BFBF72FFD204610BD00BF2C4A0A0861
:10C4E00010B50446FFF7F0FF2046FCF7DFFF2046BB
:10C4F00010BD0000064B10B503600446FDF756FD65
:10C50000606004F1080053F02FFB204610BD00BF0F
:10C51000444A0A0873B50646144675687C2303FB33
:10C520000253C4EB441405EB8404084693F8A410AA
:10C53000019010F033FC94F93C3001983BB97368DA
:10C5400093F8251002B0BDE8704010F027BC94F8B5
:10C550004010F7E737B5446801917C2505FB02459B
:10C5600095F83F3004EB8304D4F84C325BB154F0BF
:10C570003DFCC5F89C000199D4F84C0203B0BDE81D
:10C58000304003F0A7BF03B030BD00002DE9F04FED
:10C59000C2EB421447684FEA840881460E4607F111
:10C5A0003C0B08F108018BB015465944304610F099
:10C5B0002BFBD9F8040029460BEB8404FDF79CFC07
:10C5C00038B17C2303FB057393ED1A0A304610F053
:10C5D0004FFB7C2303FB057393ED146ADFED3A7A7E
:10C5E000D3ED156AB0EEC67AB4EEE77AF1EE10FA42
:10C5F0000FD5B0EEE67AB4EEE77AF1EE10FA08D590
:10C6000094ED077AB0EEC77AB4EEE77AF1EE10FA5D
:10C610001BD47C2303FB0573D86D196E5A6E9B6D7A
:10C62000029003910490079101A831468DED016AB3
:10C63000CDED056A0692089209930EF055FC86ED41
:10C64000000AC6ED010A86ED021A7C2303FB05777A
:10C650000023C7F88C30C7F88830C7F88430D9F881
:10C66000040090F95C3208F13C0A08F14808DA4409
:10C67000D84463B15DB9414600F5167004F0E2FBA1
:10C68000414630460BB0BDE8F04F10F0BDBA90F90E
:10C690003430012B0BD190ED0E0A504610F094FA75
:10C6A00084ED120AC4ED130A84ED141AE8E7022B94
:10C6B000E6D1FCF703FB002201A9FBF7CDFF002820
:10C6C000DED09DED010AE8E70000003410B54368B4
:10C6D0007C2404FB023407C904F1900383E80700BB
:10C6E00054F084FBC4F89C0054F074FBC4F8A00020
:10C6F00010BD0000F0B5074685B00D46164600F1A6
:10C700000801A92203A80AF0C7FA7C687C2303FB6E
:10C710000543D3F8B42022B903A80AF0DFFA05B024
:10C72000F0BDBEB196ED007AD3ED2A7A67EE877A36
:10C73000C3ED2A7A96ED017AD3ED2B7A67EE877AEC
:10C74000C3ED2B7A96ED027AD3ED2C7A67EE877AD9
:10C75000C3ED2C7A7C2607EE902A06FB0541A83112
:10C76000B8EE670A0846019110F096FA01992A4638
:10C770003846FFF7ABFF06FB05410023C1F8B03098
:10C78000C1F8AC30C1F8A8300023C1F8B430C3E719
:10C790004068FCF79BBF0000F7B506464068019271
:10C7A0007C2707FB01000D466C3001A914462EF0D2
:10C7B0007DF8716807FB05152C6703B0F0BD00001C
:10C7C00007B540687C2303FB010393F93C30022B3F
:10C7D0000BD000F13C03C1EB411003EB80000DF1E5
:10C7E00007018DF807202DF0BBFF03B05DF804FBB7
:10C7F00043687C2202FB013191F93C00003818BFEC
:10C800000120704743687C2000FB013181F8A4209F
:10C8100070470000F8B5054608460F4610F09AFA32
:10C8200010B100242046F8BD384610F079FA0446CD
:10C830000028F6D16B6893F934637EB1384610F066
:10C84000C1FD95ED087ADFED1F7AF0EEC76AF4EED0
:10C85000E76AF1EE10FA03D585ED080A0124E1E755
:10C8600077EE407A30EE076AF0EEE77AC7EE866A36
:10C87000F6B207EE906A9FED146AF8EE677A26EE3C
:10C88000866AF4EEC67AF1EE10FA48BFB2EE046A98
:10C89000DFED0E7A45BF6B6A66EE866AB0EE676AB8
:10C8A00087EEA66A46BF01336B620124F7EE007A79
:10C8B00077EEC67A20EE060AA7EE270A85ED080A6B
:10C8C000B0E700BF0000003400004843CDCCCC3DB1
:10C8D0002DE9F74304460E4615461F46FFF71AFE9C
:10C8E0002A4631462046FFF735FE314620462A4685
:10C8F000FFF74CFE31462046FFF78CFF28B39B2202
:10C9000004F1080101A80AF0C7F964684FF07C0936
:10C9100009FB054808F1A8083146404610F074F9B3
:10C9200009FB0542D2F8B4100131C2F8B4104FB17E
:10C93000B94207D34908C2F8B410B0EE000A404625
:10C9400010F0AAF901A80AF0C9F903B0BDE8F08314
:10C9500010B50446FCF744FFC0B23C34C0EB4010B5
:10C9600004EB800010BD0000F8B50A4E044600F547
:10C97000167704F5137555F8040B08B104F0DEF8CA
:10C98000BD42F8D13368986A036801215B68984713
:10C99000EFE700BFA425002008B5FFF7E5FF000082
:10C9A000F0B5144E00EB810773780446D7F84C02BB
:10C9B0006FF3410387B00D467370C8B102F0ACFC51
:10C9C00068B1737843F0100373702C440023A37292
:10C9D000D7F84C0207B0BDE8F04002F021BCD7F810
:10C9E0004C12684602F0C8FC009B012BEDD1E8E731
:10C9F00007B0F0BD245E002070B506460D46002449
:10CA000045FA04F3DB07E1B202D53046FFF7C8FF71
:10CA10000134032CF4D170BDFF21FFF7EDBF0000FE
:10CA200030B500F5137587B000F5167455F8041B82
:10CA300021B9A542FAD1002007B030BD684602F006
:10CA40009BFC009B013B022BF3D80120F4E7000084
:10CA50002DE9F0472DED028B88B004460D46904637
:10CA6000B0EE408AFDF790F930B90026304608B0A4
:10CA7000BDEC028BBDE8F08729462046FCF7FEFF9F
:10CA800006460028F1D004EB8507D7F83C22D7F8FA
:10CA900030329A4206D03BF0ABFA5C4A032134F0C4
:10CAA00077FCE2E7D7F84C3283B94FF49870FCF783
:10CAB000F5FC814608B103F045F9C7F84C92B9F18D
:10CAC000000F03D13BF094FA514AE7E7B4F84A3239
:10CAD000D90711D505F0CEFF90F8382390F8F4323D
:10CAE00032B9B02202FB030090F8D130012B03D8F9
:10CAF0003BF07EFA474AD1E72046FFF791FF20B985
:10CB0000454A537843F00203537094F9353053B3D8
:10CB100029462046FFF71CFF90F90030002B53D028
:10CB200029462046FFF714FF90F80490B9F12B0F27
:10CB300019D829462046D7F84CA2FFF709FF94F9E7
:10CB4000353090F90020022BD4BF00210121012BA8
:10CB5000D4BF00230123003A009118BF01224946A7
:10CB6000504602F071FB631900229A7275B3D4ED3E
:10CB7000C10AB4F84822D7F84C0270EEA00A2B463E
:10CB8000B0EE480A414602F07FFB94F83E33002B9A
:10CB900031D1224A069412680127E773906A02682D
:10CBA000156D1F4A0792029309224FF40063CDE9E5
:10CBB000003208AA12E906001A4BA847C8B93BF090
:10CBC00017FA194A02216AE79946B2E72946204630
:10CBD000FFF7BEFE90F90030002BC8D0D4EDC10A9B
:10CBE000B4F84822D4F84C022B46B0EE480A41462D
:10CBF000C9E784F83E7300230DF1170104F1240006
:10CC00008DF817302DF0B6FD30E700BF544A0A0802
:10CC1000864A0A08A94A0A08245E0020A4250020A2
:10CC200099C90108C74A0A08D24A0A082DE9F04101
:10CC30002DED028B002443739DF82030837305464D
:10CC40000F469046B0EE408A264647FA04F3DB07CB
:10CC5000E1B210D5B0EE480A42462846FFF7F8FE8A
:10CC6000064640B939462846FFF7C6FEBDEC028BA2
:10CC70003046BDE8F0810134032CE6D1F6E7000030
:10CC8000F8B500242DED028B05460F46B0EE408A24
:10CC9000427383732646E1B2B0EE480A3A4628460C
:10CCA000FFF7D6FE0134002818BF0646032CF2D148
:10CCB000BDEC028B3046F8BDF0B500EB81030D46AC
:10CCC000D3F84C129BB0044611B900201BB0F0BD44
:10CCD0000BA802F035FB6319987A0028F6D10B9A5D
:10CCE000002A48D0042AF0D101229A720DAA07CA5C
:10CCF00002AB83E8070010AA07CA05AF87E8070060
:10CD000013AA07CA9DED180A08AE86E807001A465E
:10CD1000294620468DED010AFCF744FE3A46294695
:10CD20002046FCF7EBFD324629462046FCF7F8FD8D
:10CD30009DED010A29462046FCF704FE9DF864306B
:10CD400083B129462046FFF703FE90F900304BB12E
:10CD500094F93530012B05DD9DF85D2029462046EC
:10CD6000FCF738FE2046FFF75BFE20B9034A5378F4
:10CD700043F0040353700120A8E700BF245E0020A5
:10CD80002DE9F0410546884600F513770024012679
:10CD900057F8043BE1B26BB148FA04F3DB0709D55D
:10CDA0002846FFF789FF002857F8040C08BF002623
:10CDB00002F036FA0134032CEAD13046BDE8F081A6
:10CDC0002E4B2DE9F04F1F68FB6A93F89C8087B0CB
:10CDD0000446B8F1000F38D1DFF8A8A000F51376AB
:10CDE00000F1030B054656F8040BA5EB04095FFAA6
:10CDF00089F9E8B102F07CFA28B19AF8013043F0E1
:10CE000008038AF8013056F8040C02F085FAF8B9E4
:10CE1000637B6BB1AB7A5BB956F8041C684602F0D1
:10CE2000ABFA009B042B03D149462046FFF744FF91
:10CE300001355D45D7D1124B204683F81280FFF7AC
:10CE4000EFFD054630B10123237407B0BDE8F08F34
:10CE50008046EDE7237C002BF7D0A37B002BF4D09A
:10CE6000B86A03684FF47A715B689847B86A0368D8
:10CE70009B6B294607B0BDE8F04F1847A42500205A
:10CE8000055E0020245E0020F0B5002587B000F587
:10CE900013762C46012756F8041B41B1684602F070
:10CEA0006BFA009B1BB107FA05F31C43E4B2013592
:10CEB000032DF0D1204607B0F0BD00002DE9F04F62
:10CEC0002DED028B03270E7C9FED348A91B0054631
:10CED0008846B946AC5D0134E4B2B4FBF9F303EB28
:10CEE0004303E41AE4B205EB8403D3F84C1209B906
:10CEF000AC554CE003A802F03FFADDF80CB00BF1A2
:10CF0000FF33022BF4D8304635F0E6F9824630463E
:10CF100036F0E6F800F11B039A4508D2304634F0AB
:10CF200057FC002011B0BDEC028BBDE8F08FAC5572
:10CF3000284698F810A0FFF7A7FFDDED057A8DF8D9
:10CF40003100FCEEE77A9DF810208DF8332017EEC3
:10CF5000903A8DF8343006AB03CB1B88ADF83D30EA
:10CF60005C221B23CDE90032CDF83500CDF8391015
:10CF700009AABF2150468DED098A8DED0A8A8DEDF3
:10CF80000B8A8DF830408DF832B035F00FFA013F42
:10CF900017F0FF079ED10120C4E700BF000000008A
:10CFA0002DE9F04F0F7CA1B006468846032500EB23
:10CFB000070999F805400134E4B20323B4FBF3F305
:10CFC00003EB4303E41AE4B206EB8403D3F84C12F8
:10CFD00011B989F805400AE011A802F0B1F9DDF8AD
:10CFE00044A0BAF1030F08DCBAF1000FF1DA013DF9
:10CFF00015F0FF05DDD1012012E0AAF10402032A99
:10D00000F5D8384635F068F98346384636F068F882
:10D0100000F13602934506D2384634F0D9FB0020A1
:10D0200021B0BDE8F08F89F80540304698F810B07F
:10D03000FFF72AFFDDF848E0CDF80CE0DDF84CE022
:10D04000CDF810E0DDF850E0CDF814E0DDF854E064
:10D05000CDF818E0DDF858E0CDF81CE0DDF85CE034
:10D06000CDF820E0DDF860E0CDF824E03219DDF8FD
:10D0700064E01C9BCDF828E0DDF868E092F80AC077
:10D080009DF874109DF87520CDF82CE00E93DDF816
:10D090006CE01E9B8DF835008DF83C108DF83D201E
:10D0A000CDF830E08DF834408DF836A08DF837C0DB
:10D0B0002422CDF83E303623CDE90032C0212C2386
:10D0C00003AA584635F072F991E700007FB58A8BC4
:10D0D0000B464AF2B9518A4205465FD04AF2BA512C
:10D0E0008A4274D04AF2B8518A420BD1474A126838
:10D0F000D26A92F89C203AB13AF07AFF444A05216C
:10D1000034F046F9042479E0D3ED007AF5EEC07AE4
:10D11000F1EE10FAF6D49FED3F7AF4EEC77AF1EE15
:10D1200010FAEFDC93ED017ADFED3B6A1C6993EDB9
:10D13000030AB0EEC77AB4EEE67A93ED027AFCEE1B
:10D14000E77AB0EEC77AF1EE10FAB4EEE67A17EEAF
:10D15000903A54BF01260026F1EE10FA54BF012286
:10D160000022003C18BF012413F0FF0110D18DED07
:10D17000030A0292FCF77EFB9DED030A029A234606
:10D1800031462846FFF77CFD0028BBD0002435E05F
:10D19000134600943246FFF749FDF5E7D3ED007AD8
:10D1A000F5EEC07AF1EE10FAACD49FED1A7AF4EEF7
:10D1B000C77AF1EE10FAA5DCFCEEE77A17EE903AAA
:10D1C00013F0FF0108BFFF21FFF7DAFDDCE7D3ED25
:10D1D000007AF5EEC07AF1EE10FA93D49FED0D7A55
:10D1E000F4EEC77AF1EE10FA8CDCFCEEE77A17EE7B
:10D1F000904A14F0FF0404D1FFF70EFC204604B05F
:10D2000070BD2146FFF7F8FBC0E700BFA425002052
:10D21000044B0A0800007F4300000034F0B58BB0D7
:10D220000E4614460746FFF793FB543007C884E8C0
:10D23000070031463846FFF78BFB90ED057ADFEDAE
:10D24000267AB0EEC77AB4EEE77AF1EE10FA054628
:10D2500011D590ED067AB0EEC77AB4EEE77AF1EE2A
:10D2600010FA08D590ED077AB0EEC77AB4EEE77AF7
:10D27000F1EE10FA24D431463846FFF769FB016A13
:10D28000426A836AE869D5F814E0D5F818C00990B5
:10D2900001A8CDF804E0029103920491CDF814C0E6
:10D2A0000693079208930DF0CBFF98B1214601A891
:10D2B0000DF01AFE84ED000AC4ED010A84ED021A95
:10D2C00031463846FFF744FB00F1080120460FF0D5
:10D2D000B5FC01200BB0F0BD000000342DE9F04793
:10D2E0002DED048BACB0B0EE608A0546B0EE409AEE
:10D2F0000F46F0EE418A9046FCF7BCFADFED8B7AE0
:10D30000B0EEC87AB4EEE77AF1EE10FA4BD5B0EE93
:10D31000E87AB4EEE77AF1EE10FA44D523AC204671
:10D32000FBF7EEFDF8F7DEF92146F7F79DFF06461D
:10D3300058BB05F09FFB90F8383390F8F42233B1D6
:10D34000B02303FB020393F8D130012B07D84FF031
:10D35000B00909FB020090F8D130022B0BD83AF04B
:10D3600047FE734A032134F013F830462CB0BDEC6D
:10D37000048BBDE8F08705F07DFB90F8F43209FBE3
:10D380000300DC300FC884E80F00DDED257A9FED47
:10D39000691AB8EEE78ADDED267AF8EEE78A28EE1C
:10D3A000018A68EE818A04AA03A902A8F0EE680A3D
:10D3B000B0EE480A03F002FE064618B93AF018FE2D
:10D3C0005D4ACFE79FED5D7ADDED027A9FED5C8AE5
:10D3D000DFED5C8A8DED068A67EE877A24220021D4
:10D3E00011A8CDED057A8DED078A7EF0A7F89DEDA9
:10D3F000031ADDED040ADFF858A121EE281A68EEC1
:10D40000E00AB0EE480A11A80DF03AFF05A911A8EC
:10D410000DF06AFD242200211AA8CDED060A8DED3B
:10D42000071A8DED050A7EF089F8F8F75BF990EDA3
:10D43000810A8DED010AF8F755F929EE281AD0ED89
:10D44000820A9DED010A1AA80DF01AFF1AA923A855
:10D450000DF038FE05A923A80DF046FD4FF0000998
:10D460008DED050ACDED060A8DED071A95F82230EF
:10D470005FFA89F4A3427FF678AF1FB127FA04F36D
:10D48000DB071AD52B1993F92C32B3B1B8F1000F81
:10D490000DD021462846FCF777FC88B93AF0A8FD64
:10D4A000294A2346032133F073FF00265DE7214616
:10D4B0002846FCF7E3FA0028EBD109F10109D5E78A
:10D4C00008AA214628468DED088A8DED098A8DED42
:10D4D0000A8AFFF7A3FE20B93AF08AFD1B4A2346C9
:10D4E000E0E708A905A80FF059FB0BAA214628463A
:10D4F0008DED0B0ACDED0C0A8DED0D1AFCF752FAED
:10D500009AE807000EAB83E807001A462146284632
:10D51000FCF7F4F923AA214628468DED238A8DEDE8
:10D52000248A8DED258AFCF7FBF9C6E7000000345C
:10D53000284B0A0895BFD633434B0A0800007A44AB
:10D540000000000035FA8E3C584B0A086C4B0A0864
:10D55000C4F70908012070470120704743689868A4
:10D5600070470000406803689B6C184710B5054B76
:10D5700003600446806A10B103685B6898472046E0
:10D5800010BD00BF544C0A08406803685B6A184726
:10D5900033B46C46406884E80C0003689D6A94E8E4
:10D5A0000C00AC4602B030BC6047000010B5044629
:10D5B000FFF7DCFF2046FBF779FF204610BD000097
:10D5C000406809F0ADB80000406809F00BB90000F0
:10D5D0004068012309F006B94068002309F0DEB86D
:10D5E00090F84420D20705D590F8421000F12C02A3
:10D5F000FFF780B870470000F8B504461E460F4696
:10D600001546FEF777FF084B23600023E362236390
:10D61000636394F84430A76265F3410384F8436080
:10D6200084F844302046F8BD544C0A0810B50D4B20
:10D6300083630446806A036898221B690021984727
:10D6400070B1A06A036820221B690121984738B194
:10D65000A06A0368BDE810401B6901220221184737
:10D66000002010BDC5DC6A3F37B50446806A0368F8
:10D670006A469D6803210623A847D0B1BDF8002063
:10D68000BDF8041052BA95B249BAB5F5704F0BB255
:10D6900011D013F5805F0ED0BDF802305BBA9DB299
:10D6A000B5F5704F07D052425B42A287E187A4F8DC
:10D6B000403003B030BD0020FBE70000806A036803
:10D6C00001221B690221184730B585B00446FFF7D7
:10D6D000CBFF05462046FFF7F1FF6DB3B4F93C30B0
:10D6E00094ED0E0A06EE903AB4F93E3007EE103A89
:10D6F000B4F9403007EE903AF8EEE66AB8EEC77A31
:10D70000F8EEE77A01A8CDED016A8DED027ACDED54
:10D71000037A0FF0ADFA94F842102046FFF768F84C
:10D7200018B1022101A80FF039FB94F842200E2312
:10D7300001A92046FFF7CCF805B030BDFFF7C4BF04
:10D7400013B5806A036801AA9C680A210323A047D5
:10D7500038B10549032201A87DF096FEB0FA80F0A9
:10D76000400902B010BD00BF8C4B0A082DE9F843F8
:10D7700000252DED028BDFF888819FED5D8A044640
:10D780002E462F46A06A036811221B69002101372B
:10D79000984700287BD0D8F80090D9F82800036873
:10D7A00032215B689847A06A036860221B690121E7
:10D7B000984700286BD0A06A036801221B690221E8
:10D7C0009847002863D0D9F82800036832215B68A5
:10D7D00098472046FFF748FF002858D00135022F10
:10D7E000EDB256DDB4F93C309FED425A9FED426AEE
:10D7F00007EE903AF8EEE77AC5EE276AF0EEE66AB1
:10D80000F4EEC66AF1EE10FA41DDF4EEC86AF1EE0C
:10D8100010FA3CD5B4F93E30DFED385A07EE903AB5
:10D82000F8EEE77A85EEA77AB0EEC77AB4EEC67A5C
:10D83000F1EE10FA2BDDB4EEC87AF1EE10FA26D52F
:10D84000B4F9403005EE903AF8EEE55AC5EE257A87
:10D85000F0EEE77AF4EEC67AF1EE10FA17DDF4EEA8
:10D86000C87AF1EE10FA12D594ED0B6A76EE266ABC
:10D870000136C4ED0B6AD4ED0C6A36EE877A84ED7E
:10D880000C7A94ED0D7A77EE277AC4ED0D7A192F84
:10D8900002D0052E7FF476AFA06A036810221B69C0
:10D8A00000219847052E18D1D4ED0B6AF1EE047AC9
:10D8B00086EEA77A0120D4ED0C6A84ED0B7A86EE11
:10D8C000A77AD4ED0D6A84ED0C7A86EEA77A84ED02
:10D8D0000D7ABDEC028BBDE8F8834FF07E53052D29
:10D8E000E3622363636394BF00200120F1E700BF7C
:10D8F000CDCCAC3F00002E443333333F00002244F4
:10D90000A4250020F0B50446806A036885B05B69F1
:10D910009847054648B9504B50491B6898690368B9
:10D920001B689847284605B0F0BD03689B68984778
:10D93000A06A03680A21DB6A9847A06A03689B69AA
:10D94000984760B9444B46491B68986903681B684F
:10D9500098472B682846DB6898470025E2E7204671
:10D96000FFF7EEFE0028F4D02046FFF7FFFE30B9A7
:10D97000394B3C491B68986903681B68E8E72046F7
:10D98000FFF754FE0028E4D0A06A0368DB699847DB
:10D9900030B9314B34491B68986903681B68D7E775
:10D9A00094F84430A06A43F0010384F844300368DB
:10D9B0000321DB6A98472B682846DB689847236871
:10D9C00020469B689847A06A036807215B6A9847CE
:10D9D000A06A03689B6A984704F142020146204608
:10D9E000FEF7D6FE054600289CD0A06A94F84210A7
:10D9F000036801919B6A9847019902462046FEF709
:10DA0000CBFE94F8432094F842102046FEF7FAFE2D
:10DA100094F844309B0705D594F842100122204623
:10DA2000FEF7CEFEA06A029403681E6A0F4B0393B2
:10DA300004AB13E90C0043F21541B047064BA06A52
:10DA40001B689E6933681F6803689B6A984708498A
:10DA500002463046B84765E7A4250020904B0A08E7
:10DA6000B64B0A08DC4B0A08014C0A083DD70108EE
:10DA70002F4C0A0810B5084B0360044600230868C1
:10DA800060600B60037A03F00703022B02D1C02110
:10DA900008F074FF204610BD6C4C0A0810B5044B0A
:10DAA000044640F8043BFAF745FA204610BD00BF93
:10DAB0006C4C0A0810B50446FFF7F0FF2046FBF750
:10DAC000F5FC204610BD0000F7B503680E4617466A
:10DAD0001BB90024204603B0F0BD002202600820DC
:10DAE0000193FBF7DBFC054610B101A9FFF7C2FF6C
:10DAF00001A8FAF71FFA002DEBD04820FBF7CEFC67
:10DB000004460028E5D029463B463246FFF774FD1F
:10DB10002046FFF7F7FE05460028DBD123682046A4
:10DB20005B6898472C46D5E790F82D100022FEF749
:10DB3000E1BD0000F0B50446806A036889B05B6A05
:10DB4000984703689B689847A06A03680A219B6C02
:10DB50009847A06A01230DF11702002108F042FE48
:10DB6000002838D09DF81730082B34D14E4F0525AA
:10DB700000230122A06A322108F010FE3B689B6A54
:10DB80001A68526840B90A2118469047013D15F0BD
:10DB9000FF05EDD145481CE018461421904706AE1C
:10DBA000FF238DF81830A06A01233246322108F095
:10DBB00019FE0028EAD09DF8183013F00103E5D1D2
:10DBC000A06A03930822322108F0E8FD039B58B9AC
:10DBD000374852F0C1F9A06A03685B6A9847036846
:10DBE000DB68984700255CE0A06A03931A4634215D
:10DBF00008F0D4FD0028EBD0039BA06A2422412129
:10DC000008F0CCFD0028E3D0039BA06A0822312154
:10DC100008F0C4FD0028DBD0A06A036803219B6CD8
:10DC20009847A06A03685B6A98470368DB6898476F
:10DC3000A06A102108F074FDA36A04F12D0299680E
:10DC40002046FEF7A5FD054658B3A36A94F82D10AB
:10DC50009A682046FEF7A0FDA36A16481A7A597AF8
:10DC600000919B681449D20852F076F994F82C2060
:10DC700094F82D102046FEF7C5FD94F82E302BB1F8
:10DC800094F82D1001222046FEF79AFDA06A036841
:10DC90009F6A0A4B0694079396E80C0042F21071B3
:10DCA000B847284609B0F0BDA4250020FC4C0A085E
:10DCB0009C4C0A08D34C0A08CB4C0A0849DD0108E1
:10DCC00010B586B004460123806A0DF103021021CD
:10DCD00008F088FD98B39DF80330DB072FD5A06AC4
:10DCE000062301AA112108F07DFD40B3BDF90430DF
:10DCF0009FED146A94F82D2006EE903ABDF9063097
:10DD000007EE103ABDF808305B421BB207EE903ABE
:10DD1000F8EEE66AB8EEC77AF8EEE77A66EE866A5B
:10DD200027EE067A67EE867A0A2303A92046CDED10
:10DD3000036A8DED047ACDED057AFEF7C9FD06B0D4
:10DD400010BD00BF85EBC13FFFF7BABFF7B5036851
:10DD50000D4616461BB90024204603B0F0BD00272F
:10DD600007603020CDE90073FBF798FB044650B103
:10DD7000FEF7C0FB0E4B2360019BA362019784F862
:10DD80002C6084F82E5001A8FAF7D4F86846FAF708
:10DD9000D1F8002CDFD02046FFF7CCFE0546002846
:10DDA000DAD1236820465B6898472C46D4E700BF49
:10DDB000284D0A0810B5044B044640F8283BFAF7F2
:10DDC000B9F8204610BD00BF284D0A0810B504461A
:10DDD000FFF7F0FF2046FBF769FB204610BD00006F
:10DDE00090F831100022FEF785BC000010B500232A
:10DDF00004460122806A0A2108F0D0FC10B90123F0
:10DE000084F8323010BD0000F0B50446806A036823
:10DE100089B05B6A984703689B689847A06A036863
:10DE20000A219B6C9847012200230B21A06A08F06D
:10DE3000B5FC514B1F68B86A03680A215B689847B4
:10DE4000A06A01230DF11702002108F0CBFC002885
:10DE500035D09DF81730102B31D105250023012234
:10DE60000B21A06A08F09AFCBB6A1A680A21526862
:10DE700038B918469047013D15F0FF05EED13F48EF
:10DE80001BE01846904706AEFF238DF81830A06AB5
:10DE9000012332460B2108F0A5FC0028EBD09DF8A9
:10DEA000183013F00103E6D1A06A03932422412124
:10DEB00008F074FC039B58B9314852F04DF8A06A41
:10DEC00003685B6A98470368DB68984700254FE062
:10DED000A06AC022422108F061FC0028ECD0A06AB0
:10DEE000036803219B6C98472046FFF77FFFA06AD9
:10DEF00003685B6A98470368DB689847A06A0A2151
:10DF000008F00EFCA36A04F1310299682046FEF77E
:10DF10003FFC054660B3A36A94F831109A68204626
:10DF2000FEF73AFCA36A17481A7A597A00919B685F
:10DF30001549D20852F010F894F8302094F83110B6
:10DF40002046FEF75FFC94F833302BB194F8311083
:10DF500001222046FEF734FCA06A03689F6A0B4B3F
:10DF60000694079396E80C0042F21071B847E062FD
:10DF7000284609B0F0BD00BFA42500206F4D0A0857
:10DF8000384D0A08D34C0A08674D0A085DE00108BD
:10DF900030B590F8323087B004463BB1002380F8AA
:10DFA000323007B0BDE83040FFF720BF806A06235B
:10DFB00001AA032108F016FC002849D02046FFF7EB
:10DFC00015FFA06AE16A036842F21072DB6A9847A3
:10DFD000BDF8042041F2D64013189BB242F6AC11B2
:10DFE0008B4235D8BDF90610814231DC194B99427C
:10DFF0002EDBBDF90800BDF8083042F28E05A842BC
:10E0000026DC154DA84223DB12B207EE102AB8EE2B
:10E01000C77AF0EE086A07EE901A27EE267A5B427E
:10E020001BB28DED037AB8EEE77A07EE903AF8EE80
:10E03000E77A27EE267A67EEA67A94F831208DEDFE
:10E04000047A0A2303A92046CDED057AFEF740FCA9
:10E0500007B030BD2AEBFFFF72DFFFFFFFF798BF6D
:10E06000F7B503680D4616461BB90024204603B0D9
:10E07000F0BD002707603420CDE90073FBF70EFAEE
:10E08000044650B1FEF736FA0E4B2360019BA362A3
:10E09000019784F8306084F8335001A8F9F74AFFFB
:10E0A0006846F9F747FF002CDFD02046FFF7ACFEAB
:10E0B00005460028DAD1236820465B6898472C463D
:10E0C000D4E700BF984D0A0810B5044B044640F849
:10E0D000283BF9F72FFF204610BD00BF984D0A08D6
:10E0E00010B50446FFF7F0FF2046FBF7DFF92046A6
:10E0F00010BD000090F82C100022FEF7FBBA0000C3
:10E100007FB50446806A03685B6A984703689B682A
:10E110009847A06A037A03F00703022B02D1C021BB
:10E1200008F02CFCA06A03680A219B6C9847A06A3F
:10E1300001230DF107020F2108F054FB00286BD0DA
:10E140009DF807303D2B67D10A220521A06A08F00F
:10E15000CFFA0123FC222021A06A08F01FFB012333
:10E1600000222121A06A08F019FB012300222221AC
:10E17000A06A08F013FB01230C222321A06A08F0F7
:10E180000DFB402201232421A06A08F007FBA06AAE
:10E19000036803219B6C9847A06A03685B6A9847F1
:10E1A0000368DB689847A06A082108F0B9FAA36AF7
:10E1B00004F12C0299682046FEF7EAFA0546002889
:10E1C00032D0A36A94F82C109A682046FEF7E4FA3D
:10E1D000A36A94F82C209968154851F0BDFE94F874
:10E1E0002E2094F82C102046FEF70CFB94F82D30CE
:10E1F0002BB194F82C1001222046FEF7E1FAA06A18
:10E20000029403689E6A0B4B039304AB13E90C0062
:10E2100043F2D401B04707E0A06A03685B6A9847FD
:10E220000368DB6898470025284604B070BD00BF2E
:10E23000A84D0A08C1E2010810B586B004460123C2
:10E24000806A0DF10302272108F0CCFA88B39DF80B
:10E2500003301B072DD5A06A062301AA282108F048
:10E26000C1FA30B3BDF904309FED146A94F82C2044
:10E2700006EE903ABDF9063007EE103ABDF90830C7
:10E2800007EE903AF8EEE66AB8EEC77AF8EEE77A6B
:10E2900066EE866A27EE067A67EE867A0A2303A977
:10E2A0002046CDED036A8DED047ACDED057AFEF7BB
:10E2B0000FFBA06A08F0BAFA06B010BDF1A9153E2E
:10E2C000FFF7BABFF7B503680E4615461BB9002421
:10E2D000204603B0F0BD0027076030200193FBF714
:10E2E000DDF8044650B1FEF705F90D4B2360019BA4
:10E2F000A362019784F82D6084F82E5001A8F9F7E5
:10E3000019FE002CE3D02046FFF7FAFE0546002850
:10E31000DED1236820465B6898472C46D8E700BFCB
:10E32000D84D0A0810B5044B044640F8283BF9F7CD
:10E3300001FE204610BD00BFD84D0A0810B50446A6
:10E34000FFF7F0FF2046FBF7B1F8204610BD0000B4
:10E3500090F82D100022FEF7CDB90000F8B5044664
:10E360000D4617461E46FEF7C5F8084B23602B687E
:10E37000A362002200232A6084F82E702363636363
:10E38000A36384F84E602046F8BD00BF184E0A080B
:10E39000F0B50446806A036885B05B6A98470368F5
:10E3A0009B689847A06A03680A219B6C9847A06AFB
:10E3B00001230DF10702202108F014FA002866D08D
:10E3C0009DF80730062B62D1802200230821A06A25
:10E3D00008F0E4F9334B1E68B06A03680A215B68F1
